:020000040800F2
:1000000000060020E1010008E3010008E301000808
:10001000E3010008E3010008E3010008E301000830
:10002000E3010008E3010008E3010008692F00086C
:10003000E3010008E3010008E3010008E301000810
:10004000E3010008E3010008E3010008E301000800
:10005000E3010008E301000811320008393200080A
:100060006132000889320008B1320008E30100085B
:10007000E3010008E3010008E3010008E3010008D0
:10008000E3010008E3010008E3010008E3010008C0
:10009000E3010008E3010008E3010008D932000889
:1000A000E3010008E3010008E3010008E3010008A0
:1000B000AD330008E3010008E3010008E301000894
:1000C000E3010008E3010008E3010008E301000880
:1000D000E3010008E3010008E3010008E301000870
:1000E0003D330008E3010008E3010008E3010008D4
:1000F000E3010008E3010008E3010008E301000850
:10010000E3010008E3010008E3010008E30100083F
:10011000E3010008E3010008E3010008E30100082F
:10012000E3010008E3010008E3010008E30100081F
:10013000E3010008E3010008E3010008E30100080F
:10014000E3010008E3010008E30100081D2700089F
:10015000E3010008E3010008E3010008E3010008EF
:10016000E3010008E3010008E3010008E3010008DF
:10017000E3010008E3010008E3010008E3010008CF
:10018000E3010008E3010008E3010008E3010008BF
:10019000E3010008E3010008E3010008E3010008AF
:1001A000E3010008E3010008E3010008E30100089F
:1001B000E3010008E3010008E3010008E30100088F
:1001C000E3010008E3010008E3010008E30100087F
:1001D000E3010008E3010008E3010008E30100086F
:1001E00002E000F000F8FEE772B6374880F30888B6
:1001F000364880F3098836483649086040F20000E6
:10020000CCF200004EF63471CEF200010860BFF36C
:100210004F8FBFF36F8F40F20000C0F2F0004EF638
:100220008851CEF200010860BFF34F8FBFF36F8F8C
:100230004FF00000E1EE100A4EF63C71CEF20001E4
:100240000860062080F31488BFF36F8F01F02EFF43
:1002500002F028FE4FF055301F491B4A91423CBF27
:1002600041F8040BFAE71D49184A91423CBF41F896
:10027000040BFAE71A491B4A1B4B9A423EBF51F83E
:10028000040B42F8040BF8E700201849184A914281
:100290003CBF41F8040BFAE701F00CFF02F056FEF8
:1002A000144C154DAC4203DA54F8041B8847F9E7A7
:1002B00000F042F8114C124DAC4203DA54F8041B22
:1002C0008847F9E701F0F4BE000600200022002074
:1002D0000000000808ED00E00000002000060020FB
:1002E0007037000800220020402200204022002019
:1002F000602E0020E0010008E0010008E001000895
:10030000E00100082DE9F04F2DED108AC1F80CD066
:10031000C3689D46BDEC108ABDE8F08F002383F3CF
:1003200011882846A047002001F074FAFEE701F08A
:1003300003FA00DFFEE7000038B500F0BFFB01F074
:1003400085FE054601F0A8FE0446C8B90E4B9D4245
:1003500018D001339D4218BF044641F2883504BFCE
:1003600001240025002001F07BFE0CB100F074F8A0
:1003700000F002FD284600F0C3F800F06DF8F9E740
:100380000025EFE70546EDE7010007B008B500F0EE
:1003900067FBA0F120035842584108BD07B541F260
:1003A0001203022101A8ADF8043000F077FB03B07E
:1003B0005DF804FB38B5302383F3118817480368D0
:1003C0000BB101F0F3FA164A144800234FF47A7186
:1003D00001F0E2FA002383F31188124C236813B171
:1003E0002368013B2360636813B16368013B63606A
:1003F0000D4D2B7833B963687BB9022000F026FCE1
:10040000322363602B78032B07D163682BB902205A
:1004100000F01CFC4FF47A73636038BD402200206A
:10042000B50300086023002058220020084B1870F4
:1004300003280CD8DFE800F008050208022000F0CD
:10044000FDBB022000F0F0BB024B00225A60704757
:100450005822002060230020244B254A10B51C465A
:100460001968013140D004339342F9D16268214BBD
:100470009A4239D9204B9B6803F1006303F580331E
:100480009A4231D2002000F033FB0220FFF7CEFF6A
:100490001A4B1A6C00221A64196E1A66196E596C7E
:1004A0005A64596E5A665A6E5A6942F080025A610D
:1004B0005A6922F080025A615A691A6942F0005260
:1004C0001A611A6922F000521A611B6972B64FF064
:1004D000E0233021C3F8084DD4E9003281F31188BC
:1004E0009D4683F30888104710BD00BF0000010837
:1004F00020000108FFFF0008002200200038024011
:100500002DE9F04F93B0AA4B00902022FF210AA8BA
:100510009D6800F0DBFBA74A1378A3B9A648012128
:1005200003601170302383F3118803680BB101F06D
:100530003DFAA24AA04800234FF47A7101F02CFA48
:10054000002383F31188009B13B19D4B009A1A601E
:100550009C4A009C1378032B1EBF00231370984AFB
:100560004FF0000A18BF5360D3465646D1460120CB
:1005700000F064FB24B1924B1B68002B00F0118249
:10058000002000F06DFA0390039B002BF2DB0120AA
:1005900000F04AFB039B213B162BE8D801A252F83E
:1005A00023F000BF0106000829060008BD06000868
:1005B0006F0500086F0500086F0500084707000871
:1005C000170900083108000893080008BB08000854
:1005D000E10800086F050008F30800086F0500082F
:1005E00065090008A10600086F050008A9090008B0
:1005F0000D060008A10600086F0500089308000812
:100600000220FFF7C3FE002840F0F581009B022185
:10061000BAF1000F08BF1C4605A841F21233ADF82D
:10062000143000F03BFAA2E74FF47A7000F018FAA9
:10063000071EEBDB0220FFF7A9FE0028E6D0013FF2
:10064000052F00F2DA81DFE807F0030A0D101336F8
:1006500005230593042105A800F020FA17E054486B
:100660000421F9E758480421F6E758480421F3E744
:100670004FF01C08404600F03DFA08F104080590D0
:10068000042105A800F00AFAB8F12C0FF2D10120DC
:1006900000FA07F747EA0B0B5FFA8BFB4FF00009F4
:1006A00000F060FB26B10BF00B030B2B08BF0024FE
:1006B000FFF774FE5BE746480421CDE7002EA5D086
:1006C0000BF00B030B2BA1D10220FFF75FFE0746B7
:1006D00000289BD0012000F00BFA0220FFF7A6FEB5
:1006E00000261FFA86F8404600F012FA044690B140
:1006F0000021404600F01CFA01360028F1D1BA462C
:10070000044641F21213022105A8ADF814303E460A
:1007100000F0C4F92BE70120FFF788FE2546244BA3
:100720009B68AB4207D9284600F0E4F9013040F05D
:1007300067810435F3E7234B00251D70204BBA4633
:100740005D603E46ACE7002E3FF460AF0BF00B035C
:100750000B2B7FF45BAF0220FFF768FE322000F026
:100760007FF9B0F10008FFF651AF18F003077FF4EE
:100770004DAF0F4A926808EB050393423FF646AF30
:10078000B8F5807F3FF742AF124B0193B84523DDA8
:100790004FF47A7000F064F90390039A002AFFF690
:1007A00035AF019B039A03F8012B0137EDE700BF3A
:1007B000002200205C23002040220020B503000816
:1007C000602300205822002004220020082200205C
:1007D0000C2200205C220020C820FFF7D7FD07462E
:1007E00000283FF413AF1F2D11D8C5F12002424558
:1007F0000AAB25F0030028BF424683490192184402
:1008000000F03EFA019A8048FF2100F05FFA4FEABB
:10081000A8037D490193C8F38702284600F05EFAD9
:10082000064600283FF46DAF019B05EB830537E7D3
:100830000220FFF7ABFD00283FF4E8AE00F0A4F97A
:1008400000283FF4E3AE0027B846704B9B68BB42DC
:1008500018D91F2F11D80A9B01330ED027F003039C
:1008600012AA134453F8203C05934046042205A9DC
:1008700000F0ACFA04378046E7E7384600F03AF972
:100880000590F2E7CDF81480042105A800F006F9E0
:1008900006E70023642104A8049300F0F5F800287B
:1008A0007FF4B4AE0220FFF771FD00283FF4AEAE36
:1008B000049800F051F90590E6E70023642104A8AC
:1008C000049300F0E1F800287FF4A0AE0220FFF7C7
:1008D0005DFD00283FF49AAE049800F04DF9EAE778
:1008E0000220FFF753FD00283FF490AE00F05CF9C2
:1008F000E1E70220FFF74AFD00283FF487AE05A993
:10090000142000F057F904210746049004A800F0D1
:10091000C5F83946B9E7322000F0A2F8071EFFF605
:1009200075AEBB077FF472AE384A926807EB0903D5
:1009300093423FF66BAE0220FFF728FD00283FF4FC
:1009400065AE27F003074F44B9453FF4A9AE4846CA
:1009500000F0D0F80421059005A800F09FF809F1F7
:100960000409F1E74FF47A70FFF710FD00283FF417
:100970004DAE00F009F9002844D00A9B01330BD09A
:1009800008220AA9002000F0A9F900283AD0202264
:10099000FF210AA800F09AF9FFF700FD1C4800F0BB
:1009A0003FFF13B0BDE8F08F002E3FF42FAE0BF0E9
:1009B0000B030B2B7FF42AAE0023642105A80593BB
:1009C00000F062F8074600287FF420AE0220FFF70F
:1009D000DDFC804600283FF419AEFFF7DFFC41F252
:1009E000883000F01DFF059800F0EEF9464600F053
:1009F000B9F93C46BBE5064652E64FF0000905E66C
:100A0000BA467EE637467CE65C22002000220020C3
:100A1000A086010070B50F4B1B780133DBB2012BB0
:100A20000C4611D80C4D29684FF47A730E6AA2FB5C
:100A30000332014622462846B047844204D1074B80
:100A400000221A70012070BD4FF4FA7000F0E8FE29
:100A50000020F8E710220020082600209423002020
:100A600007B50023024601210DF107008DF807307C
:100A7000FFF7D0FF20B19DF8070003B05DF804FB3D
:100A80004FF0FF30F9E700000A4608B50421FFF7F0
:100A9000C1FF80F00100C0B2404208BD30B4054C37
:100AA0002368DD69044B0A46AC460146204630BC4B
:100AB000604700BF08260020A086010070B501F045
:100AC000CBF9094E094D30800024286833888342D1
:100AD00008D901F0BBF92B6804440133B4F5803F19
:100AE0002B60F2D370BD00BF962300206823002046
:100AF00001F060BA00F1006000F5803000687047D6
:100B000000F10060920000F5803001F0EBB90000C8
:100B1000054B1A68054B1B889B1A834202D9104467
:100B200001F094B90020704768230020962300202C
:100B300038B5084D044629B128682044BDE838403E
:100B400001F0A4B92868204401F088F90028F3D006
:100B500038BD00BF6823002010F003030AD1B0F5B0
:100B6000047F05D200F10050A0F51040D0F8003805
:100B7000184670470023FBE700F10050A0F5104035
:100B8000D0F8100A70470000064991F8243033B1BC
:100B90000023086A81F824300822FFF7B1BF012042
:100BA000704700BF6C230020014B1868704700BFDE
:100BB000002004E070B5194B1D68194B0138C5F3CE
:100BC0000B0408442D0C04221E88A6420BD15C683D
:100BD0000A46013C824213460FD214F9016F4EB10E
:100BE00002F8016BF6E7013A03F10803ECD1814208
:100BF0000B4602D22C2203F8012B0A4A0524168840
:100C0000AE4204D1984284BF967803F8016B013C50
:100C100002F10402F3D1581A70BD00BF002004E0B5
:100C2000903400087C340008022802BF024B4FF4C5
:100C300000129A61704700BF00040240022802BF00
:100C4000014B20229A61704700040240022801BF34
:100C5000024A536983F02003536170470004024045
:100C600070B504464FF47A764CB1412C254628BF26
:100C7000412506FB05F000F0D3FD641BF4E770BDD1
:100C800010B50023934203D0CC5CC4540133F9E780
:100C900010BD000010B5013810F9013F3BB191F9CA
:100CA00000409C4203D11AB10131013AF4E71AB174
:100CB00091F90020981A10BD1046FCE70346024641
:100CC000D01A12F9011B0029FAD1704702440346D9
:100CD000934202D003F8011BFAE770472DE9F8436D
:100CE0001F4D144695F824200746884652BBDFF86E
:100CF00070909CB395F824302BB92022FF214846F0
:100D00002F62FFF7E3FF95F82400C0F10802A2422A
:100D100028BF2246D6B24146920005EB8000FFF77D
:100D2000AFFF95F82430A41B1E44F6B2082E1744DA
:100D30009044E4B285F82460DBD1FFF725FF00285A
:100D4000D7D108E02B6A03EB82038342CFD0FFF7B1
:100D50001BFF0028CBD10020BDE8F8830120FBE772
:100D60006C230020024B1A78024B1A70704700BFA8
:100D7000942300201022002010B5104C104800F0E1
:100D8000B5F821460E4800F0DDF82468626DD2F80F
:100D9000043843F00203C2F804384FF47A70FFF7C6
:100DA0005FFF0849204600F0D3F9626DD2F804389D
:100DB00023F00203C2F8043810BD00BF5C35000800
:100DC00008260020643500087047000030B5094D42
:100DD0000A4491420DD011F8013B5840082340F3DA
:100DE0000004013B2C4013F0FF0384EA5000F6D1CD
:100DF000EFE730BD2083B8ED02684368114301601E
:100E000003B118477047000013B5446BD4F894340D
:100E10001A681178042915D1217C022912D1197977
:100E2000128901238B4013420CD101A904F14C001B
:100E300001F0F4FED4F89444019B21790246206825
:100E400000F0D0F902B010BD143001F077BE000000
:100E50004FF0FF33143001F071BE00004C3001F050
:100E600049BF00004FF0FF334C3001F043BF00009A
:100E7000143001F045BE00004FF0FF31143001F096
:100E80003FBE00004C3001F015BF00004FF0FF32B4
:100E90004C3001F00FBF00000020704710B5D0F8B3
:100EA00094341A6811780429044617D1017C022968
:100EB00014D15979528901238B4013420ED1143039
:100EC00001F0D8FD024648B1D4F894444FF4807341
:100ED00061792068BDE8104000F072B910BD0000D3
:100EE000406BFFF7DBBF0000704700007FB5124B7F
:100EF000036000234360C0E90233012502260F4B43
:100F0000057404460290019300F18402294600967C
:100F10004FF48073143001F089FD094B0294CDE940
:100F2000006304F523724FF48073294604F14C00EA
:100F300001F050FE04B070BDB0340008E10E0008AE
:100F4000090E00080B68302282F311880A7903EB3E
:100F5000820290614A79093243F822008A7912B1FB
:100F600003EB820398610223C0F8941403740020F9
:100F700080F311887047000038B5037F044613B131
:100F800090F85430ABB9201D01250221FFF734FF42
:100F900004F1140025776FF0010100F069FC84F87A
:100FA000545004F14C006FF00101BDE8384000F0EE
:100FB0005FBC38BD10B5012104460430FFF71CFFAB
:100FC0000023237784F8543010BD000038B5044660
:100FD0000025143001F042FD04F14C00257701F0AA
:100FE00011FE201D84F854500121FFF705FF204613
:100FF000BDE83840FFF752BF90F8443003F060037B
:10100000202B07D190F84520212A4FF0000303D868
:101010001F2A06D800207047222AFBD1C0E90E33D0
:1010200003E0034A82630722C2630364012070471E
:101030001122002037B5D0F894341A6811780429A9
:1010400004461AD1017C022917D11979128901238A
:101050008B40134211D100F14C05284601F092FE5D
:1010600058B101A9284601F0D9FDD4F89444019B58
:1010700021790246206800F0B5F803B030BD0000C9
:10108000F0B500EB810385B09E6904460D46FEB1C4
:10109000302383F3118804EB8507301D0821FFF707
:1010A000ABFEFB685B691B6806F14C001BB101904D
:1010B00001F0C2FD019803A901F0B0FD024648B15C
:1010C000039B2946204600F08DF8002383F3118806
:1010D00005B0F0BDFB685A691268002AF5D01B8A7A
:1010E000013B1340F1D104F14402EAE7093138B57C
:1010F00050F82140DCB1302383F31188D4F89424D4
:101100001368527903EB8203DB689B695D6845B124
:1011100004216018FFF770FE294604F1140001F065
:10112000B3FC2046FFF7BAFE002383F3118838BDD5
:101130007047000001F012B8012303700023C0E9DA
:101140000133C36183620362C36243620363704716
:1011500038B50446302383F311880025C0E90355D0
:10116000C0E90555416001F009F80223237085F3B9
:101170001188284638BD000070B500EB8103054694
:101180005069DA600E46144618B110220021FFF7AC
:101190009DFDA06918B110220021FFF797FD31468F
:1011A0002846BDE8704001F0B3B80000826802F044
:1011B000011282600022C0E90422826101F034B988
:1011C000F0B400EB81044789E4680125A4698D40EF
:1011D0003D43458123600023A2606360F0BC01F0C1
:1011E0004FB90000F0B400EB81040789E4680125E1
:1011F00064698D403D43058123600023A2606360E4
:10120000F0BC01F0C9B9000070B502230025044606
:101210000370C0E90255C0E90455C564856180F8D2
:10122000345001F011F863681B6823B12946204649
:10123000BDE87040184770BD0378052B10B5044613
:101240000AD080F850300523037043681B680BB147
:10125000042198470023A36010BD000001780529F0
:1012600006D190F85020436802701B6803B11847FC
:101270007047000070B590F83430044613B1002375
:1012800080F8343004F14402204601F0EFF863683E
:101290009B68B3B994F8443013F0600535D0002151
:1012A000204601F08FFB0021204601F081FB63689E
:1012B0001B6813B1062120469847062384F8343072
:1012C00070BD204698470028E4D0B4F84A30E26B5D
:1012D0009A4288BFE36394F94430E56B002B4FF0EA
:1012E000300380F20381002D00F0F280092284F89F
:1012F000342083F311880021D4E90E232046FFF720
:1013000071FF002383F31188DAE794F8452003F096
:101310007F0343EA022340F20232934200F0C58089
:1013200021D8B3F5807F48D00DD8012B3FD0022BB8
:1013300000F09380002BB2D104F14C02A263022290
:10134000E2632364C1E7B3F5817F00F09B80B3F5CE
:10135000407FA4D194F84630012BA0D1B4F84C3092
:1013600043F0020332E0B3F5006F4DD017D8B3F568
:10137000A06F31D0A3F5C063012B90D8636894F8B7
:1013800046205E6894F84710B4F848302046B047CD
:10139000002884D04368A3630368E3631AE0B3F5CD
:1013A000106F36D040F6024293427FF478AF5C4B28
:1013B000A3630223E3630023C3E794F84630012BC1
:1013C0007FF46DAFB4F84C3023F00203C4E90E553E
:1013D000A4F84C30256478E7B4F84430B3F5A06F36
:1013E0000ED194F8463084F84E30204600F084FF49
:1013F00063681B6813B101212046984703232370BB
:101400000023C4E90E339CE704F14F03A3630123D7
:10141000C3E72378042B10D1302383F311882046AF
:10142000FFF7C4FE85F311880321636884F84F50E9
:1014300021701B680BB12046984794F84630002B6A
:10144000DED084F84F300423237063681B68002BC0
:10145000D6D0022120469847D2E794F848301D069E
:1014600003F00F0120460AD500F0F2FF012804D056
:1014700002287FF414AF2B4B9AE72B4B98E700F030
:10148000D9FFF3E794F84630002B7FF408AF94F8C7
:10149000483013F00F01B3D01A06204602D501F0F0
:1014A000A5FAADE701F098FAAAE794F84630002BC8
:1014B0007FF4F5AE94F8483013F00F01A0D01B066E
:1014C000204602D501F07EFA9AE701F071FA97E71B
:1014D000142284F8342083F311882B462A462946A7
:1014E0002046FFF76DFE85F31188E9E65DB1152210
:1014F00084F8342083F311880021D4E90E23204698
:10150000FFF75EFEFDE60B2284F8342083F311889A
:101510002B462A4629462046FFF764FEE3E700BF34
:10152000E0340008D8340008DC34000838B590F8FE
:1015300034300446002B3ED0063BDAB20F2A34D8B2
:101540000F2B32D8DFE803F0373131082232313146
:101550003131313131313737C56BB0F84A309D42C6
:1015600014D2C3681B8AB5FBF3F203FB12556DB9A5
:10157000302383F311882B462A462946FFF732FE93
:1015800085F311880A2384F834300EE0142384F89C
:101590003430302383F3118800231A46194620463D
:1015A000FFF70EFE002383F3118838BD036C03B1EF
:1015B00098470023E7E70021204601F003FA0021C5
:1015C000204601F0F5F963681B6813B10621204637
:1015D00098470623D7E7000010B590F83430142B55
:1015E000044629D017D8062B05D001D81BB110BD51
:1015F000093B022BFBD80021204601F0E3F9002132
:10160000204601F0D5F963681B6813B10621204616
:101610009847062319E0152BE9D10B2380F83430C5
:10162000302383F3118800231A461946FFF7DAFDA9
:10163000002383F31188DAE7C3689B695B68002B9A
:10164000D5D1036C03B19847002384F83430CEE73A
:1016500000230375826803691B6899689142FBD275
:101660005A68036042601060586070470023037539
:10167000826803691B6899689142FBD85A680360C5
:10168000426010605860704708B50846302383F305
:1016900011880B7D032B05D0042B0DD02BB983F3C0
:1016A000118808BD8B6900221A604FF0FF338361F7
:1016B000FFF7CEFF0023F2E7D1E9003213605A6052
:1016C000F3E70000FFF7C4BF054BD9680875186839
:1016D00002681A60536001220275D860FEF712BEDC
:1016E0009823002030B50C4BDD684B1C87B00446B6
:1016F0000FD02B46094A684600F04EF92046FFF706
:10170000E3FF009B13B1684600F050F9A86907B0E9
:1017100030BDFFF7D9FFF9E79823002089160008AC
:10172000044B1A68DB6890689B68984294BF00205D
:101730000120704798230020084B10B51C68D8681A
:1017400022681A60536001222275DC60FFF78EFF69
:1017500001462046BDE81040FEF7D4BD9823002086
:1017600038B5074C074908480123002523706560F8
:1017700001F040FB0223237085F3118838BD00BFC0
:1017800000260020E83400089823002000F044B927
:10179000034A516853685B1A9842FBD8704700BFF0
:1017A000001000E08B60022308618B8208467047BE
:1017B0008368A3F1840243F8142C026943F8442C93
:1017C000426943F8402C094A43F8242CC26843F884
:1017D000182C022203F80C2C002203F80B2C044ACC
:1017E00043F8102CA3F12000704700BF1D03000830
:1017F0009823002008B5FFF7DBFFBDE80840FFF79E
:1018000061BF0000024BDB6898610F20FFF75CBFEF
:1018100098230020302383F31188FFF7F3BF0000E3
:1018200008B50146302383F311880820FFF75AFFDB
:10183000002383F3118808BD064BDB6839B1426889
:1018400018605A60136043600420FFF74BBF4FF0ED
:10185000FF307047982300200368984206D01A682A
:101860000260506099611846FFF72CBF7047000076
:1018700038B504460D462068844200D138BD03685F
:1018800023605C608561FFF71DFFF4E710B5036816
:101890009C68A2420CD85C688A600B604C60216036
:1018A000596099688A1A9A604FF0FF33836010BDBF
:1018B0001B68121BECE700000A2938BF0A2170B52B
:1018C00004460D460A26601901F08EFA01F07AFAF4
:1018D000041BA54203D8751C2E460446F3E70A2EC6
:1018E00004D9BDE87040012001F0C4BA70BD000009
:1018F000F8B5144B0D46D96103F1100141600A2A75
:101900001969826038BF0A22016048601861A8180E
:10191000144601F05BFA0A2701F054FA431BA34274
:10192000064606D37C1C281901F05EFA2746354688
:10193000F2E70A2F04D9BDE8F840012001F09ABA75
:10194000F8BD00BF98230020F8B506460D4601F00B
:1019500039FA0F4A134653F8107F9F4206D12A46A0
:1019600001463046BDE8F840FFF7C2BFD169BB6809
:10197000441A2C1928BF2C46A34202D92946FFF746
:101980009BFF224631460348BDE8F840FFF77EBF83
:1019900098230020A823002010B4C0E903230023CB
:1019A0005DF8044B4361FFF7CFBF000010B5194C41
:1019B000236998420DD0D0E90032816813605A60E3
:1019C0009A680A449A60002303604FF0FF33A361D2
:1019D00010BD2346026843F8102F536000220260B6
:1019E00022699A4203D1BDE8104001F0F7B993682B
:1019F00081680B44936001F0E5F92269E16992681E
:101A0000441AA242E4D91144BDE81040091AFFF774
:101A100053BF00BF982300202DE9F047DFF8BC80BA
:101A200008F110072C4ED8F8105001F0CBF9D8F877
:101A30001C40AA68031B9A423ED81444D5E90032E0
:101A40004FF00009C8F81C4013605A60C5F80090B8
:101A5000D8F81030B34201D101F0C0F989F31188F0
:101A6000D5E9033128469847302383F311886B6901
:101A7000002BD8D001F0A6F96A69A0EB04094A4509
:101A800082460DD2022001F0F5F90022D8F810307C
:101A9000B34208D151462846BDE8F047FFF728BFBA
:101AA000121A2244F2E712EB090938BF4A462946C6
:101AB0003846FFF7EBFEB5E7D8F81030B34208D050
:101AC0001444211AC8F81C00A960BDE8F047FFF7CC
:101AD000F3BEBDE8F08700BFA823002098230020B4
:101AE00000207047FEE70000704700004FF0FF3015
:101AF0007047000002290CD0032904D001290748AF
:101B000018BF00207047032A05D8054800EBC20023
:101B10007047044870470020704700BFC035000878
:101B2000202200207435000870B59AB0054608469A
:101B300001A9144600F0C2F801A8FFF7BFF8431C42
:101B40005B00C5E900340022237003236370C6B232
:101B500001AB02341046D1B28E4204F1020401D826
:101B60001AB070BD13F8011B04F8021C04F8010C34
:101B70000132F0E708B5302383F311880348FFF7FB
:101B800059FA002383F3118808BD00BF08260020FE
:101B900090F8443003F01F02012A07D190F8452045
:101BA0000B2A03D10023C0E90E3315E003F06003D4
:101BB000202B08D1B0F848302BB990F84520212AC5
:101BC00003D81F2A04D8FFF717BA222AEBD0FAE766
:101BD000034A82630722C26303640120704700BF87
:101BE0001822002007B5052917D8DFE801F01916DB
:101BF00003191920302383F31188104A0190012121
:101C0000FFF7BAFA01980E4A0221FFF7B5FA0D481C
:101C1000FFF7DCF9002383F3118803B05DF804FBC0
:101C2000302383F311880748FFF7A6F9F2E7302342
:101C300083F311880348FFF7BDF9EBE7143500087B
:101C4000383500080826002038B50C4D0C4C0D49DD
:101C50002A4604F10800FFF767FF05F1CA0204F104
:101C600010000949FFF760FF05F5CA7204F118007A
:101C70000649BDE83840FFF757BF00BFD02A002013
:101C800020220020F4340008FE3400080935000842
:101C900070B5044608460D46FFF710F8C6B2204658
:101CA000013403780BB9184670BD32462946FEF759
:101CB000F1FF0028F3D10120F6E700002DE9F84FED
:101CC00005460C46FEF7FAFF2949C6B22846FFF73B
:101CD000DFFF08B10136F6B226492846FFF7D8FFE4
:101CE00008B11036F6B2632E0DD8DFF88490DFF815
:101CF00084A0214FDFF888B0DFF888802E7846B9BD
:101D00002670BDE8F88F29462046BDE8F84F01F05F
:101D100097BB252E28D1072249462846FEF7BAFF51
:101D200040B9D8F800302360D8F804306360073534
:101D30000834E3E7082251462846FEF7ABFF98B97E
:101D40000E4BA21C197809090232C95D02F8041C65
:101D500013F8011B01F00F015B45C95D02F8031C7C
:101D6000F0D118340835C9E704F8016B0135C5E72F
:101D7000E035000809350008F1350008107AFF1F2A
:101D80001C7AFF1FE8350008BFF34F8F024AD36863
:101D9000DB03FCD4704700BF003C024008B5094B90
:101DA0001B7873B9FFF7F0FF074B1A69002ABFBF12
:101DB000064A5A6002F188325A601A6822F4806238
:101DC0001A6008BD2E2D0020003C0240230167450B
:101DD00008B50B4B1B7893B9FFF7D6FF094B1A696F
:101DE00042F000421A611A6842F480521A601A687E
:101DF00022F480521A601A6842F480621A6008BDA8
:101E00002E2D0020003C02400B28F0B516D80C4CBB
:101E10000C4923787BB90C4D0E460C234FF0006221
:101E200055F8047B46F8042B013B13F0FF033A44BA
:101E3000F6D10123237051F82000F0BD0020FCE70B
:101E4000602D0020302D002004360008014B53F88F
:101E500020007047043600080C2070470B2810B58E
:101E6000044601D9002010BDFFF7CEFF064B53F802
:101E700024301844C21A0BB90120F4E71268013269
:101E8000F0D1043BF6E700BF043600080B2810B57C
:101E9000044621D8FFF778FFFFF780FF0F4AF323AE
:101EA000D360C300DBB243F4007343F00203136159
:101EB000136943F480331361FFF766FFFFF7A4FF54
:101EC000074B53F8241000F0D9F8FFF781FF2046A4
:101ED000BDE81040FFF7C2BF002010BD003C02402B
:101EE00004360008F8B512F00103144642D18218F6
:101EF000B2F1016F57D82D4B1B6813F0010352D07C
:101F00002B4DFFF74BFFF323EB60FFF73DFF40F254
:101F10000127032C15D824F001046618244C401A1C
:101F200040F20117B142236900EB010524D123F0EF
:101F300001032361FFF74CFF0120F8BD043C04308E
:101F4000E7E78307E7D12B6923F440732B612B6903
:101F50003B432B6151F8046B0660BFF34F8FFFF7D3
:101F600013FF03689E42E9D02B6923F001032B6124
:101F7000FFF72EFF0020E0E723F44073236123697D
:101F80003B4323610B882B80BFF34F8FFFF7FCFE91
:101F90002D8831F8023BADB2AB42C3D0236923F0A8
:101FA00001032361E4E71846C7E700BF0038024099
:101FB000003C0240084908B50B7828B11BB9FFF76F
:101FC000EDFE01230B7008BD002BFCD0BDE80840DE
:101FD0000870FFF7FDBE00BF2E2D002010B5024493
:101FE000064BD2B2904200D110BD441C00B253F84F
:101FF000200041F8040BE0B2F4E700BF5028004095
:102000000F4B30B51C6F240407D41C6F44F40074CC
:102010001C671C6F44F400441C670A4C236843F49B
:10202000807323600244084BD2B2904200D130BD8D
:10203000441C00B251F8045B43F82050E0B2F4E7CE
:1020400000380240007000405028004007B50122CF
:1020500001A90020FFF7C2FF019803B05DF804FB5F
:1020600013B50446FFF7F2FFA04205D0012201A9F3
:1020700000200194FFF7C4FF02B010BD70470000BC
:10208000034B1A681AB9034AD2F874281A607047C9
:10209000642D00200030024008B5FFF7F1FF024B2D
:1020A0001868C0F3407008BD642D00207047000020
:1020B000FEE700000A4B0B480B4A90420BD30B4B38
:1020C000DA1C121AC11E22F003028B4238BF002212
:1020D0000021FEF7FBBD53F8041B40F8041BECE79E
:1020E000B0370008602E0020602E0020602E0020F7
:1020F00070B5D0E915439E6800224FF0FF3504EB20
:1021000042135101D3F800090028BEBFD3F80009DB
:1021100040F08040C3F80009D3F8000B0028BEBF90
:10212000D3F8000B40F08040C3F8000B0132631875
:102130009642C3F80859C3F8085BE0D24FF0011388
:10214000C4F81C3870BD0000890141F02001016114
:1021500003699B06FCD41220FFF71ABB10B5054C8F
:102160002046FEF7E9FF4FF0A0436365024BA365ED
:1021700010BD00BF682D00205836000870B50378E8
:10218000012B054650D12A4B446D98421BD1294B57
:102190005A6B42F080025A635A6D42F080025A65CF
:1021A0005A6D5A6942F080025A615A6922F08002DF
:1021B0005A610E2143205B6900F022FC1E4BE36054
:1021C0001E4BC4F800380023C4F8003EC02323602F
:1021D0006E6D4FF40413A3633369002BFCDA012303
:1021E00033610C20FFF7D4FA3369DB07FCD41220EB
:1021F000FFF7CEFA3369002BFCDA0026A6602846EA
:10220000FFF776FF6B68C4F81068DB68C4F81468E1
:10221000C4F81C684BB90A4BA3614FF0FF336361EC
:10222000A36843F00103A36070BD064BF4E700BF51
:10223000682D0020003802404014004003002002B6
:10224000003C30C0083C30C0F8B5446D0546002164
:102250002046FFF779FFA96D00234FF001128F6828
:10226000C4F834384FF00066C4F81C284FF0FF3033
:1022700004EB431201339F42C2F80069C2F8006BBD
:10228000C2F80809C2F8080BF2D20B686A6DEB6558
:10229000636210231361166916F01006FBD1122039
:1022A000FFF776FAD4F8003823F4FE63C4F8003858
:1022B000A36943F4402343F01003A3610923C4F846
:1022C0001038C4F814380A4BEB604FF0C043C4F820
:1022D000103B084BC4F8003BC4F81069C4F800393F
:1022E000EB6D03F1100243F48013EA65A362F8BDBD
:1022F0003436000840800010426D90F84E10D2F83D
:10230000003823F4FE6343EA0113C2F80038704733
:102310002DE9F84300EB8103456DDA68166806F095
:102320000306731E022B05EB41130C4680460FFA81
:1023300081F94FEA41104FF00001C3F8101B4FF034
:10234000010104F1100398BFB60401FA03F3916987
:102350008EBF334E06F1805606F5004600293AD06E
:10236000578A04F15801490137436F50D5F81C18BA
:102370000B43C5F81C382B180021C3F810195369FA
:102380000127611EA7409BB3138A928B9B08012AE9
:1023900088BF5343D8F85C20981842EA034301F100
:1023A000400205EB8202C8F85C00214653602846D3
:1023B000FFF7CAFE08EB8900C3681B8A43EA84530F
:1023C000483464011E432E51D5F81C381F43C5F80C
:1023D0001C78BDE8F88305EB4917D7F8001B21F4FA
:1023E0000041C7F8001BD5F81C1821EA0303C0E719
:1023F00004F13F0305EB83030A4A5A60284621464D
:10240000FFF7A2FE05EB4910D0F8003923F4004392
:10241000C0F80039D5F81C3823EA0707D7E700BF12
:102420000080001000040002826D1268C265FFF790
:102430005FBE00005831436D49015B5813F4004002
:1024400004D013F4001F0CBF0220012070470000CD
:102450004831436D49015B5813F4004004D013F434
:10246000001F0CBF022001207047000000EB81011B
:10247000CB68196A0B6813604B68536070470000A3
:1024800000EB810330B5DD68AA691368D36019B920
:10249000402B84BF402313606B8A1468426D1C4438
:1024A000013CB4FBF3F46343033323F0030302EB77
:1024B000411043EAC44343F0C043C0F8103B2B68CB
:1024C00003F00303012B09B20ED1D2F8083802EB56
:1024D000411013F4807FD0F8003B14BF43F08053C9
:1024E00043F00053C0F8003B02EB4112D2F8003B2E
:1024F00043F00443C2F8003B30BD00002DE9F04139
:10250000244D6E6D06EB40130446D3F8087BC3F8E8
:10251000087B38070AD5D6F81438190706D505EB15
:1025200084032146DB6828465B689847FA071FD575
:10253000D6F81438DB071BD505EB8403D968CCB972
:102540008B69488A5A68B2FBF0F600FB16228AB9FA
:102550001868DA6890420DD2121AC3E900243023B9
:1025600083F311880B482146FFF78AFF84F3118813
:10257000BDE8F081012303FA04F26B8923EA020328
:102580006B81CB68002BF3D021460248BDE8F041B7
:10259000184700BF682D002000EB810370B5DD688F
:1025A000436D6C692668E6604A0156BB1A444FF4D5
:1025B0000020C2F810092A6802F00302012A0AB2B8
:1025C0000ED1D3F8080803EB421410F4807FD4F83E
:1025D000000914BF40F0805040F00050C4F80009DA
:1025E00003EB4212D2F8000940F00440C2F800099F
:1025F000D3F83408012202FA01F10143C3F8341878
:1026000070BD19B9402E84BF4020206020682E8AFA
:102610008419013CB4FBF6F440EAC44040F0005099
:102620001A44C6E72DE9F8433B4D6E6D06EB4013A7
:102630000446D3F80889C3F8088918F0010F4FEA57
:1026400040171AD0D6F81038DB0716D505EB8003F3
:10265000D9684B691868DA68904230D2121A4FF084
:1026600000091A60C3F80490302383F311882146CF
:102670002846FFF791FF89F3118818F0800F1CD0CE
:10268000D6F834380126A640334216D005EB840331
:102690006D6DD3F80CC0DCF814200134E4B2D2F82C
:1026A00000E005EB04342F445168714515D3D5F88B
:1026B000343823EA0606C5F83468BDE8F8830123F8
:1026C00003FA04F22B8923EA02032B818B68002B87
:1026D000D3D0214628469847CFE7BCF81000AEEB90
:1026E0000103834228BF0346D7F8180980B2B3EB31
:1026F000800FE2D89068A0F1040959F8048FC4F85B
:102700000080A0EB09089844B8F1040FF5D81844EC
:102710000B4490605360C7E7682D00202DE9F74F08
:10272000A24C656D6E69AB691E4016F480586E61EF
:1027300007D02046FEF768FD03B0BDE8F04F00F07B
:1027400047BC002E12DAD5F8003E98489B071EBF02
:10275000D5F8003E23F00303C5F8003ED5F8043851
:1027600023F00103C5F80438FEF778FD370505D5D9
:102770008E48FFF7BDFC8D48FEF75EFDB0040CD51A
:10278000D5F8083813F0060FEB6823F470530CBF2C
:1027900043F4105343F4A053EB6031071BD5636837
:1027A000DB681BB9AB6923F00803AB612378052B09
:1027B0000CD1D5F8003E7D489A071EBFD5F8003EE3
:1027C00023F00303C5F8003EFEF748FD6368DB68AD
:1027D0000BB176489847F30274D4B70227D5D4F8E2
:1027E0005490DFF8C8B100274FF0010A09EB4712F7
:1027F000D2F8003B03F44023B3F5802F11D1D2F877
:10280000003B002B0DDA62890AFA07F322EA030380
:10281000638104EB8703DB68DB6813B139465846F4
:102820009847A36D01379B68FFB29F42DED9F0063F
:1028300017D5676D3A6AC2F30A1002F00F0302F46B
:10284000F012B2F5802F00F08580B2F5402F08D14C
:1028500004EB83030022DB681B6A07F58057904274
:102860006AD13003D5F8184813D5E10302D500200A
:10287000FFF744FEA20302D50120FFF73FFE6303EA
:1028800002D50220FFF73AFE270302D50320FFF707
:1028900035FE75037FF550AFE00702D50020FFF746
:1028A000C1FEA10702D50120FFF7BCFE620702D5D9
:1028B0000220FFF7B7FE23077FF53EAF0320FFF7A7
:1028C000B1FE39E7636DDFF8E4A0019300274FF014
:1028D0000109A36D9B685FFA87FB9B453FF67DAFBF
:1028E000019B03EB4B13D3F8001901F44021B1F520
:1028F000802F1FD1D3F8001900291BDAD3F8001953
:1029000041F09041C3F80019D3F800190029FBDB0E
:102910005946606DFFF718FC218909FA0BF321EA8B
:102920000303238104EB8B03DB689B6813B15946D7
:10293000504698470137CCE7910708BFD7F8008089
:10294000072A98BF03F8018B02F1010298BF4FEAF2
:10295000182884E7023304EB830207F58057526896
:10296000D2F818C0DCF80820DCE9001CA1EB0C0C44
:10297000002188420AD104EB830463689B699A684A
:1029800002449A605A6802445A606AE711F0030FE1
:1029900008BFD7F800808C4588BF02F8018B01F191
:1029A000010188BF4FEA1828E3E700BF682D002027
:1029B000436D03EB4111D1F8003B43F40013C1F820
:1029C000003B7047436D03EB4111D1F8003943F4EC
:1029D0000013C1F800397047436D03EB4111D1F882
:1029E000003B23F40013C1F8003B7047436D03EB39
:1029F0004111D1F8003923F40013C1F800397047B0
:102A000000F1604303F561430901C9B283F8001383
:102A1000012200F01F039A4043099B0003F1604329
:102A200003F56143C3F880211A60704730B5039CF9
:102A30000172043304FB0325C0E90653049B0363BE
:102A40000021059BC160C0E90000C0E90422C0E983
:102A50000842C0E90A11436330BD0000416A002208
:102A6000C0E90411C0E90A22C2606FF00101FEF75B
:102A7000FFBE0000D0E90432934201D1C2680AB916
:102A8000181D70470020704703691960C268013241
:102A9000C260C269134482690361934224BF436ADE
:102AA00003610021FEF7D8BE38B504460D46E36841
:102AB0003BB16269131D1268A3621344E3620020F4
:102AC00007E0237A33B929462046FEF7B5FE0028F1
:102AD000EDDA38BD6FF00100FBE70000C368C269A2
:102AE000013BC3604369134482694361934224BF3D
:102AF000436A436100238362036B03B11847704745
:102B000070B53023044683F31188866A3EB9FFF717
:102B1000CBFF054618B186F31188284670BDA36A1D
:102B2000E26A13F8015BA362934202D32046FFF7E7
:102B3000D5FF002383F31188EFE700002DE9F84F5C
:102B400004460E46174698464FF0300989F311881F
:102B50000025AA46D4F828B0BBF1000F09D14146A0
:102B60002046FFF7A1FF20B18BF311882846BDE86E
:102B7000F88FD4E90A12A7EB050B521A934528BF28
:102B80009346BBF1400F1BD9334601F1400251F887
:102B9000040B43F8040B9142F9D1A36A4033403649
:102BA000A3624035D4E90A239A4202D32046FFF7B4
:102BB00095FF8AF31188BD42D8D289F31188C9E7FD
:102BC00030465A46FEF75CF8A36A5B445E44A36253
:102BD0005D44E7E710B5029C0172043303FB042156
:102BE000C0E906130023C0E90A33039B0363049B77
:102BF000C460C0E90000C0E90422C0E908424363A0
:102C000010BD0000026AC260426AC0E904220022CC
:102C1000C0E90A226FF00101FEF72ABED0E90423C1
:102C20009A4201D1C26822B9184650F8043B0B60A1
:102C3000704700231846FAE7C368C2690133C360CE
:102C40004369134482694361934224BF436A4361E9
:102C50000021FEF701BE000038B504460D46E368CA
:102C60003BB123691A1DA262E2691344E3620020AA
:102C700007E0237A33B929462046FEF7DDFD002818
:102C8000EDDA38BD6FF00100FBE700000369196061
:102C9000C268013AC260C269134482690361934207
:102CA00024BF436A036100238362036B03B11847A7
:102CB0007047000070B530230D460446114683F37B
:102CC0001188866A2EB9FFF7C7FF10B186F3118805
:102CD00070BDA36A1D70A36AE26A01339342A362C6
:102CE00004D3E16920460439FFF7D0FF002080F3C8
:102CF0001188EDE72DE9F84F04460D4690469946B8
:102D00004FF0300A8AF311880026B346A76A4FB9FC
:102D100049462046FFF7A0FF20B187F311883046CF
:102D2000BDE8F88FD4E90A073A1AA8EB06079742DC
:102D300028BF1746402F1BD905F1400355F8042B37
:102D400040F8042B9D42F9D1A36A4033A362403678
:102D5000D4E90A239A4204D3E16920460439FFF7F3
:102D600095FF8BF311884645D9D28AF31188CDE7B8
:102D700029463A46FDF784FFA36A3B443D44A362DB
:102D80003E44E5E7D0E904239A4217D1C3689BB1DA
:102D9000836A8BB1043B9B1A0ED01360C368013B5E
:102DA000C360C3691A44836902619A4224BF436ABB
:102DB0000361002383620123184670470023FBE769
:102DC00000F030B94FF08043586A70474FF08043AD
:102DD000002258631A610222DA6070474FF0804384
:102DE0000022DA60704700004FF08043586370475C
:102DF000FEE7000070B51B4B01630025044686B05A
:102E0000586085620E4600F0BFF804F11003C4E973
:102E100004334FF0FF33C4E90635C4E90044A5602C
:102E2000E562FFF7CFFF2B460246C4E9082304F111
:102E300034010D4A256580232046FEF7B3FC0123AB
:102E4000E0600A4A0375009272680192B268CDE9A7
:102E50000223074B6846CDE90435FEF7CBFC06B0EC
:102E600070BD00BF002600206436000869360008E7
:102E7000F12D0008024AD36A1843D062704700BFA0
:102E8000982300204B6843608B688360CB68C360E5
:102E90000B6943614B6903628B6943620B68036092
:102EA0007047000008B5264B26481A6940F2FF110A
:102EB0000A431A611A6922F4FF7222F001021A61B0
:102EC0001A691A6B0A431A631A6D0A431A651E4A75
:102ED0001B6D1146FFF7D6FF02F11C0100F5806063
:102EE000FFF7D0FF02F1380100F58060FFF7CAFF5D
:102EF00002F1540100F58060FFF7C4FF02F1700198
:102F000000F58060FFF7BEFF02F18C0100F58060E4
:102F1000FFF7B8FF02F1A80100F58060FFF7B2FFEC
:102F200002F1C40100F58060FFF7ACFF02F1E0019F
:102F300000F58060FFF7A6FFBDE8084000F0EEB89E
:102F400000380240000002407036000808B500F06A
:102F500059FAFEF705FCFFF793F8BDE80840FEF7C5
:102F600073BE000070470000EFF3098305494A6B08
:102F700022F001024A63683383F30988002383F354
:102F80001188704700EF00E0302080F3118862B6AE
:102F90000C4B0D4AD96821F4E0610904090C0A437D
:102FA000DA60D3F8FC20094942F08072C3F8FC20B3
:102FB0000A6842F001020A602022DA7783F82200D0
:102FC000704700BF00ED00E00003FA05001000E0CC
:102FD00010B5302383F311880E4B5B6813F4006344
:102FE00014D0F1EE103AEFF30984683C4FF080738F
:102FF000E361094BDB6B236684F30988FEF790FBE2
:1030000010B1064BA36110BD054BFBE783F311889C
:10301000F9E700BF00ED00E000EF00E02F0300083B
:10302000320300080F4B1A6C42F001021A641A6E48
:1030300042F001021A660C4A1B6E936843F00103CA
:1030400093604FF0804353229A624FF0FF32DA626E
:1030500000229A615A63DA605A6001225A611A604A
:10306000704700BF00380240002004E04FF080426B
:1030700008B51169D3680B40D9B2C9439B071161E8
:1030800007D5302383F31188FEF780FB002383F3F9
:10309000118808BD1F4B1A696FEAC2526FEAD252FB
:1030A0001A611A69C2F308021A614FF0FF301A69F7
:1030B0005A69586100215A6959615A691A6A62F05D
:1030C00080521A621A6A02F080521A621A6A5A6AA6
:1030D00058625A6A59625A6A1A6C42F080521A64EB
:1030E0001A6E42F080521A661A6E0B4A106840F44B
:1030F00080701060186F00F44070B0F5007F1EBF44
:103100004FF4803018671967536823F400735360D5
:1031100000F054B90038024000700040334B4FF0CB
:1031200080521A64324A4FF4404111601A6842F0EA
:1031300001021A601A689107FCD59A6822F003020E
:103140009A602A4B9A6812F00C02FBD1196801F0C0
:10315000F90119609A601A6842F480321A601A689C
:103160009203FCD55A6F42F001025A671F4B5A6F07
:103170009007FCD51F4A5A601A6842F080721A60A4
:103180001B4A53685904FCD5184B1A689201FCD5A8
:10319000194A9A60194B1A68194B9A42194B21D156
:1031A000194A1168194A91421CD140F205121A605D
:1031B000144A136803F00F03052BFAD10B4B9A68DE
:1031C00042F002029A609A6802F00C02082AFAD1D0
:1031D0005A6C42F480425A645A6E42F480425A66F3
:1031E0005B6E704740F20572E1E700BF00380240B5
:1031F000007000400854400700948838002004E024
:1032000011640020003C024000ED00E041C20F418B
:10321000074A08B5536903F00103536123B1054A16
:1032200013680BB150689847BDE80840FFF7D0BE5F
:10323000003C0140E02D0020074A08B5536903F027
:103240000203536123B1054A93680BB1D0689847D4
:10325000BDE80840FFF7BCBE003C0140E02D002067
:10326000074A08B5536903F00403536123B1054AC3
:1032700013690BB150699847BDE80840FFF7A8BE35
:10328000003C0140E02D0020074A08B5536903F0D7
:103290000803536123B1054A93690BB1D06998477C
:1032A000BDE80840FFF794BE003C0140E02D00203F
:1032B000074A08B5536903F01003536123B1054A67
:1032C000136A0BB1506A9847BDE80840FFF780BE0B
:1032D000003C0140E02D0020164B10B55C6904F461
:1032E00078725A61A30604D5134A936A0BB1D06A67
:1032F0009847600604D5104A136B0BB1506B984782
:10330000210604D50C4A936B0BB1D06B9847E205AC
:1033100004D5094A136C0BB1506C9847A30504D52A
:10332000054A936C0BB1D06C9847BDE81040FFF78D
:103330004FBE00BF003C0140E02D0020194B10B5EE
:103340005C6904F47C425A61620504D5164A136D27
:103350000BB1506D9847230504D5134A936D0BB1FB
:10336000D06D9847E00404D50F4A136E0BB1506E30
:103370009847A10404D50C4A936E0BB1D06E9847C0
:10338000620404D5084A136F0BB1506F98472304A9
:1033900004D5054A936F0BB1D06F9847BDE8104034
:1033A000FFF716BE003C0140E02D002008B5FFF7F6
:1033B0005DFEBDE80840FFF70BBE0000062108B522
:1033C0000846FFF71DFB06210720FFF719FB062122
:1033D0000820FFF715FB06210920FFF711FB062146
:1033E0000A20FFF70DFB06211720FFF709FB062136
:1033F0002820FFF705FBBDE8084007211C20FFF748
:10340000FFBA000008B5FFF745FE00F00BF8FDF726
:1034100091FEFDF769FDFFF7A5FDBDE80840FFF748
:10342000CFBC00000023054A19460133102BC2E926
:10343000001102F10802F8D1704700BFE02D002012
:10344000034611F8012B03F8012B002AF9D170472C
:1034500053544D3332463F3F3F0053544D33324671
:103460003430780053544D3332463432780053545C
:103470004D333246343436585800000001203300B2
:103480000010410001105A000310590007103100CC
:103490000000000050340008130400005A340008F3
:1034A0001904000064340008210400006E34000890
:1034B00000000000650E0008510E00088D0E000887
:1034C000790E0008850E0008710E00085D0E0008D8
:1034D000490E0008990E00080000000001000000DD
:1034E0000000000063300000E4340008F0230020F6
:1034F000002600204172647550696C6F740025428B
:103500004F415244252D424C002553455249414CD0
:1035100025000000020000000000000081100008EB
:10352000ED10000840004000A02A0020B02A002032
:103530000200000000000000030000000000000086
:10354000311100080000000010000000C02A002017
:10355000000000000100000000000000682D0020B5
:1035600001010200E51B0008F51A0008911B000884
:10357000751B0008430000007C3500080902430069
:10358000020100C03209040000010202010005240A
:103590000010010524010001042402020524060094
:1035A00001070582030800FF09040100020A000068
:1035B00000070501024000000705810240000000ED
:1035C00012000000C835000812011001020000407E
:1035D000091241570002010203010000040309041B
:1035E00025424F4152442500537563636578463444
:1035F000003031323334353637383941424344456F
:1036000046000000004000000040000000400000B4
:103610000040000000000100000002000000020065
:103620000000020000000200000002000000020092
:103630000000020000000000751200082D150008AF
:10364000D915000840004000C82D0020C82D0020DA
:1036500001000000D82D0020800000004001000083
:10366000030000006D61696E0069646C6500000014
:103670000001806A00000000AAAAAAAA0001006452
:10368000FFFF00000000000000A00A00000400018D
:1036900000000000AAAAAAAA00000001DFFF0000A3
:1036A00000000000000000004000000000000000DA
:1036B000AAAAAAAA40000000FFFF00000000000024
:1036C000000000000000000000000000AAAAAAAA52
:1036D00000000000FFFF00000000000000000000EC
:1036E0000000000000000000AAAAAAAA0000000032
:1036F000FFFF0000000000000000000000000000CC
:1037000000000000AAAAAAAA00000000FFFF000013
:1037100000000000000000000000000000000000A9
:10372000AAAAAAAA00000000FFFF000000000000F3
:103730000000000000000000000000000A0000007F
:103740000000000003000000000000000000000076
:103750000000000000000000000000000000000069
:103760000000000000000000000000000000000059
:10377000F30300000000000000000F000000000044
:10378000FF009600000000080096000000000800FE
:1037900004000000DC35000800000000000000000C
:1037A0000000000000000000000000000000000019
:1037B000FFFFFFFFFFFFFFFFFFFFFFFFFFFFFFFF19
:1037C000FFFFFFFFFFFFFFFFFFFFFFFFFFFFFFFF09
:1037D000FFFFFFFFFFFFFFFFFFFFFFFFFFFFFFFFF9
:020000040801F1
:10000000000600208912010815F7060871F6060897
:10001000DDF6060871F60608A9F606088B12010837
:100020008B1201088B1201088B120108AD300908F0
:100030008B1201088B1201088B1201088B12010828
:100040008B1201088B1201088B1201088B12010818
:100050008B1201088B120108C9420908F1420908F4
:10006000194309084143090869430908DDEC0808F8
:1000700005ED080831ED08085DED080889ED080870
:10008000B1ED0808DDED080861EC08088B120108E5
:100090008B1201088B1201088B1201089143090889
:1000A000B5440908B9440908CD440908D1440908F0
:1000B0008B120108D5440908E944090869F30808C6
:1000C00011F508088B1201088B1201088B12010828
:1000D0008B12010865440908794409088D44090810
:1000E000F54309088B1201088B1201080D45090818
:1000F00011450908254509082945090809EE080898
:100100008B1201088B120108FD4409088B120108AB
:100110008B1201088B1201088B1201088B12010847
:1001200035EE08085DEE080889EE0808B5EE080807
:10013000E1EE08088B1201088B1201088B120108EE
:100140008B1201088B1201088B120108D93709089C
:1001500009EF080835EF080861EF0808A14409080D
:100160008B1201088B1201088B1201088B120108F7
:100170008B1201088B1201088B1201088B120108E7
:100180008B1201088B1201088B1201088B120108D7
:100190008B1201088B1201088B1201088B120108C7
:1001A0008B1201088B1201088B1201088B120108B7
:1001B0008B1201088B1201088B1201088B120108A7
:1001C0008B1201088B1201088B1201088B12010897
:1001D0008B1201088B1201088B1201088B12010887
:1001E000D52501088DAE010855A2040845BF0408B5
:1001F00075160508391E05087121050811860508C0
:1002000055A30508952E060809430608E1EF0608E0
:10021000BDA3070851E407082D160808D563080890
:10022000A58A0808C99408086DC4080835CA0808D2
:1002300081F0004102E000BF83F0004330B54FEA97
:1002400041044FEA430594EA050F08BF90EA020F04
:100250001FBF54EA000C55EA020C7FEA645C7FEA97
:10026000655C00F0E2804FEA5454D4EB5555B8BFBA
:100270006D420CDD2C4480EA020281EA030382EA2B
:10028000000083EA010180EA020281EA0303362DBD
:1002900088BF30BD11F0004F4FEA01314FF4801C90
:1002A0004CEA113102D0404261EB410113F0004FA2
:1002B0004FEA03334CEA133302D0524263EB430359
:1002C00094EA050F00F0A780A4F10104D5F1200EF7
:1002D0000DDB02FA0EFC22FA05F2801841F1000152
:1002E00003FA0EF2801843FA05F359410EE0A5F126
:1002F00020050EF1200E012A03FA0EFC28BF4CF057
:10030000020C43FA05F3C01851EBE37101F000450C
:1003100007D54FF0000EDCF1000C7EEB00006EEB19
:100320000101B1F5801F1BD3B1F5001F0CD34908A3
:100330005FEA30004FEA3C0C04F101044FEA4452FA
:1003400012F5800F80F09A80BCF1004F08BF5FEA81
:10035000500C50F1000041EB045141EA050130BD61
:100360005FEA4C0C404141EB0101013C28BFB1F573
:10037000801FE9D291F0000F04BF01460020B1FABE
:1003800081F308BF2033A3F10B03B3F120020CDA91
:100390000C3208DD02F1140CC2F10C0201FA0CF06F
:1003A00021FA02F10CE002F11402D8BFC2F1200CD4
:1003B00001FA02F120FA0CFCDCBF41EA0C0190408A
:1003C000E41AA2BF01EB0451294330BD6FEA0404D3
:1003D0001F3C1CDA0C340EDC04F11404C4F12002BE
:1003E00020FA04F001FA02F340EA030021FA04F3D0
:1003F00045EA030130BDC4F10C04C4F1200220FA27
:1004000002F001FA04F340EA0300294630BD21FA64
:1004100004F0294630BD94F0000F83F4801306BF2A
:1004200081F480110134013D4EE77FEA645C18BF1E
:100430007FEA655C29D094EA050F08BF90EA020FB5
:1004400005D054EA000C04BF1946104630BD91EAAD
:10045000030F1EBF0021002030BD5FEA545C05D1B0
:100460004000494128BF41F0004130BD14F58004EF
:100470003CBF01F5801130BD01F0004545F0FE4163
:1004800041F470014FF0000030BD7FEA645C1ABF98
:10049000194610467FEA655C1CBF0B46024650EACF
:1004A000013406BF52EA033591EA030F41F40021FB
:1004B00030BD00BF90F0000F04BF0021704730B581
:1004C0004FF4806404F132044FF000054FF0000156
:1004D00050E700BF90F0000F04BF0021704730B517
:1004E0004FF4806404F1320410F0004548BF4042EC
:1004F0004FF000013EE700BF42004FEAE2014FEA41
:1005000031014FEA02701FBF12F07F4393F07F4F1B
:1005100081F06051704732F07F4208BF704793F01E
:100520007F4F04BF41F40021704730B54FF4607431
:1005300001F0004521F000411CE700BF50EA010234
:1005400008BF704730B54FF000050AE050EA0102DD
:1005500008BF704730B511F0004502D5404261EB4D
:1005600041014FF4806404F132045FEA915C3FF48E
:10057000D8AE4FF003025FEADC0C18BF03325FEA2B
:10058000DC0C18BF033202EBDC02C2F1200300FADC
:1005900003FC20FA02F001FA03FE40EA0E0021FA01
:1005A00002F11444BDE600BF70B54FF0FF0C4CF4EF
:1005B000E06C1CEA11541DBF1CEA135594EA0C0FA1
:1005C00095EA0C0F00F0DEF82C4481EA030621EADC
:1005D0004C5123EA4C5350EA013518BF52EA033517
:1005E00041F4801143F4801338D0A0FB02CE4FF0C9
:1005F0000005E1FB02E506F00042E0FB03E54FF0F9
:100600000006E1FB03569CF0000F18BF4EF0010EF0
:10061000A4F1FF04B6F5007F64F5407404D25FEAEC
:100620004E0E6D4146EB060642EAC62141EA55519F
:100630004FEAC52040EA5E504FEACE2EB4F1FD0CE1
:1006400088BFBCF5E06F1ED8BEF1004F08BF5FEA5F
:10065000500E50F1000041EB045170BD06F0004611
:1006600046EA010140EA020081EA0301B4EB5C04BE
:10067000C2BFD4EB0C0541EA045170BD41F48011B6
:100680004FF0000E013C00F3AB8014F1360FDEBFDB
:10069000002001F0004170BDC4F10004203C35DAB7
:1006A0000C341BDC04F11404C4F1200500FA05F33A
:1006B00020FA04F001FA05F240EA020001F00042DB
:1006C00021F0004110EBD37021FA04F642EB060151
:1006D0005EEA430E08BF20EAD37070BDC4F10C047B
:1006E000C4F1200500FA04F320FA05F001FA04F23F
:1006F00040EA020001F0004110EBD37041F100012B
:100700005EEA430E08BF20EAD37070BDC4F1200535
:1007100000FA05F24EEA020E20FA04F301FA05F29D
:1007200043EA020321FA04F001F0004121FA04F245
:1007300020EA020000EBD3705EEA430E08BF20EA15
:10074000D37070BD94F0000F0FD101F0004640004F
:1007500041EB010111F4801F08BF013CF7D041EAD1
:10076000060195F0000F18BF704703F000465200D5
:1007700043EB030313F4801F08BF013DF7D043EAA6
:100780000603704794EA0C0F0CEA135518BF95EA5C
:100790000C0F0CD050EA410618BF52EA4306D1D1E3
:1007A00081EA030101F000414FF0000070BD50EA02
:1007B000410606BF1046194652EA430619D094EA8C
:1007C0000C0F02D150EA013613D195EA0C0F05D176
:1007D00052EA03361CBF104619460AD181EA0301CA
:1007E00001F0004141F0FE4141F470014FF0000082
:1007F00070BD41F0FE4141F4780170BD70B54FF01D
:10080000FF0C4CF4E06C1CEA11541DBF1CEA13559C
:1008100094EA0C0F95EA0C0F00F0A7F8A4EB05047E
:1008200081EA030E52EA03354FEA013100F0888075
:100830004FEA03334FF0805545EA131343EA12633E
:100840004FEA022245EA111545EA10654FEA0026F3
:100850000EF000419D4208BF964244F1FD0404F5AC
:10086000407402D25B084FEA3202B61A65EB030508
:100870005B084FEA32024FF480104FF4002CB6EBC5
:10088000020E75EB030E22BFB61A754640EA0C0045
:100890005B084FEA3202B6EB020E75EB030E22BF85
:1008A000B61A754640EA5C005B084FEA3202B6EBC6
:1008B000020E75EB030E22BFB61A754640EA9C0085
:1008C0005B084FEA3202B6EB020E75EB030E22BF55
:1008D000B61A754640EADC0055EA060E18D04FEA13
:1008E000051545EA16754FEA06164FEAC30343EAB3
:1008F00052734FEAC2025FEA1C1CC0D111F4801F80
:100900000BD141EA00014FF000004FF0004CB6E778
:1009100011F4801F04BF01430020B4F1FD0C88BF17
:10092000BCF5E06F3FF6AFAEB5EB030C04BFB6EB22
:10093000020C5FEA500C50F1000041EB045170BD15
:100940000EF0004E4EEA113114EB5C04C2BFD4EB42
:100950000C0541EA045170BD41F480114FF0000EC6
:10096000013C90E645EA060E8DE60CEA135594EA42
:100970000C0F08BF95EA0C0F3FF43BAF94EA0C0F45
:100980000AD150EA01347FF434AF95EA0C0F7FF4BA
:1009900025AF104619462CE795EA0C0F06D152EA0E
:1009A00003353FF4FDAE1046194622E750EA4106F2
:1009B00018BF52EA43067FF4C5AE50EA41047FF403
:1009C0000DAF52EA43057FF4EBAE12E74FF0FF3C68
:1009D00006E000BF4FF0010C02E000BF4FF0010C39
:1009E0004DF804CD4FEA410C7FEA6C5C4FEA430CB2
:1009F00018BF7FEA6C5C1BD001B050EA410C0CBF01
:100A000052EA430C91EA030F02BF90EA020F002062
:100A1000704710F1000F91EA030F58BF994208BFC9
:100A200090422CBFD8176FEAE37040F00100704786
:100A30004FEA410C7FEA6C5C02D150EA013C07D1DD
:100A40004FEA430C7FEA6C5CD6D152EA033CD3D028
:100A50005DF8040B704700BF8446104662468C4622
:100A60001946634600E000BF01B5FFF7B7FF002855
:100A700048BF10F1000F01BD4DF808EDFFF7F4FF7E
:100A80000CBF012000205DF808FB00BF4DF808ED09
:100A9000FFF7EAFF34BF012000205DF808FB00BF2C
:100AA0004DF808EDFFF7E0FF94BF012000205DF84E
:100AB00008FB00BF4DF808EDFFF7CEFF94BF012003
:100AC00000205DF808FB00BF4DF808EDFFF7C4FFFC
:100AD00034BF012000205DF808FB00BF4FEA410C45
:100AE0007FEA6C5C02D150EA013C0AD14FEA430C28
:100AF0007FEA6C5C02D152EA033C02D14FF0000065
:100B000070474FF0010070474FEA410212F50012A2
:100B100015D211D56FF47873B3EB625212D94FEA44
:100B2000C12343F0004343EA505311F0004F23FA2E
:100B300002F018BF404270474FF00000704750EA83
:100B4000013005D111F0004008BF6FF00040704740
:100B50004FF00000704700BF4A0011D212F500129A
:100B600011D20DD56FF47873B3EB62520ED44FEA05
:100B7000C12343F0004343EA505323FA02F0704785
:100B80004FF00000704750EA013002D14FF0FF30C3
:100B900070474FF0000070474FEA4102B2F1E04366
:100BA00024BFB3F5001CDCF1FE5C0DD901F0004C54
:100BB0004FEAC0024CEA5070B2F1004F40EB8300A4
:100BC00008BF20F00100704711F0804F21D113F1D0
:100BD0003872BCBF01F00040704741F480114FEA09
:100BE0005252C2F11802C2F1200C10FA0CF320FA92
:100BF00002F018BF40F001004FEAC1234FEAD323AF
:100C000003FA0CFC40EA0C0023FA02F34FEA430318
:100C1000CCE77FEA625307D150EA01331EBF4FF0A1
:100C2000FE4040F44000704701F0004040F0FE40BC
:100C300040F40000704700BF80F0004002E000BFB9
:100C400081F0004142001FBF5FEA410392EA030FB7
:100C50007FEA226C7FEA236C6AD04FEA1262D2EB01
:100C60001363C1BFD218414048404140B8BF5B4206
:100C7000192B88BF704710F0004F40F4000020F09F
:100C80007F4018BF404211F0004F41F4000121F0B5
:100C90007F4118BF494292EA030F3FD0A2F10102FF
:100CA00041FA03FC10EB0C00C3F1200301FA03F13D
:100CB00000F0004302D5494260EB4000B0F5000F60
:100CC00013D3B0F1807F06D340084FEA310102F11F
:100CD0000102FE2A51D2B1F1004F40EBC25008BFD1
:100CE00020F0010040EA03007047490040EB00009B
:100CF000013A28BFB0F5000FEDD2B0FA80FCACF19C
:100D0000080CB2EB0C0200FA0CF0AABF00EBC250C8
:100D100052421843BCBFD0401843704792F0000FB6
:100D200081F4000106BF80F400000132013BB5E709
:100D30004FEA41037FEA226C18BF7FEA236C21D07F
:100D400092EA030F04D092F0000F08BF08467047E4
:100D500090EA010F1CBF0020704712F07F4F04D1B2
:100D6000400028BF40F00040704712F100723CBFC5
:100D700000F50000704700F0004343F0FE4040F4EF
:100D8000000070477FEA226216BF08467FEA2363AD
:100D90000146420206BF5FEA412390EA010F40F498
:100DA000800070474FF0000304E000BF10F00043E4
:100DB00048BF40425FEA000C08BF704743F09643CB
:100DC00001464FF000001CE050EA010208BF7047E6
:100DD0004FF000030AE000BF50EA010208BF70476D
:100DE00011F0004302D5404261EB41015FEA010C82
:100DF00002BF84460146002043F0B64308BFA3F17A
:100E00008053A3F50003BCFA8CF2083AA3EBC2535B
:100E100010DB01FA02FC634400FA02FCC2F120027A
:100E2000BCF1004F20FA02F243EB020008BF20F0B1
:100E30000100704702F1200201FA02FCC2F1200217
:100E400050EA4C0021FA02F243EB020008BF20EA0C
:100E5000DC7070477BB972B90029BEBF00204FF02B
:100E6000004106E008BF00281CBF6FF000414FF0B2
:100E7000FF3000F007BAADF1080C6DE904CE00298F
:100E800009DB002B1ADB00F095F8DDF804E0DDE962
:100E9000022304B07047404261EB4101002B1BDB91
:100EA00000F088F8DDF804E0DDE9022304B04042F8
:100EB00061EB4101524263EB43037047524263EBE3
:100EC000430300F077F8DDF804E0DDE9022304B025
:100ED000404261EB41017047524263EB430300F033
:100EE00069F8DDF804E0DDE9022304B0524263EB67
:100EF0004303704753B94AB9002908BF00281CBFF3
:100F00004FF0FF314FF0FF3000F0BCB9ADF1080CED
:100F10006DE904CE00F04EF8DDF804E0DDE90223CF
:100F200004B07047430803F05533C01A830803F038
:100F3000333300F03330184400EB101000F00F3062
:100F400000EB002000EB0040000E704707EE900A17
:100F5000F5EEC07AF1EE10FA01D400F00BB8F1EE24
:100F6000677A08B517EE900A00F004F8404261EB8A
:100F7000410108BDD0B5FFF7BFFA0C4B0022064671
:100F80000F46FFF711FBFFF7E7FD0446FFF792FA64
:100F9000074B0022FFF708FB02460B463046394656
:100FA000FFF74AF9FFF7D8FD2146D0BD0000F03D1C
:100FB0000000F0412DE9F047089D04468E46002BC5
:100FC0004DD18A42944669D9B2FA82F252B101FAFD
:100FD00002F3C2F1200120FA01F10CFA02FC41EA0D
:100FE000030E94404FEA1C48210CBEFBF8F61FFA92
:100FF0008CF708FB16E341EA034306FB07F199422D
:101000000AD91CEB030306F1FF3080F01F819942DF
:1010100040F21C81023E63445B1AA4B2B3FBF8F0B9
:1010200008FB103344EA034400FB07F7A7420AD940
:101030001CEB040400F1FF3380F00A81A74240F268
:1010400007816444023840EA0640E41B00261DB1D3
:10105000D4400023C5E900433146BDE8F0878B4208
:1010600009D9002D00F0EF800026C5E900013046C7
:101070003146BDE8F087B3FA83F6002E4AD18B42A1
:1010800002D3824200F2F980841A61EB030301204B
:101090009E46002DE0D0C5E9004EDDE702B9FFDE37
:1010A000B2FA82F2002A40F09280A1EB0C014FEAE2
:1010B0001C471FFA8CFE0126200CB1FBF7F307FB3F
:1010C000131140EA01410EFB03F0884208D91CEBE2
:1010D000010103F1FF3802D2884200F2CB8043467F
:1010E000091AA4B2B1FBF7F007FB101144EA01445E
:1010F0000EFB00FEA64508D91CEB040400F1FF31ED
:1011000002D2A64500F2BB800846A4EB0E0440EADA
:1011100003409CE7C6F12007B34022FA07FC4CEAE3
:10112000030C20FA07F401FA06F31C43F9404FEAD6
:101130001C4900FA06F3B1FBF9F8200C1FFA8CFEEB
:1011400009FB181140EA014108FB0EF0884202FA3F
:1011500006F20BD91CEB010108F1FF3A80F0888000
:10116000884240F28580A8F102086144091AA4B2BD
:10117000B1FBF9F009FB101144EA014100FB0EFE3E
:101180008E4508D91CEB010100F1FF346CD28E456D
:101190006AD90238614440EA0840A0FB0294A1EBFE
:1011A0000E01A142C846A64656D353D05DB1B3EB5B
:1011B000080261EB0E0101FA07F722FA06F3F1408B
:1011C0001F43C5E9007100263146BDE8F087C2F132
:1011D0002003D8400CFA02FC21FA03F391400143AA
:1011E0004FEA1C471FFA8CFEB3FBF7F007FB1036E3
:1011F0000B0C43EA064300FB0EF69E4204FA02F48F
:1012000008D91CEB030300F1FF382FD29E422DD9E1
:10121000023863449B1B89B2B3FBF7F607FB163316
:1012200041EA034106FB0EF38B4208D91CEB010196
:1012300006F1FF3816D28B4214D9023E6144C91A16
:1012400046EA004638E72E46284605E70646E3E626
:101250001846F8E64B45A9D2B9EB020864EB0C0E30
:101260000138A3E74646EAE7204694E74046D1E73F
:10127000D0467BE7023B614432E7304609E76444ED
:10128000023842E7704700BF02E000F000F8FEE7D6
:1012900072B6374880F30888364880F309883648A4
:1012A0003649086040F20000CCF200004EF634717E
:1012B000CEF200010860BFF34F8FBFF36F8F40F293
:1012C0000000C0F2F0004EF68851CEF20001086036
:1012D000BFF34F8FBFF36F8F4FF00000E1EE100AA6
:1012E0004EF63C71CEF200010860062080F31488AF
:1012F000BFF36F8F81F038FF82F082FE4FF05530E0
:101300001F491B4A91423CBF41F8040BFAE71D49B3
:10131000184A91423CBF41F8040BFAE71A491B4AAC
:101320001B4B9A423EBF51F8040B42F8040BF8E7FE
:1013300000201849184A91423CBF41F8040BFAE7D3
:1013400081F016FF82F0B0FE144C154DAC4203DA6A
:1013500054F8041B8847F9E701F02CF9114C124DA1
:10136000AC4203DA54F8041B8847F9E781F0FEBE6B
:1013700000060020002200200000010808ED00E027
:101380000000002000060020B0810B080022002091
:10139000C8250020C8250020581E0120E0010108B2
:1013A0003002010830020108300201082DE9F04F37
:1013B0002DED108AC1F80CD0C3689D46BDEC108A93
:1013C000BDE8F08F002383F311882846A047002052
:1013D00080F052FEFEE780F0AFFC00DFFEE7000089
:1013E00001F0FF01102A2BDB10F0070F08D010F8D6
:1013F000013B013A8B422DD010F0070F42B3F6D1DA
:10140000F0B441EA012141EA014122F007047FF0F2
:1014100000070023F0E80256083C85EA010586EA49
:10142000010685FA47F5A3FA87F586FA47F6A5FA85
:1014300087F68EB9EED1F0BC01F0FF0102F0070291
:1014400032B110F8013B013A83EA010313B1F8D13C
:101450000020704701387047002D06BF354603381D
:10146000073815F0010F07D1013015F4807F02BF56
:10147000013015F4C03F0130F0BC0138704700BFA7
:1014800010F8012B11F8013B012A28BF9A42F7D02E
:10149000D01A7047034613F8012B002AFBD1181A03
:1014A0000138704738B50022002304460D46FFF787
:1014B000EDFA28B920462946BDE8384000F00AB8C0
:1014C000204605F1004100F005F8404261EB410182
:1014D00038BD00BFD0B50C4B002206460F46FFF7C3
:1014E00063F8FFF739FB0446FEF7E4FF074B0022E1
:1014F000FFF75AF802460B4630463946FEF79CFE87
:10150000FFF72AFB2146D0BD0000F03D0000F0416E
:10151000036800221B6818470120704737B5019106
:10152000202104465BF040FDD0B10E4B93F922140C
:10153000A1B1B3F92414D3F8F43B019AB3F90A50DA
:1015400001F10A039D4203DD40F28D33994205DC2F
:101550002046054B20215BF02FFD002003B030BD5D
:101560000120FBE7D045002010B4090807B5044866
:101570005CF04EFF00F0010003B05DF804FB00BF1B
:10158000DC5A00202DE9F0438FB00E46054605F0E9
:10159000EBFD002780462E22394602A8019785F0F0
:1015A0006BFD322301AA3946404605F027F904466F
:1015B00048B9184A01AB314628465BF0DFFE2046A9
:1015C0000FB0BDE8F083DFF85890D9F8200A03681F
:1015D0009B6898470028F2D0A9F5405003F0B8FD69
:1015E000814630B90C4A314628465BF0C7FE4C466E
:1015F000E5E76946404604F057FF0028DFD09DF834
:1016000001305B06DBD5054A314628465BF0B6FE65
:101610003C46D4E724B409082DB4090844B40908A9
:10162000D055002008B5064B93F8893E9B0704D59A
:10163000044A5BF0A3FE002008BD0120FCE700BFC8
:10164000D045002054B4090870B50C4C0546D4F8B8
:10165000200A0368DB680E46984710B10124204633
:1016600070BDA4F5405003F091FD04460028F5D16B
:10167000034A314628465BF081FEF0E7D055002052
:1016800064B409082DE97043264BD3F88C3E1D7BCA
:10169000804689465DB9244B1B68986A03685B6B7A
:1016A000984738B9214A494640465BF067FE2846CC
:1016B000BDE8708347F0F0F9202148F067F938B1B0
:1016C00047F0EAF91F2148F061F908B1184AEAE742
:1016D000D8F808303BB9D8F80030494640465B6B33
:1016E000BDE87043184749464046FFF717FF494693
:1016F000064640465CF0D0FA2021064040465BF0AA
:1017000053FC49464046FFF78DFFF5B20540494678
:101710004046FFF799FF4946054040465CF086FC8D
:101720000540C4E7D0450020F860002078B40908DF
:101730008FB4090808B5FFF7A5FF054A92F8781E8F
:1017400060F3410182F8781E024A907108BD00BF23
:10175000D045002085610020F7B505460F465BF0B7
:10176000CBFB044678B1022128465BF01DFC0646FF
:1017700048B115485CF04CFEC205C0F30723C0F326
:10178000002403D53446204603B0F0BD9B07F9D5AD
:101790000D485CF047FE0D4B03F21443D3ED007A85
:1017A000F8EEE77A30EE670ADFED097AB0EEC00AAC
:1017B000B4EEE70AF1EE10FAE4DD064B3A460221F8
:1017C00028465BF0F9FBDEE7DC5A0020D05500200C
:1017D0000000C842ACB40908F8B504460F465BF0F7
:1017E00075FE1021054620465BF0DEFB58B1204611
:1017F000FFF7BCFE064630B9044B3A46102120469E
:101800005BF0DAFB35462846F8BD00BFC0B40908D6
:1018100070B505460E465BF06FFB044678B180213B
:1018200028465BF0C1FB50B1094B93F8113443B12A
:10183000084B3246802128465BF0BEFB0024204640
:1018400070BD31462846BDE870405CF007B800BF67
:10185000D0550020D4B409082DE9F04180460E4649
:10186000FFF790FE1A4F044610B90024FC710AE0FD
:10187000184D05F54053D3F8200A03689B68984734
:1018800020B90123FB712046BDE8F08108214046C4
:101890005BF08AFB0028F4D095F81434B02202FBE8
:1018A000035305F50055B3F81E22B5F920349A42CA
:1018B00006DD094B3246082140465BF07DFBD4E74C
:1018C000314640465BF07EFC0028DAD1CDE700BF10
:1018D00085610020D0250020E8B409085CF0BEB87E
:1018E00070B505460E46FFF74DFE084B0446D8710D
:1018F00031462846FFF7A8FE31460028284608BF93
:1019000000245CF04FFA204070BD00BF85610020CC
:101910002DE9F843414F3B788146002B7BD1404C69
:10192000D4F88C5E2D7B01263E701DB13B7028469D
:10193000BDE8F8835CF034FC054630B9394A3870AC
:10194000137843F001031370F1E7DFF8F4803CF003
:101950004BF931463BF082FA88F804600B2634F0EC
:10196000F7FF013E34F0AAFF16F0FF06F7D12E492B
:1019700048465CF02FFB05F0F7FBD0F80022C4F8D6
:101980009C2E90F87C32DA0733D404F09DFF3CF0B3
:101990002BF93C213CF064F804F6846300221A60C1
:1019A000224B1B68D86A036801211B689847D4F84A
:1019B0008C2E137B1BB90123137388F804303CF081
:1019C00013F994F87D2E94F87C1E3BF01FFC39F03F
:1019D00055FC38F095FF00233B705DF0D1FE144BB1
:1019E000C3F8100A94F8793E43F0200384F8793E56
:1019F0009DE79B07D4D431460E4802F0F9F90E4812
:101A00005CF010FDDFED0D7A20EE270A04F684630A
:101A100083ED000AC4E7002589E700BFC825002040
:101A2000D0450020A4610020F8B40908F860002027
:101A3000D0550020D0250020DC5A00200AD7233CB6
:101A4000856100202DE9F0432B4DD5F88C3E1B7BA2
:101A500087B00646002B4CD05CF04EFC04460028B4
:101A600043D0264930465CF0B5FA05F07DFB0746C9
:101A700009F08AFF8046384604F0E2F9D8B198F9B7
:101A80002430022B17D100264FF00009F1B203AA2F
:101A900038460191CDF80C90CDF81090CDF8149007
:101AA00004F048FD019918B103AA404609F078FCFA
:101AB0000136032EEAD1D5F88C2E137B1BB10023FF
:101AC00013730F4A13713CF08FF800213BF0C6F9F5
:101AD0000C4B1B68D86A036800211B68984795F86F
:101AE000793E6FF3451385F8793E204607B0BDE88F
:101AF000F0830124F9E700BFD045002008B50908AC
:101B000085610020F860002008B500F5005090F8CD
:101B1000783EC3F380028A420BD061F3820380F8DF
:101B2000783E31B13CF060F8BDE808400F213BF051
:101B300097BF08BD10B500F500520C4692F8893EDB
:101B400003F00101A14209D064F3000382F8893E49
:101B5000DB0704D402F09CFB024B9C7210BD02F028
:101B60004BFCF9E78561002000F5005090F8893EB4
:101B700061F3410380F8893E014B1973704700BF40
:101B800085610020002070470020704700207047CA
:101B900000207047002070470020704700207047E9
:101BA00000207047002070470020704700207047D9
:101BB0007047000000F51050303070470048704703
:101BC000B8E1090800F5005090F87C0E704700005D
:101BD000034808601D21117008221A60704700BF79
:101BE000E4B7090839F094BA18F0FAB93BF0B4BA7E
:101BF00046F09EBB44F0D4BC02F06ABB02F09CBA33
:101C000002F0C2B934F05ABE4BF0D2BA03F086B833
:101C100046F090BE12F0DEBB02F0D8B802F09CBDD8
:101C200002F052BA02F0F0BC03F062B818F0CABD7C
:101C300003F0C4BA02F082BB02F03ABC70B5224B8A
:101C4000036000F500550446D5F80C0E1F4BC5F88F
:101C5000503C08B109F02CF91D4B236095F88430F5
:101C600043B9D5F880502DB1284616F047FF2846D5
:101C700009F01AF904F5975010305AF0F1FB04F509
:101C80009550143048F01AFD04F6E46504F68466B5
:101C9000B54204D0183D284616F0A0FBF8E70D4BDE
:101CA000C4F8C83804F628203DF0AEF804F6FC105D
:101CB0003DF0AAF804F65C103DF0A6F804F51360B8
:101CC0003DF0A2F8204670BD34BA090870930A08A6
:101CD00004740A08044B0A0838B54D4B044640F812
:101CE000043B49F01FFE04F1100008F023FD04F14D
:101CF000680038F09BFF04F5907010F0CDFF04F5FC
:101D00008C6007F0A3FA04F2845009F0D3F804F6CB
:101D1000C80017F0ABFF04F5666049F08BFD04F5D1
:101D2000736038F037FC04F58F503AF0F7FF04F594
:101D3000945018304FF038FA04F59550143048F0AC
:101D4000A5FC04F5975010305AF076FB04F5985036
:101D50000C3039F02DFB04F59B504AF08DFF04F553
:101D6000805300252B4A83F8845304F59C5004F5D6
:101D70009C5304331430136034F00EFC04F59F5070
:101D80002946083003F04EFD04F5D250103054F0CF
:101D900017FD04F5F850143057F086FB04F5005099
:101DA0002C3059F0A3FC04F5025010305AF0D8F84A
:101DB00004F50350283003F095FB04F50950083072
:101DC00055F05CF904F50A501349203037F0D6FC81
:101DD00004F50A5038304FF08BFC04F50D503430C8
:101DE0005AF0C6FE04F5005304F50F5083F8CC53A7
:101DF0000A4D24305AF0DEFF2B6813B108485DF01D
:101E00008DFC2046074937F0B9FC2C60204638BDD0
:101E100004740A08086B0020F42F0B085862002095
:101E20005CB509081C730A0810B503F0B5F846F054
:101E300033FE0368BDE810405B681847FFF7F4BF46
:101E400038B500F53A5520350446284608F04CFBD5
:101E500009F09AFD90F92130D3B190F84033BBB12D
:101E60002846002108F0D4F8DFED0A7A04F2DC738A
:101E700093ED287A20EE270ADFED077AA7EE270AEE
:101E800004F2845083ED280ABDE8384009F08CBC88
:101E900038BD00BFCDCCCC3D6666663FFFF7D0BFF6
:101EA00010B50121044603F0ADF910B1204601F050
:101EB000F1F84FF48051204603F0A4F920B12046F8
:101EC000BDE8104001F0A8B810BD0000FFF7E8BF62
:101ED00013B50221044603F095F938B101212046DB
:101EE00003F090F910B9204601F0D4F80221204601
:101EF00003F088F950B3204601F0DAF8402120467B
:101F000003F080F960B104F58F5001903AF0FCFACB
:101F100004F58053019893F9B4320BB13AF036FCD2
:101F20004FF48061204603F06DF918B104F58F502D
:101F30003AF084FB8021204603F064F968B119F07F
:101F40003DFE02B0BDE8104017F088BC01212046DC
:101F500003F058F90028CED1D0E74FF48021204675
:101F600003F050F90028EAD14FF40021204603F095
:101F700049F90028E3D102B010BD0000FFF7A8BF67
:101F800010B50121044603F03DF910B1204601F0DF
:101F90008FF88021204603F035F928B119F00EFEA4
:101FA000BDE8104017F036BC10BD0000FFF7E8BFD9
:101FB00038B54FF6FF71044603F024F904F50055D7
:101FC00028B1D5F8782E0721204601F079F848F09D
:101FD000BBF947F05FFF95F8783E074A83F010039E
:101FE000C3F30013537139F049F938F0B1FDBDE87E
:101FF0003840024853F0C2BE85610020F85E0020E0
:10200000FFF7D6BF2DE9F04F2DED028B00F59F5461
:102010000834A3B005460121204605F02BF805F54C
:1020200050513431204604F0B1FE05F551510C31C8
:10203000204603F0A7FF05F5B95104F545701CF0E3
:102040009BFC05F5405404F58B6304F2344783EDA3
:10205000000A04F587693968D9F80020209105F550
:10206000515020A920301D9321923DF097FE05F597
:10207000505105F552503C312430B0EE608AF0EEFC
:10208000408A3DF00DFD05F5515804F2444A04F52F
:10209000896B414605F55350C8ED008A18318AED29
:1020A000008A18308BED000A3DF0FAFC04F25C4225
:1020B00082ED000A1C923BF097FD05465DF068FB3F
:1020C0001B912D4906460868FEF716FACDE918015E
:1020D00004F254410868FEF70FFACDE9160104F541
:1020E0008A610868FEF708FACDE9140104F24C4150
:1020F00004F23C440868FEF7FFF9CDE912011C9A8E
:102100001068FEF7F9F9CDE910011D9B1868FEF77C
:10211000F3F9CDE90E01DBF80000FEF7EDF9CDE9AA
:102120000C012068FEF7E8F9CDE90A01DAF80000B1
:10213000FEF7E2F9CDE90801D9F80000FEF7DCF975
:10214000CDE90601D8F80000FEF7D6F9CDE9040183
:102150003868FEF7D1F91B9B0193CDE90201074BCB
:10216000074A0849009628463BF0B4FA23B0BDEC74
:10217000028BBDE8F08F00BFC43B002070B509089A
:102180007EB50908ABB50908FFF73CBF10B504469A
:1021900002F074FF1021204603F034F828B119F042
:1021A0000DFDBDE8104017F031BC10BDFFF7EEBFCC
:1021B00000F5805000F5C76300F24460D3ED005A8B
:1021C000D0ED006AD1ED017A91ED006A26EEE77A52
:1021D00067EEA57AA6EE257AE6EE267A81ED007AFC
:1021E000C1ED017A7047000000F5805000F5C7632B
:1021F00000F24460D3ED005AD0ED006AD1ED017ACF
:1022000091ED006A27EEA67A67EEA57AA6EE257A0A
:10221000E6EE667A81ED007AC1ED017A7047000042
:102220002DE9F0432DED028B044687B0FFF754FDF6
:10223000C84B236004F51150243001F05DFC04F517
:10224000005504F51053283304F530560436C5F80C
:10225000FC3B062385F8003C30465AF059FE0DF150
:102260001008BD4BC5F8043C301D0123414604F560
:1022700031578DF81030103738F058F8B74BC5F893
:10228000503C07F114005CF031FC04F5325604F5C3
:102290003359083609F12C093046143642F048FA11
:1022A0004E45F9D10723C5F8103E0023A5F8143E8A
:1022B0004FF4CB7008F0F6FDC5F80C0E04F538505D
:1022C00018305CF013FC04F539501C305CF00EFC47
:1022D000A34B1A6802B91F60A24BC5F8503C04F525
:1022E00039500123A5F87C3E3E305CF025F89E4B2A
:1022F00005939E4B0494009304F53A5098E80C0023
:102300004FF40071203007F035FD04F5505003A95B
:10231000F7EE008A1830CDED038A3DF02DF904F573
:1023200050509FED938A04F54055243008F0ECFAA4
:1023300005F2344383ED008A83ED018A83ED028A3E
:1023400004F5515383ED008A83ED018A83ED028AFF
:1023500005F24C4383ED008A83ED018A83ED028A06
:1023600005F2844383ED008A83ED018A05F28C43F4
:1023700083ED008A83ED018A05F2944383ED008AA0
:1023800083ED018A05F29C4383ED008A83ED018A87
:1023900005F20C5383ED008A83ED018A83ED028AF6
:1023A00005F5A3639FED732A83ED008A83ED018A0F
:1023B00083ED028A04F59F530833B0EE083A04F522
:1023C0005450C5F82435F0EE432AF0EE420AB0EE40
:1023D000430AF0EE481AB0EE481A283053F06CFE6B
:1023E000B0EE083A04F55950F0EE432AB0EE682AF0
:1023F000F0EE481AB0EE481AF7EE080AB1EE0C0AF1
:10240000343054F03DF8B0EE083A04F55B50F0EE8D
:10241000432AB0EE430A9FED572ADFED570AF0EE4C
:10242000481AB0EE481A2C3054F02AF8B0EE083AA8
:1024300004F55D50F0EE432A9FED502ADFED500A7F
:10244000F0EE481AB0EE481AB0EE680A243053F0A5
:1024500033FEB0EE083A04F56250F0EE432A9FEDE9
:10246000490AB0EE482AF0EE481AB0EE481AF0EEEB
:10247000480A303054F004F8F0EE083A04F564509D
:102480009FED410AB0EE485AF0EE684AB0EE484A75
:10249000B0EE633AF0EE632AB0EE002AF0EE481A8E
:1024A000B0EE481AF6EE000A283053F017FC374910
:1024B00037480860002304F5685285F8153A1C3245
:1024C00014279EB207FB06010133097C0029F8D1CD
:1024D000304B1E80304B196811B130485DF01EF949
:1024E00004F568502430C5F8200A1A6002F0EEF8AE
:1024F0002B4BC5F8243A04F56950143002F0E6F885
:10250000284BC5F8543A04F56A50043002F0DEF85E
:10251000254BC5F8843A04F56A50343002F0D6F8F9
:10252000224BC5F8B43A04F56B5005F6E42383ED6D
:10253000008A83ED018A83ED028A343002F0C6F806
:102540001B4BC5F8F43A204607B0BDEC028BBDE842
:10255000F08300BF34BA090824B5090870930A084B
:102560009C650020ECBA0908391C010828BA090842
:1025700000000000CDCC4C3ECDCCCC3ECDCCCC3DF3
:10258000CDCC4C3D3333333F9A99993F20620020A4
:102590009CF309081E620020DC610020B0B5090828
:1025A00030FD090878FC0908DCFD0908D4FC09089D
:1025B0007CFD090838B5054B1C6823680A461D6870
:1025C000034B01462046A847002038BDF860002094
:1025D000D025002010B55CF0FFFC064C064B1860BF
:1025E0002046FFF71DFE2046044A0549BDE810407D
:1025F00082F014B8D0250020F8600020BCBC002078
:102600003D1C010810B504460180024937F0B6F8B8
:10261000204610BDB4BA090810B500234FF07C5213
:10262000274C03654FF07E51C0F88030C0F89030E1
:10263000C0F8A030C0F8C0304365C0F88430C0F89E
:102640009430C0F8A430C0F8C43083668367C0F803
:102650009830C0F8A830C0F8B830C366C367C0F877
:102660009C30C0F8AC30C0F8BC304FF03F4302673C
:10267000C0F8B0204267C0F8B420C0F88820C0F885
:10268000C820C0F88C20016644668465C165C0F826
:10269000CC304FF47A71212047F084FB4FF47A71EB
:1026A000222047F07FFB4FF47A71232047F07AFB1A
:1026B000BDE810404FF47A71242047F073BB00BF8F
:1026C000000080BFF8B52DED068B037B044643B9AF
:1026D0000023C0F8D430C0F8D830C0F8E030C0F8DB
:1026E000DC30D4ED371A94ED381AD4ED360A94ED77
:1026F000350A8548DFED858A00F022FC5820B7EEC8
:10270000001AFFEE000A94ED350A19F075FF592002
:1027100084ED350AB7EE001AFFEE000A94ED360A92
:1027200019F06AFF5A2084ED360AB7EE001AFFEE60
:10273000000A94ED380A19F05FFF5B2084ED380A37
:10274000B7EE001AFFEE000A94ED370A19F054FFB5
:1027500084ED370A5DF008F807EE900A9FED6C7A79
:10276000F8EE677A04F1100567EE877A2126C4ED4A
:10277000027A2F46F7EE009A94ED35AAD5ED100AAD
:10278000B0EE680A6AEE200A82F0F4F894ED368A18
:10279000D5ED140AB0EE409A68EE200AB0EE680A51
:1027A00082F0E8F8D4ED385AD5ED186A94ED376A1E
:1027B00095ED1C7A65EEA66A79EE007AF0EEE66A8F
:1027C00026EE077A77EEA67AB0EEC77A77EE877AAA
:1027D000B5EEC09AE5EC017A95ED235AC5ED079A5E
:1027E00028EE058A95ED1F5AAAEE058A95ED275A1F
:1027F000A5EE858AD5ED2B5AA6EE258AF1EE10FAC4
:10280000CCBF01230023B5EEC00A85ED038AF1EEAB
:1028100010FA84F8D030C8BF94F8D030F5EEC06A12
:10282000C4BF013384F8D030F1EE10FAC8BF94F879
:10283000D030B5EEC07AC4BF013384F8D030F1EEA9
:1028400010FAC2BF94F8D030013384F8D03094F934
:10285000D030002BC1BF07EE103AB8EEC77AC8EEF1
:10286000076AC5ED036A95ED038AB0EEC87A77EE84
:10287000877AF4EEE97AF1EE10FAC4BF79EEC77AFE
:1028800045ED017A94F9E83015ED019A83B1DFED59
:10289000217AB4EEE79AF1EE10FA09D8DFED1E7A4C
:1028A000B4EEE77AF1EE10FAA4BF4FF08043EB618B
:1028B00094ED390AD5ED077A20EE270AD4ED027A95
:1028C00020EE270ADFED157A30EE000A20EE270A07
:1028D00081F0CAFFA9EE008A30B201369FED100ADE
:1028E00085ED0B8A28EE000AB6B247F037FA252E9E
:1028F0007FF442AFBDEC068B04F12002394602485A
:10290000BDE8F84000F04EBBD025002000000000DC
:10291000BD3786359A99193FCDCCCC3EDB0F494067
:1029200000007A440022C0F8D420C0F8D820C0F8B3
:10293000E020C0F8DC20FFF7C5BE00000020704793
:10294000002070470120704790F89C308B4286BF72
:10295000283150F8210000207047000090F89C308A
:102960008B4286BF283150F82100002070470000BC
:10297000FA207047014B93F812047047D0450020AD
:10298000D0E90B3242F4E0520263426B43F4F84365
:1029900042F4E0524263C36270470000014802F013
:1029A0004BBC00BFD025002013B54FF44470CDE9D7
:1029B000002108F071FA044628B1DDE9002144F055
:1029C00095FD024B2360204602B010BDD4BC09081F
:1029D00070470000704700000020704770470000FB
:1029E00000207047704700007047000003207047C8
:1029F00008207047064BD3F88C3E3BB11B7B002B65
:102A00000CBF5020D02040F0010070475020FAE762
:102A1000D045002070470000014B93F81404704724
:102A2000D0450020034B93F96804003818BF0120FB
:102A3000704700BFD0450020014B93F91604704742
:102A4000D04500207047000010B52DED028B174BCC
:102A5000D3F88C4E3CB3D4ED360A94ED380AF0EE40
:102A6000E00AB0EEC00A81F085FFD4ED370AB0EE7F
:102A7000408A94ED350AF0EEE00AB0EEC00A81F02B
:102A800079FFF0EE400AB0EE480A81F073FFDFED07
:102A9000087A20EE270ABDEEC00A10EE103A18B2EE
:102AA000BDEC028B10BD2046FAE700BFD0450020E8
:102AB0000000C84243F014BC10B5044640F04CFF7F
:102AC000054802F0B9FB054A034606212046BDE849
:102AD000104040F029BF00BFD025002024BB0908CA
:102AE00040F018B808B5084607F0E4FF00280CBF0E
:102AF0000420002008BD0000162A01D03FF04ABD86
:102B000003220A700120704710B44B7A8C7ACA7A7B
:102B100043EA042343EA0243863B012B03D95DF8D1
:102B2000044B44F0C1BA5DF8044B704708B53FF060
:102B30008DFF40F41C6040F00D0008BD10B5044648
:102B400008F0B2F9204610BD08B5094B93F8782E6D
:102B5000D2060BD403F58053D3F8200A03689B6A8E
:102B6000984700280CBF0220042008BD0120FCE784
:102B7000D0450020044B187820B9044B93F8790E07
:102B8000C0F38010704700BF54610020D045002082
:102B90001FB5002301930293039304F0E5FA01A902
:102BA00004F0D0F828B101A81CF068FA05B05DF86F
:102BB00004FB11F04DFC90F8F432B02202FB03004C
:102BC00090ED3B0AF2E700000C4B93F811248AB910
:102BD000A3F5805393F8892E51070BD193F8782EE3
:102BE000D20609D493F8793E13F0020F14BF0420E3
:102BF000012070470520704703207047D055002002
:102C00002DE9F04F354E96F87C3E012B8DB00446F1
:102C100052D9334F082506F5C75A17F9018BB6F973
:102C20003C3408F1FF3B43FA0BF3D90740D5207C35
:102C30003EF07AFB8146207C3FF07AFA00F12103D6
:102C4000994505D2207C0DB0BDE8F04F3DF0E8BDC0
:102C5000BBF1070F2CD8DFE80BF03E0432343638D6
:102C60003A3C204B186959695A6AD3F804B0D3F832
:102C700018E0D3F80CC0D3ED007A1B6ACDF82520FC
:102C8000CDF8293062222123CDE900320790089146
:102C9000207CCDED037A192303AAC221CDF810B010
:102CA000CDF814E0CDF818C08DF824803EF0A6FBD6
:102CB000013D15F0FF05B0D10DB0BDE8F08F0A4B16
:102CC000D0E70A4BCEE70A4BCCE70A4BCAE753469C
:102CD000C8E7094BC6E7094BC4E700BFD045002051
:102CE000A8BD0908645B0020745C0020EC5C002037
:102CF000745D0020A05D00208C5F0020385B002008
:102D0000094BD3F86C24920701D43FF037BC03F58C
:102D1000805303F5856393ED000ADFED047AB8EE86
:102D2000C00A20EE270A7047D04500200AD7233C6E
:102D300010B594B0044603A807F0E6FD1A4BD3F88B
:102D4000200A036803A91B6B984750B3247C5CF0EE
:102D500017FD059BDDED047A0893069B099300237C
:102D6000F8EEE77A9FED117A0B930C930D930E9387
:102D70000F931093119312934FF6F853ADF84C3014
:102D80000023962267EE877A8DF84E303323CDE903
:102D90000032079007AA57212046CDED0A7A3EF06F
:102DA0002DFB14B010BD00BFD05500200AD7233C26
:102DB000014802F03FBA00BFD0250020014B93F834
:102DC0007C0E7047D0450020024B93F8790EC0F37B
:102DD00040007047D045002030B52DED028B154BDB
:102DE00091ED018A0546D3F8200A036885B0DB69B6
:102DF0000C46984728B9BDEEC88A18EE103ADB0792
:102E000012D5D4E9040119F0FDFD68B1684607F058
:102E10007BFD6A462146284643F0BAFC20B10649AC
:102E2000684607F053FE00B1022005B0BDEC028BEE
:102E300030BD00BFD0550020F45900208B8B162BDD
:102E400005D0C02B01D1FFF7C7BF44F053BF00200E
:102E50007047000030B52DED028B8DB00023054684
:102E600003930493059304F07FF903A903F06AFF29
:102E700058B304F079F900F55A7393E8070006ACEB
:102E800084E80700DDED060A9DED070A2D7CF1EED2
:102E9000600AB1EE400A81F009FF2046B0EE408A98
:102EA0001CF0ECF8DFED0B7A089B0B93012228EE67
:102EB000278A0C23CDE90032A82109AA28468DEDE6
:102EC000098A8DED0A0A3EF099FA0DB0BDEC028B2D
:102ED00030BD00BFE02E6542242938B505460FD02D
:102EE00003D81B2907D1012412E04029FBD0A1F10E
:102EF0004203012BF7D92846BDE8384043F006BE0F
:102F00000C213DF09FFC044610B12846FFF7A2FFBC
:102F1000204638BD08B591ED007AF6EE007AB4EEA1
:102F2000E77AF1EE10FA06DD044801220521FEF7EA
:102F300089FD002008BD0420FCE700BFD45100201B
:102F40002DE9F04188B080461B22002101A810EE37
:102F5000107A10EE906A11EE105A11EE904A84F039
:102F60008BF8A3238DF8043095238DF805300B23BF
:102F70008DF806305CF00CFC1B22CDF80700CDF874
:102F80000B1008F58F5001A9CDF80F70CDF8136024
:102F9000CDF81750CDF81B4039F078FF08B0BDE8E8
:102FA000F081000070B58CB00D46144606462B2209
:102FB000002101A884F060F8A3238DF80430952344
:102FC0008DF805300C238DF806305CF0E1FB2B68A2
:102FD000CDF80F302368CDF813306B68CDF817307B
:102FE0006368CDF81B30AB68CDF81F30A368CDF80F
:102FF0002330EB68CDF80700CDF80B10CDF8273063
:103000002B22E368CDF82B3001A906F58F5039F05B
:103010003DFF0CB070BD000070B500F58F5500F598
:103020005456044606F1680228460E2139F0FEFD8A
:1030300006F1940228460F2139F0F8FD04F55A52A2
:1030400028462432102139F0F1FD04F55C5228465F
:1030500004F55D561C32112139F0E8FD06F16402D9
:1030600028466E2139F0E2FD06F1900228466F21D4
:1030700039F0DCFD04F56352284620320D2139F089
:10308000D5FD04F5665228463C32BDE870406B2100
:1030900039F0CCBD1FB500F59F50002301A90830C1
:1030A00001930293039302F0C7FA05B05DF804FBA5
:1030B00008B504F059F8BDE8084003F0F5BD00007C
:1030C0007FB50E464FF6FF710446154602F09AF89A
:1030D000E0B110220021684683F0CEFFA3238DF8D3
:1030E000003095238DF8013004238DF802305CF018
:1030F0004FFB1022CDF80300CDF8071004F58F50D8
:1031000069468DF80B60039539F040FF04B070BD3F
:10311000A320704738B5044600F58F5502F08CF8AF
:103120000C49024628463AF04DF804F5005328466B
:1031300093F87D2E93F87C1E3AF068F804F59F50C2
:10314000083004F021FA04F59070BDE8384010F022
:10315000E9B900BF24BB090837B5069D044600B98C
:103160002C7801B9697802B9AA7803B9EB78002004
:1031700064F3070061F30F2062F3174063F31F60ED
:1031800003B030BD2DE9F04F2DED0C8B9DB0DB4C25
:103190000D93D4ED379ADFEDDA5A90ED006A04F51D
:1031A0000054F7EE006AD4F88C3ED3ED367A93EDF6
:1031B000387AF0EEE77AB0EEC77A77EE877A914602
:1031C000F4EEE67AF1EE10FAC8BF86EEA78A06465C
:1031D0000F46DFEDCC7AD8BFB0EE668A28EE277AAC
:1031E000A6EE257A80ED007AD4F88C3E93ED357A00
:1031F00093ED376AB0EEC77AB0EEC66A37EE067A5C
:10320000B4EEE67AF1EE10FACCBFC6EE878AF7EE9E
:10321000008A90ED017A68EEA77AE7EE257AC0ED94
:10322000017A3AF0E1FC05465CF0B2FA824618EE0B
:10323000900A8846FDF760F9CDE9080118EE100AFA
:10324000FDF75AF9CDE906017068FDF755F9CDE9AA
:1032500004013068FDF750F9AB4BAC4ACDE90201EF
:10326000CDE900A82846AA49AA4D3AF033FAAA495E
:1032700095ED00AA38461BF0EDFA8DED160A99ED92
:10328000000ACDED170A30EE4A0A8DED181A19F032
:103290009FF904F25C439DED167AD3ED007AB0EE0F
:1032A000C77AB4EEE77AA5F2F453F1EE10FA0C9374
:1032B00000F12582D4F88C3E1B7B002B00F01F828E
:1032C000B4F85A34C3F340039DED177A0B93B0EE74
:1032D000C77AF4EEC77AF1EE10FA00F31282D4F84E
:1032E0008C3E1B7B002B00F00C82B4F85A3403F0A8
:1032F00001039DED187A0A93B0EEC77AF4EEC77A0F
:10330000F1EE10FA00F3FF81D4F88C3E1B7B002B0A
:1033100000F0F981B4F85A34C3F38008B0EEC00A63
:10332000F4EEC07AF1EE10FA00F3F081D4F88C3E9E
:103330001B7B002B00F0EA81B4F85A34C3F3C00AB7
:103340000DAB0093DDE90A1053464246FFF704FF38
:10335000C3B20BEE103AC0F307230AEE903AC0F363
:1033600007430CEE903A030E0DEE103A9DF8343000
:103370009FED6A8A0F90002B40F0CB819DF835308D
:10338000002B40F0C681F8EE4B7A634ACDED197AF6
:10339000F8EE6A7AB0EE690ACDED1A7AF8EE6C7A38
:1033A00019AB394602F54670CDED1B7A53F046F85D
:1033B0008DED140ACDED150AB0EE409AF0EE608A5C
:1033C0009DF83630564D002B40F0A88105F254434D
:1033D0001CEE901AD3ED000A97ED020AB0EE691ABE
:1033E00005F50B6053F048F9B0EE40CA9DF8373050
:1033F000002B40F0968199ED000A30EE4A0A19F050
:10340000E7F81DEE101A4748F0EE690A52F016FE72
:1034100005F6BC13D9F800201A60434BF0EE40BA11
:1034200083ED00AA414C94ED001A4720F1EE410AC9
:10343000B0EE490A19F0E0F8A346BBEC011AB0EE71
:1034400040AAF1EE410A4820B0EE680A19F0D4F81B
:103450009BED001AB0EE409AF1EE410A4920B0EE21
:103460004C0A19F0C9F894ED021AF0EE408A4A208D
:10347000B0EE6B0AF1EE410A19F0BEF896ED007A53
:10348000D6ED017A8DED148A6AEE076A04F5805B49
:10349000CDED106A69EE276A05F24443CDED116A5D
:1034A000DBED006A8DED158A27EE267AD3ED006AF2
:1034B0009DF834308DED127A67EEA67AF0EE40BAC0
:1034C000CDED137AA4F5886493BB9DF835307BBBB2
:1034D000B8EE4BBAF8EE6AAAB0EE690A19AB12AAB6
:1034E00010A90BF1E8008DED19BACDED1AAA52F032
:1034F00071FE8DED140ACDED150A19E0D0250020DE
:10350000A4707D3F00D7233C6DC3090860F0090813
:1035100079F00908C43B00201C5A0020000000007C
:10352000D0550020F85E0020905F0020104A002057
:103530009DF83630002B40F0F78005F5896396ED55
:10354000000AD3ED000A904860EE200A1CEE901AA3
:1035500028EE800AB0EE691A53F08EF8F0EE40AA19
:103560008A4814A9FEF740FE9DF83730002B40F042
:10357000DE8005F25C4396ED010AD3ED000A844833
:1035800060EE200AB0EE691A1DEE101A20EE2B0A2A
:1035900053F072F8F0EE409AD4F88C3E1B7B7BBB64
:1035A00019A97C488DED198A8DED1A8A52F05CFFBD
:1035B0009FED790A794853F07BF89FED770A7848B8
:1035C00052F066FD19A977488DED198A8DED1A8A9A
:1035D00052F04AFF9FED700A6B4853F069F86C484F
:1035E0009FED6D0A53F064F805F24C4393E8070031
:1035F0000C9B87E8070003F2F4531B68C9F80030FE
:103600000B9B002B00F09680D4F88C3E83ED368A1D
:103610000A9B002B00F09980D4F88C3E83ED358A0C
:10362000B8F1000F00F09C80D4F88C3E83ED388A0E
:10363000BAF1000F00F09E80D4F88C3E83ED378AFB
:1036400005F24C439FED588A9FED534ADBED002A6B
:1036500093ED001AD7ED000A62EE882A2AEE082AB6
:1036600021EE081A60EE880AF0EE443AB0EE443AD1
:10367000F0EE441AB0EE440A5BF0A0F905F24443C0
:10368000D3ED002A9FED444AD7ED010A05F58A6380
:1036900093ED001A62EE882A29EE082A21EE081A14
:1036A00060EE880AF0EE443AB0EE443AF0EE441A86
:1036B000B0EE440A5BF086F905F5896305F25445DE
:1036C0009FED354AD3ED002A95ED001AD7ED020A99
:1036D00062EEC82A28EEC82A21EE481A60EEC80A0F
:1036E000F0EE443AB0EE443AF0EE441AB0EE440A3A
:1036F0005BF06CF91DB0BDEC0C8BBDE8F08F0123C5
:10370000E2E50123F5E54FF0010807E64FF0010A75
:1037100016E6F0EE488AB0EE489A51E69FED1ECAD2
:1037200064E6DFED1DBA7DE6DFED1BAA18E7DFEDED
:103730001A9A31E79DF83430002B7FF469AFD4F842
:103740008C3E149AC3F8D82062E79DF83530002BE0
:103750007FF466AFD4F88C3E159AC3F8D4205FE7A7
:103760009DF83630002B7FF463AFD4F88C3EC3ED68
:1037700038AA5DE79DF83730002B7FF461AFD4F8AD
:103780008C3EC3ED379A5BE7445C0020D0250020D7
:10379000BC5C0020345D002000000000805E002042
:1037A000F85E0020F85A00200000C8422DE9F04FD2
:1037B0002DED088B8FB0CDE90223C84C94ED37BABC
:1037C00004F500548046D4F88C3E1B7B0E46002B3B
:1037D00000F04F81B4F85A54C5F3400B05F0010ACC
:1037E000C5F3800915F0080500D0012503AB51464B
:1037F000BB4F00934A462B465846FFF7ADFC97ED6A
:10380000001A96ED000A0590F1EE410A9A2018F090
:10381000F3FE97ED001A9FEDB38AF1EE410AF0EE48
:10382000409A9B2096ED010A18F0E6FE04F244420D
:1038300092ED001AB0EE409AF1EE410A96ED020ABE
:103840009C2018F0D9FE04F58962029B92ED001AC3
:10385000F0EE408A9D2093ED000AF1EE410A18F047
:10386000CBFE98ED007AD8ED017A8DED0A8A69EEEB
:10387000876A07F53C66CDED066A69EE276A07F5AB
:103880008057CDED076AD7ED006A8DED0B8A06F201
:10389000444327EE267AD3ED006A9DF80C308DED77
:1038A000087A67EEA67AB0EE40AACDED097AFBB9A8
:1038B0009DF80D30E3B99DF8143007EE103A9DF8ED
:1038C000153007EE903AB8EE477AF8EE677AB0EE28
:1038D0004B0A0CAB08AA06A906F5A5608DED0C7A7B
:1038E000CDED0D7A52F076FC8DED0A0ACDED0B0A86
:1038F0009DF80E30002B40F0C18006F5896398EDED
:10390000000AD3ED000A9DF81610774860EE200AF1
:10391000B0EE4B1A28EE800A52F0AEFEF0EE40AA4E
:103920006E480AA9FEF760FC9DF80F30002B40F0AE
:10393000A88006F25C4398ED010AD3ED000A9DF8D9
:1039400017106A4860EE200AB0EE4B1A20EE0A0A01
:1039500052F092FEB0EE40AAD4F88C3E1B7B8BB99D
:1039600063488DED0C8A0CA98DED0D8A52F07CFD1B
:103970009FED5C0A5C4852F09BFE9FED5A0A5B4843
:1039800052F096FEBBF1000F7ED0D4F88C3E83ED52
:10399000368ABAF1000F00F08180D4F88C3E83EDB6
:1039A000358AB9F1000F00F08480D4F88C3E83EDA5
:1039B000388A002D00F08780D4F88C3E83ED378A5A
:1039C00006F24C439FED4B8A9FED464AD7ED002A05
:1039D00093ED001A62EE882A29EE882A21EE081A51
:1039E000F0EE443AB0EE443AF0EE441AF0EE440AF7
:1039F000B0EE440A5AF0E2FF06F24443D3ED002A47
:103A00009FED384A06F58A6393ED001A62EE882A24
:103A100029EE082A21EE081AF0EE443AB0EE443AB4
:103A2000F0EE441AF0EE440AB0EE440A5AF0CAFF2F
:103A300006F5896306F254469FED2A4AD3ED002A23
:103A400096ED001A62EEC82A28EEC82A21EE481A1E
:103A5000F0EE443AB0EE443AF0EE441AF0EE440A86
:103A6000B0EE440A5AF0B2FF0FB0BDEC088BBDE8CF
:103A7000F08F4FF00109CA46CB46B6E6DFED19AA32
:103A80004EE79FED18AA67E79DF80C30002B80D118
:103A9000D4F88C3E0A9AC3F8D8207AE79DF80D3006
:103AA000002B7FF47EAFD4F88C3E0B9AC3F8D42061
:103AB00077E79DF80E30002B7FF47BAFD4F88C3E77
:103AC000C3ED38AA75E79DF80F30002B7FF478AF6F
:103AD000D4F88C3E83ED37AA72E700BFD0250020D2
:103AE000104A002000000000445C0020BC5C002064
:103AF000F85A00200000C84270B50446143044F063
:103B000039FE0B4E0B4B63616425601944F0FAFFDC
:103B100066513035B5F5597FF7D104F5597046F047
:103B2000EBFA2046044935F029FE204670BD00BF5F
:103B300038FA09084CFA0908FCF2090837B500F50B
:103B4000105101221031044637F0B4FE184A1368B0
:103B5000D90706D4174904F5095308330B6001232C
:103B6000136004F51150134901222430012535F06A
:103B70003DFA114A0095002304F58F51FD2035F0E0
:103B8000E3F90E4B1A68D20705D40D4A1D6004F5FF
:103B900098540C3414600A48012135F043FA35F08A
:103BA000F3FF084A138843F04003138003B030BD8D
:103BB000FC60002000220020A07A0A08006100209A
:103BC0000C220020106200200069C0F340107047F2
:103BD0000F299DBF302303FB0100503000207047A8
:103BE000014B93F92E047047D0450020024B93F807
:103BF000890E00F001007047D0450020014BD3F83A
:103C0000F80B7047D0450020054A92F8893E92F89B
:103C1000882E03F0010313430CBF012000207047DE
:103C2000D0450020002910B517DB104C94F8002C6B
:103C3000CBB29A4211D3D4F8FC3B0122595CA4F5D3
:103C4000005000F0B1FD94F8793E38B99A0704D5D8
:103C5000074A137843F00403137010BD9B07FCD58B
:103C6000034A137843F00203F6E700BFD045002073
:103C7000A4610020022A10B50F4C12D13522A4F500
:103C8000005000F091FD94F8793E9B0705D50B4B51
:103C90001A7818B142F002021A7010BD42F0040204
:103CA000FAE794F87C2E8A42F7D144F0F5FEBDE89D
:103CB000104044F07BBE00BFD0450020A46100202E
:103CC00010B500F50053DFED186AD3F8F02BD3F8E8
:103CD000EC3BB2F90820B3F908309FED147A07EEF7
:103CE000902AF8EEE77A0446C7EEA60A00F59F5040
:103CF0000121083007EE903AF8EEE77A60EE870A85
:103D000087EEA60A20EE070A03F0B8FA39F06CFF36
:103D1000262139F0A5FE04F53150054ABDE81040D2
:103D2000062110303CF05CBB0000C84235FA8E3CE6
:103D300088F80908332901D045F08EBC704700008F
:103D4000332910B519D0382913D0052917D1022AE3
:103D50000DD10D4890F87C3E012B08D8D0F8F43BEB
:103D6000B3F908301BB9A0F50050FFF7A9FF0120F7
:103D700010BD0321FFF77EFFF9E70121FAE7BDE857
:103D8000104045F0C7B900BFD045002030B504460B
:103D900089B0684604F59F5506F0B6FD083504A8BD
:103DA00006F0B2FD6946284602F094FF60B104A90E
:103DB000284602F0DFFF38B1059B019323680022FB
:103DC000DB6C69462046984709B030BD00F580524B
:103DD00092F86426D2070AD400F50052D2F88C2E4D
:103DE000117B09B1FFF7D2BF03689B6C184770477E
:103DF00010B586B0044602A8019106F085FD04F5D1
:103E00009F5002A9083002F065FF28B12368019A8B
:103E1000DB6C02A92046984706B010BDF0B50446F9
:103E200085B004F59F56684608360F46154606F0DD
:103E30006BFD6946304602F09DFF10B9002005B0C9
:103E4000F0BD3946304602F021FE0028F6D0002DA4
:103E5000F5D004F58054284694F8643643F0020304
:103E600084F86436EBE7000010B500F51054D4ED8B
:103E70000E7AF5EEC07AF1EE10FA8AB04FF0000338
:103E800004F1380444D907930893099306AB0193CE
:103E900000F59F5007AB03AA04A90093083005ABB7
:103EA00002F08CFEDDED080A9DED070A80F062FD50
:103EB000DDED090A80F05EFDD4ED007A9DED047A17
:103EC00077EEA76AB4EEE70AF1EE10FAF4EEC76AED
:103ED000ACBF01200020F1EE10FA0CD802309DEDAD
:103EE000037AF4EEC77AF1EE10FA0CD8003818BF56
:103EF00001200AB010BDF4EEC77AF1EE10FA9CBFB3
:103F00000130C0B2EBE7012894BF00200120F0E7A8
:103F10000020EEE738B500F50055044695F8893ED7
:103F20005A071AD443F0040385F8893E39F05CFE41
:103F30000122112139F0B4FD084BD3F8200A03689F
:103F40009B68984718B995F93534032B05D120465D
:103F50000621BDE8384000F021BD38BDD055002015
:103F600008B500F5005090F8893E5A070BD56FF35D
:103F7000820380F8893E39F037FEBDE80840002210
:103F8000112139F08DBD08BD2DE9F043054685B0FE
:103F900005F59F58684608F1080806F0B5FC694623
:103FA000404602F0E7FED8B105F50053434CD3F884
:103FB0008C2E434F127B42B103F58763D3ED007A19
:103FC000F5EEC07AF1EE10FA0DD8238823F4FF73D2
:103FD00023F00103238028460023FB73FFF7C0FF73
:103FE00005B0BDE8F083284601F0C8F8064618B9C8
:103FF000284601F089F806462846FFF735FF814636
:1040000040B93EB12378002B41D1637803F001031E
:10401000FB73E5E76378DB07F7D423780133DBB282
:10402000082B237006D12846FFF71EFF10B140462B
:1040300002F030FE2378092B02D1404602F022FE26
:104040002378092BE1D9238823F4FF7323F001039C
:1040500043F48573238039F0C7FD0222102139F023
:104060001FFD5BF08DFB6368C01A47F23053984226
:1040700009D905F53150134A022110303CF0B0F94E
:104080005BF07EFB60602846FFF744FFBDE7013B25
:1040900023702388C3F30803B3F5807FB5D1637819
:1040A00060F30003637039F09FFD4A46102139F038
:1040B000F7FC2846FFF754FFA7E700BF0461002084
:1040C0008561002068FA090837B5044600F59F505D
:1040D00001A9083004F5005502F0EEFBD5F83C3C90
:1040E000834206D0C5F83C0C39F07EFD3E2139F004
:1040F000B7FC04F5805395F9401C93F8F82693F922
:10410000F836994213D0FF2A11D085F8403C39F097
:104110006BFD95F8402C182139F0C2FC04F53150A4
:1041200095F9403C034A042110303CF059F903B0A2
:1041300030BD00BF78FA09082DE9F04395B0064676
:104140005BF01EFB06F59F5803AB019308F10808CE
:1041500002AB0024009305460EAB0BAA08A940460B
:10416000089409940A940B940C940D940E940F9453
:10417000109402F011FDDFED437A9DED0A7AB4EE62
:10418000E77AF1EE10FA074637DB9DED0D7AB4EED3
:10419000E77AF1EE10FAACBF4FF001094FF00009D9
:1041A00007AB019311AB009304AA06AB05A94046E7
:1041B00011941294139402F001FD06F500540028A6
:1041C00094F9E03B08BF002783B17FB1D4F88C3E5F
:1041D0001B7B5BB1B9F1000F08D09DED057AF7EEBE
:1041E000007AB4EEE77AF1EE10FA09D594F8443C7F
:1041F00073B90023C4F8483C0FE04FF00009CFE743
:10420000D4F8480C20BBC4F8485CC4F84C0C04E05B
:10421000D4F84C0C20B9C4F84C5C15B0BDE8F08360
:10422000281A43F698239842E3D9002584F8445C81
:10423000C4F84C5C39F0D8FC2A461D2139F030FC1A
:1042400006F53150104A022110303CF0C9F8D0E791
:104250002D1AB5F57A7FE0D994F8443C002BDCD1D7
:10426000012584F8445C39F0BFFC2A461D2139F051
:1042700017FC06F53150054A022110303CF0B0F829
:10428000CBE700BF0000003490FA0908ABFA090838
:1042900010B5044639F0A8FC0022052139F000FCD5
:1042A00004F53150034ABDE81040042110303CF0C1
:1042B00097B800BFC8FA090800F5005090F8793E99
:1042C0009B065ABF90F8780EC0F30010012070478B
:1042D00037B5044600F554500C305AF099F804F5FF
:1042E0000052C0F3803592F8793EC3F30011A94221
:1042F0001DD065F3041304F5315482F8793E10346F
:104300006DB139F071FC02220B2139F0C9FB094A69
:104310000221204603B0BDE830403CF061B839F0DE
:1043200063FC2A460B2139F0BBFB034AF0E703B0DC
:1043300030BD00BFE0FA0908EBFA090870B500F5D6
:104340000055044695F91E34B3B3D5F8086E9EB3F4
:104350005BF016FA05F6E83393ED000ADFED177A05
:104360009FED171ADFED170A861B20EE270A6B2038
:1043700018F042F9BCEEC00A10EE103A9E4209D283
:1043800095F8893E9A0717D520460021BDE8704070
:10439000FDF7EABB10D995F8893E9B070CD420465F
:1043A0000121FDF7E1FB04F530500122BDE870402A
:1043B00012210430FDF746BB70BD00BF00007A44F7
:1043C0000000804F000000000B46012B10B4114686
:1043D00004D0052B06D05DF8044B70475DF8044B04
:1043E00000F0DCBA00F530505DF8044B01221421D6
:1043F0000430FDF727BB00002DE9F041044604F529
:10440000005839F0F1FB0122052139F049FB98F9F8
:1044100022542046003D18BF0125FFF74DFF04F54B
:104420003156103698B11E4A042130463BF0D8FF71
:1044300004F53050012210210430FDF703FB002564
:10444000294620460322BDE8F041FFF7BDBF04F531
:104450004057D7F8200A03689B6A984768B197F8D5
:10446000113453B197F91034012B06DC0D4A0421A5
:1044700030463BF0B5FF0125E2E7D7F8200A036894
:104480009B6A984718B1D8F8E43B1B0705D4064A45
:10449000042130463BF0A4FFD2E7044AE7E700BF1F
:1044A00000FB09081BFB090849FB090858FB090820
:1044B00070B50446154639F097FB0122062139F004
:1044C000EFFA2046FFF7F8FE04F53156103698B1A2
:1044D00004F53050012207210430FDF7B3FA154AE4
:1044E000042130463BF07CFF00252946204604226B
:1044F000BDE87040FFF768BF04F54053EDB2D3F854
:10450000200A03689B6A984768B104F50053D3F802
:10451000E43B1B0707D535B1074A042130463BF081
:104520005FFF0125E1E7054A042130463BF058FFD3
:10453000DBE700BF7CFB090823FB090899FB09089E
:10454000F8B504465BF010F9284BB4F8BE20198882
:10455000274E914205460ED01A80264B18603378BC
:10456000A3B10024347039F03FFB22461321BDE88B
:10457000F84039F095BA33781F4FC3B93B782BB167
:104580001C4B1E4A1B68C31A934200D8F8BD012376
:10459000337004F50053D3F88C0E037B0BB1FEF798
:1045A000C1F939F021FB0122132139F079FA3B7866
:1045B000002BEBD03378002BE8D00E4A104913685B
:1045C000EB1A8B42E2D904F500541560D4F88C2E16
:1045D000137B002BDAD0002313730A4AD4F88C0E15
:1045E0001371BDE8F840FEF76DB800BF0E61002002
:1045F0000C610020106100200D61002080841E00ED
:1046000040420F008561002070B500F5005300F5B1
:1046100054550C3586B093F8441C0446284659F08E
:10462000A5FE02A806F070F904F59F5002A9083013
:1046300002F050FB04F54053049AC3F82C24059A69
:10464000C3F83024284659F0E3FE82061AD52846DE
:1046500059F0E8FE04F55055FDEEC07A243504F516
:10466000805417EE901A0222284617EE906A06F040
:1046700051F994F86436DB0706D401223146284606
:1046800006F048F906B070BD0121284606F0D4F9BD
:104690000028F2D0F6E700000120704700207047A4
:1046A00000207047002070470020704700207047AE
:1046B0000020704700207047002070479FED010ADE
:1046C000704700BF00000000704700000F4A026002
:1046D0000F4A426002F1540181600E49C1600E49E7
:1046E000016102F67C21416102F52861816102F2DB
:1046F000DC71C16102F5FC61016202F2E47102F554
:10470000FD628262054A4162C262704724FC090868
:10471000E0490020DC5A0020B8390020E8260020BB
:10472000042917D8DFE801F003070B0F130000F589
:1047300069501430704700F568502430704700F518
:104740006A500430704700F56A503430704700F505
:104750006B50FAE70020704700F54050D0F8200A6F
:1047600003685B681847000038B500F540550446FB
:10477000D5F8200A03685B6998470A4B04F5005294
:10478000187492F87C2ED5F8200ADA7003685B6AF8
:104790009847014604F59C501430BDE8384032F08B
:1047A000BFB800BF856100202DE9F84F00F5005A21
:1047B00006469AF87C3E8B420F46914605D18AF810
:1047C0007D2E01252846BDE8F88FFFF7A9FF044696
:1047D00020B9304637F0F6FA2546F3E7DAF88C3E92
:1047E0001B7B06F5315883F0010B08F11008E3B983
:1047F000236859461B6820469847054678B306F556
:1048000040534A46C3F8204A394606F58F508AF885
:104810007C7E8AF87D9E38F0F9FC4046002143F00A
:1048200041FA3046FFF7A0FFCCE703689B68984742
:10483000E0B11C4800F08CFC0546B8B9236820465E
:104840001B6A9847184A0346042140463BF0C8FDBE
:1048500039F0CAF93A460A2139F022F9B2E7236859
:1048600020461B6A9847114A0346EDE70D4800F0C1
:104870008DFC0028BCD106F54053D3F8200A03680C
:10488000DB6898470028B3D023682046DB68984748
:1048900005460028ACD1236820461B6A9847044A85
:1048A0000346D1E7D0250020ACFB0908FEFB090830
:1048B000D5FB09080148FFF777BF00BFD0250020CE
:1048C00070B5234B93F8893EDB0705460C46164628
:1048D00005D5002363602360A360336070BD44F09E
:1048E000DBF8037F002BF4D0EB699FED1A7A1B688D
:1048F000B3F9083007EE903AF8EEE77AC7EE876A28
:10490000C4ED016A2B6A1B68B3F9083007EE903AD0
:10491000F8EEE77AC7EE876AC4ED006A6B6A1B6837
:10492000B3F908305B4207EE903AF8EEE77AC7EE4B
:10493000876AC4ED026AAB6A1B68B3F9083007EEF8
:10494000903AF8EEE77AC7EE876AC6ED006AC5E7E7
:10495000D045002000007A440020704701207047B5
:1049600000207047002070470048704768FC090825
:104970000048704768FC090843691A680023C2F8B8
:10498000D43042691268C2F8D83042691268C2F85D
:10499000DC3042691268C2F8E03070470A4608B558
:1049A0000021FFF701FF034A137843F00803137057
:1049B00008BD00BFA461002001207047002070479F
:1049C000012070470020704700487047BCFC090870
:1049D00000487047C4FC090830B5084B03F5515234
:1049E0000C32044600F1300507CA85E8070003F5DC
:1049F000AF53143301201B68E36330BDD025002082
:104A000030B52DED028B044687B05A4D002301AA24
:104A100003A995ED378A039304930593FFF750FF9D
:104A200063689DED037AD3ED0F7A68EE277A27EE5F
:104A3000277A8DED037A9DED047A67EE277ACDED26
:104A4000047AD3ED107A28EE277ADDED057A67EE49
:104A5000877ACDED057AD3ED117A93F9483028EEB7
:104A6000278ADDED017A27EE888A8DED018A1BB950
:104A700003A92846FDF79CFB3F4B94ED0C7AD3ED40
:104A8000007A626894ED0F0AD2ED0F6A77EE677ACA
:104A9000A3F24C43F0EEE77AF4EEE67AF1EE10FA88
:104AA00044BFDDED037A77EE877A03F58A6148BF6C
:104AB000C4ED0C7A94ED0D7AD1ED007AD2ED0F6A47
:104AC00077EE677A03F25443F0EEE77AF4EEE67A93
:104AD000F1EE10FA44BFDDED047A77EE877A94EDBB
:104AE0000E7A48BFC4ED0D7AD3ED007AD2ED106A8C
:104AF000236977EE677AF0EEE77AF4EEE67AF1EE84
:104B000010FA42BFDDED057A77EE877AC4ED0E7AB2
:104B1000D3ED837A30EE670A17F05AFD6368D3ED60
:104B2000117AB0EEC00AB4EEE70AF1EE10FA09D538
:104B300094ED0F0ADDED017A30EE270A17F048FDFB
:104B400084ED0F0A00230D488DF808308DF80930E8
:104B50008DF80A308DF80B30029BD0F8900E04F1DE
:104B60003C0204F13001FEF70DFB07B0BDEC028BF7
:104B700030BD00BFD02500201C5A0020D0450020A9
:104B800000207047012070470120704700207047C7
:104B90000048704718FD09080048704720FD0908C3
:104BA0001FB5044600236A4601A9019302930393AB
:104BB000FFF786FE6369029A1B68C3F8D420636915
:104BC000019A1B68C3F8D8206369009A1B68C3F870
:104BD000DC206369039A1B68C3F8E02004B010BDB1
:104BE0000120704700207047012070470020704767
:104BF00000487047D4C8090800487047D4C809085D
:104C0000012070477FB5002303930493059301931C
:104C1000094800238DF808308DF809308DF80A30E6
:104C20008DF80B30029BD0F8900E01AA03A9FEF775
:104C3000A9FA07B05DF804FBD045002001207047B9
:104C400000207047012070470020704700487047DF
:104C5000C0FD090800487047CCFD090810B504469E
:104C600086B0002301AA03A9039304930593FFF7D9
:104C700027FE63689DED037AD3ED0C6ADDED047ABF
:104C800093F9483027EE267A67EEA67A8DED037AFF
:104C9000CDED047A1BB9144803A9FDF789FA6368BE
:104CA000DDED057A93ED0D7A104867EE877A93ED86
:104CB0000E7ACDED057ADDED017AD0F8900E002365
:104CC00067EE877A8DF808308DF809308DF80A3054
:104CD0008DF80B30029BCDED017A01AA03A9FEF7F6
:104CE00065FD06B010BD00BFD0250020D0450020D6
:104CF00038B5044645F054FA45F026FB04F5005457
:104D0000054645F0B7FA44F043FFD4F88C0EFDF7A2
:104D1000D9FC2846BDE8384045F0B4BA70B500F576
:104D20000055044695F9143C43B1D5F8F42B344EA4
:104D3000B2F90820002A02DD0023338070BDD5F8C7
:104D4000F82BB2F90820B2F5617F31DDB6F90030F9
:104D5000642BDCBF01333380B6F90030142B0DD146
:104D6000D5F88C3E197B0029E8D100F5305001229E
:104D70000430FCF7CDFD08B93080DFE7B6F900302C
:104D8000642BDBD1D5F88C3E1B7B002BD6D095F85D
:104D90007C3E012BD2D104F531501A4A0621103045
:104DA00004F540543BF01CFBFA23A4F8143AC5E781
:104DB00012F5617FC0DA022BBED100F54053D3F863
:104DC000200A0368DB68984718B995F8783EDB0637
:104DD000B2D5B6F90030142BB0DC01331BB2142B62
:104DE0003380ABD1D5F88C3E1B7B002BA6D004F5CD
:104DF00030500122BDE8704000210430FCF722BE93
:104E00001461002020FE090810B500F5005414219B
:104E1000D4F8EC0B43F08AFED4F8F00B142143F0E5
:104E200085FED4F8F40B1E2143F080FED4F8F80B75
:104E3000142143F07BFE43F02FFE036805211B681D
:104E40009847BDE81040002143F070BE38B50546D4
:104E500043F022FE43F0F8FD05F50054C4F8EC0BD6
:104E600043F01AFE43F0FAFDC4F8F00B43F014FED1
:104E700043F0FEFDC4F8F40B43F00EFE43F002FED7
:104E80004FF47A71C4F8F80BD4F8EC0B43F04AFEF7
:104E9000D4F8F00B4FF47A7143F044FED4F8F80BD9
:104EA0004FF47A7143F03EFED4F8F40B4FF47A716C
:104EB00043F038FE2846FFF7A7FF94F8793E43F009
:104EC000080384F8793E38BD08B545F03DFA44F052
:104ED000E1FFBDE8084044F093BF000000F500503A
:104EE000D0F88C0EFDF71EBD38B500F50054054610
:104EF00094F92234BBB1B4F824348B421DD994F810
:104F0000893EDA070FD443F0C7FD037F1BB9D4F8FD
:104F10008C3E1B7B3BB194F8883E01335BB2022B85
:104F200002DC84F8883E38BD032384F8883E0121E2
:104F30002846BDE83840FCF7FDBD94F8883E013BAB
:104F40005BB2002BEDDC94F8893E0021DB0784F88E
:104F5000881EE8D5EDE7000038B50D4604465AF046
:104F60000FFC002D0B4B09DD04F50054186094F87C
:104F7000793E6FF3C30384F8793E38BD1B68C01ACD
:104F8000B0F5C87FF9D904F5005494F8793E43F0A0
:104F90000803F0E718610020F7B504465AF0F0FB6B
:104FA000064643F079FD43F01FFC04F50055B0B30D
:104FB00095F8783E43F0200385F8783ED5F8F43B29
:104FC0002046D988FFF790FFD5F8F43B04F5405709
:104FD000B3F908102046FFF7BFFFD7F8183A9FED46
:104FE000267AF31A07EE903AD5F8F43BF8EE677A92
:104FF000B3F9083067EE877A04F55050CDED007AAA
:1050000007EE903AF8EEE77A6A4601A91830CDED3E
:10501000017A3AF0BFFAC7F8186A03B0F0BD95F804
:10502000893EDB07F9D404F54053D3F8180A361A41
:1050300043F064FC002814BF4FF47A734FF4FA7302
:10504000B342EAD895F92234002BE6D043F024FD90
:10505000037F23B9D5F88C3E1B7B002BDDD038F0C5
:10506000C3FD0222114638F01BFD0121204603B08A
:10507000BDE8F040FCF75EBD6F12833A38B50446D8
:1050800000F58C65284604F071FA94F871049FEDE0
:10509000097A242202FB0055D5ED0B7A67EE877A58
:1050A00004F54053FDEEE77A17EE902AC3F8142476
:1050B00038BD00BF0000C842FEF72CB80148FFF71A
:1050C0003FBA00BFD025002038B500F59F55083500
:1050D0000446284600F01EFD04F58053022283F8A2
:1050E000FC25B4F9A43004F6C8001BB9B4F8A2300A
:1050F000A4F8A430B4F8A41016F006FE2846BDE8C3
:10510000384000F001BE000013B5044600F59F5082
:10511000083000F003FF98B104F5545004F5005432
:105120000C3059F075F9D4F88C2E0190127BC3B273
:10513000C0F3001032B918B99DF80500C0F3400063
:1051400002B010BD0028FBD083F08000C009F7E753
:1051500038B500F50053054693F8893E5B070AD43D
:10516000FFF7D2FF044620B905F59F50083000F044
:10517000D5FE204638BD0024FBE7000008B500F549
:105180009F50083000F0CAFE002008BD13B5044649
:1051900000F59F50083000F0C1FE58B104F554509E
:1051A0000C3059F035F94207C3B203D5C3F34010B0
:1051B0009B0600D4002002B010BD000038B500F5F9
:1051C0000055044695F8783E590719D5D5F88C3E18
:1051D0001B7B2BB920460021BDE83840FCF794BC6E
:1051E00000F54053D3F8200A0368DB68984738B1CC
:1051F00095F8793E1A0703D595F8893EDB07E9D57E
:1052000038BD000037B500F58F55044604F500544D
:105210002846019137F05AFF94F8783E019960F3DF
:10522000C303284684F8783E03B0BDE8304038F028
:10523000A5BC0000072070470048704730FE0908F1
:1052400037B5154BB3F9A42005461AB9B3F8A22017
:10525000A3F8A420B3F8A4100191EC2005F01CFEE3
:10526000044610B10199FDF7CDF905F50050C0F8DD
:105270008C4E24B990F97414084805F00BFB0849CA
:10528000204634F089FC012034F016F903B0BDE863
:10529000304034F079BC00BFD025002038FE09082A
:1052A000B4BA0908F7B5044600F59C50143031F043
:1052B00003FB2046FFF758FA04F53A50203004F07B
:1052C00005FE04F59550143004F58C6745F004FA9A
:1052D000384604F077FC04F5315010303FF06EFA98
:1052E0006B4E2046FFF7B2FD2046FFF7A9FFB6F947
:1052F000A4301BB9B6F8A230A6F8A430082005F0F7
:10530000CBFD18B14FF07E530360436004F50055A8
:10531000C5F8900E43F0C0FB9922292144F078FB98
:1053200043F0BAFB43F060FB2046FFF7CDFD95F854
:10533000793E43F0400385F8793E04F59B5047F0F1
:1053400067FE544B54491B68986A03684FF47A729D
:10535000DB6A98470423C4F8A43104F590700DF07B
:105360002FFD06F011FB4FF40053036306F00CFB16
:1053700007F0D0FB8023C4F874340121384604F0D0
:1053800005FA464B0193009602AB13E9060004F5BB
:105390008F5037F057FD2046FFF796FE4FF400235D
:1053A000C4F8B83DD5F88C0EFDF736F904F5305049
:1053B00001210430FCF7B0F810B12046FFF78EFD54
:1053C000B4F9A43004F5515020301BB9B4F8A23020
:1053D000A4F8A430B4F8A420D5F88C3E00EE102A2E
:1053E000D3ED390AB8EE400AF2EE0E1AB6EE001A04
:1053F0003AF0D2FDB4F9A43004F5525024301BB970
:10540000B4F8A230A4F8A430B4F8A420D5F88C3EA7
:1054100000EE102AD3ED390AB8EE400AF2EE0E1A69
:10542000B7EE001A3AF0CCFBB4F9A43004F55350AF
:1054300018301BB9B4F8A230A4F8A430B4F8A420F2
:10544000D5F88C3E00EE102AD3ED390AB8EE400AAA
:10545000F2EE0E1AB1EE041A3AF0B2FB95F82F14E0
:105460001A222046FFF7A0F960B921220121204627
:10547000FFF79AF995F8793E43F0020385F8793EF3
:1054800003B0F0BD064A137843F008031370F1E748
:10549000D0250020F8600020BD500108B950010857
:1054A000A461002070470000002070477047000092
:1054B0000020704700207047002070470020704790
:1054C0009FED010A704700BF000000009FED010A38
:1054D000704700BF000000007047000000207047C8
:1054E0007047000010B50446143000F019F804F1BC
:1054F0002C0000F015F804F174005AF04DF904F195
:10550000F4005AF049F94FF0FF33C4F85031204607
:1055100010BD0000014B1868704700BF1C610020DF
:1055200070470000F0B52DED048B91B004466D4638
:10553000284605F0E9F994F8BC33002B72D004F545
:105540007A730FCB85E80F0094F8F833D4EDEC8A2A
:1055500094EDED8A94EDEE9A002B63D094F8D0335D
:10556000002B5FD02D22002104A8D4F8C073D4F8FA
:10557000C463D4F8C853D4F8CC4381F07DFDA32391
:105580008DF8103095238DF8113046238DF81230A8
:105590005AF0FEF89FED250A9FED257ACDF81710F9
:1055A00068EE807ACDF8130067EE877AFDEEE77A31
:1055B00017EE903A68EE007A29EE000A67EE877AD5
:1055C000ADF81B30FDEEE77A20EE070A17EE903AB1
:1055D000ADF81D3016F0D0FFDDED017A9FED157AA4
:1055E000CDF82D70BCEEC00AF8EEE77A10EE103A56
:1055F00067EE877AADF81F3017EE903ACDF821307C
:10560000029BCDF82530039BCDF82930CDF83160D1
:10561000CDF83550CDF8394038F0E6FA2D2204A9FE
:1056200037F034FC11B0BDEC048BF0BDE02E6542C8
:105630000000C8420AD7233C30B52DED028B8BB059
:10564000044624220D4601A8002181F015FDA32364
:105650008DF8043095238DF8053048239FED1F8A7F
:105660008DF806305AF094F8D4ED817A2B68CDF895
:105670000F3067EE887A95ED020ACDF80B1017EE21
:10568000903AD4ED827ACDF8133067EE887A6B6861
:10569000CDF8173017EE903ACDF80700CDF81B3053
:1056A00016F040FF10EE103A94ED830ACDF81F304B
:1056B00020EE080A16F036FF10EE103ACDF823302F
:1056C00094F80C338DF8273038F08EFA242201A993
:1056D00037F0DCFB0BB0BDEC028B30BDE02E654239
:1056E00030B587B014460D4618220021684681F077
:1056F000C3FCA3238DF8003095238DF80130492396
:105700008DF802305AF044F8A3680393E3680493D9
:105710006368CDF807100593CDF803008DF80B50A2
:1057200038F062FA1822694637F0B0FB07B030BD96
:1057300010B58EB0044602A805F0E6F802A920468E
:1057400001F0C8FA002845D001F00EFD694601F0CD
:1057500047F91F22002106A881F08EFCA3238DF8B3
:10576000183095238DF819304A238DF81A305AF0E5
:105770000FF8DDED037A9FED1B7A049BCDF8233003
:10578000F8EEE77A059BCDF8273067EE877ACDF8FB
:105790001B0017EE903ADDED007ACDF82B30F1EEDC
:1057A000677A17EE903ACDF81F10204601A9CDF880
:1057B0002F3000F01DFC78B1DDED017AF1EE677A53
:1057C00017EE903ACDF8333038F00EFA1F2206A9C2
:1057D00037F05CFB0EB010BD38F006FADFED027A50
:1057E000EEE700BF0AD7233C5241C07F002303608D
:1057F00043608360C360036143618361C36103628B
:105800007047000090F8F432B02202FB030390F8D6
:10581000382393F8D13012B1012B28BF0123184649
:10582000704700002DE9F04F04468BB04FF0000A9E
:105830000D461AF055FD84F814A204F506704FF0D9
:105840007E5759F053F94FF47A73A4F8623284F812
:105850006852C4F84872C4F84C72C4F8507204F527
:105860001B70002505F050F804F52B790323C4F8CC
:10587000803204F53476C4F89452C4F89852C4F8CF
:105880009C52C4F8A052C4F8A452C4F8A852484686
:10589000FFF7ACFF04F5487B3046FFF7A7FFC4F8DD
:1058A0001453C4F81853C4F81C535846FFF79EFF0E
:1058B000C4F84453C4F84853C4F84C53C4F8505384
:1058C000C4F85453C4F85853C4F85C53C4F8605334
:1058D000C4F86453C4F86853C4F86C53C4F87053E4
:1058E000C4F88C53C4F89053C4F89453C4F8A85324
:1058F000C4F8A453C4F8A053C4F8B053C4F8B453C4
:10590000C4F8B853C4F8CC53C4F8C853C4F8C4534B
:10591000C4F89C73C4F8C07304F5757004F0F4FF08
:1059200004F57A7004F0F0FF04F58063C4F8FC53CA
:105930001D6004F5816304F583601D605D609D60FA
:1059400004F0E2FF04F22C4304F264481D605D6041
:105950009D606D4BC4F83C3404F50D73C4F84034BD
:1059600004F50E73C4F8443404F50F73C4F84834D6
:1059700004F51073C4F84C3404F24523C4F85034D1
:1059800004F51173C4F8543404F58B6340461D606C
:105990005D609D60FFF72AFF04F59160FFF726FF29
:1059A00004F5976304F23C421D605D609D6004F263
:1059B000C44304F2BC501D605D609D6004F59A63B1
:1059C0001D605D609D6004F2DC431D605D609D6054
:1059D00004F2EC431D605D609D6004F2FC431D60B9
:1059E0005D609D6004F5A1631D605D609D6004F2D3
:1059F0002C53C2F8E070C2F8E4701D605D609D60D9
:105A000004F5A7631D605D609D6004F244531D6052
:105A10005D609D6004F5AC631F605D6004F28453BB
:105A20001D605D609D6004F5B2631D605D609D60FA
:105A300004F5B5631D605D609D6004F065FF04F2D0
:105A4000CC5324221D605D6004F2D45351461D6086
:105A50005D6004F2DC5340461D605D6081F00CFB2C
:105A600004F2FC50C8F82070C8F81070C8F8007034
:105A7000FFF7BCFE04F5C46304F5CA601D605D60F9
:105A80009D6004F22C631D605D609D6004F5C7633A
:105A90001D605D609D6004F244631D605D609D60FB
:105AA00004F032FF194B1A491C60204633F066FEA1
:105AB00051462422584681F0DFFAC4F84073C4F8F6
:105AC0003073C4F8207304F5257207CA04F52873EF
:105AD00083E80700484694EDAA1AD4EDA90A94ED8C
:105AE000A80A17F081F93546494668466E4617F010
:105AF0009DF80FCE0FC50FCE0FC533682B60204623
:105B00000BB0BDE8F08F00BFAC000A082061002098
:105B100074FF090810B5044688B001F0F1FB94F950
:105B20003232012B02D1274804F0D2FE022B0AD1D7
:105B3000032384F8323204A9012304F111008DF803
:105B4000103034F0E3FB94F8323284F8903204F2EF
:105B50003C4001F049FB94F93132642B30D165238C
:105B600004A904F231208DF8103034F00DFC04A9A2
:105B7000204632F06DFF18B304238DF8183000234F
:105B8000CDE9013303930F230593694604A833F04D
:105B9000DFF8059B28B108AA02EB8302009942F8BE
:105BA000581C0133112B0593EFD957F095F99DED52
:105BB000031ADDED020A9DED010A652157F04AF94D
:105BC00008B010BD58FE090870B500F5257600F53F
:105BD00028758CB004463146284618F0DBFDE0B944
:105BE00096E8070085E8070004F52B7194EDAA1AE2
:105BF000D4EDA90A94EDA80A0191084617F0F4F82B
:105C000002AD019902A817F011F80FCD04F5347414
:105C10000FC40FCD0FC42B6823600CB070BD000003
:105C200013B540F2411200F50671044601A812F0C6
:105C300021FD04F23C4001F001FD20461AF098FDE0
:105C400001A812F039FD02B010BD0000F8B50B68D4
:105C5000C0F804324B68C0F808328B68C0F80C32C8
:105C600001F10C0607460C4600F548750FCE0FC52E
:105C70000FCE0FC533682B6004F1300207CA07F559
:105C8000457383E8070004F13C0207CA07F5517326
:105C900083E8070004F1480207CA07F5547383E854
:105CA0000700543494E8070007F5577383E80700AA
:105CB000384601F039FC3846BDE8F84001F01CBC1C
:105CC00013B5044600F23C40019003F0FFF804F5E0
:105CD000BE610198009102F009FC0099204602B0D3
:105CE000BDE81040FFF7B2BF4A78064BC2F340123E
:105CF0001A754A78C2F380125A750A78C2F30012F4
:105D00009A7570478561002013B540F2F52204466C
:105D100000F5067101A812F0ADFC002104F23C4030
:105D200001F000FF94F8603223B120461AF03CFFE6
:105D300084F8600201A812F0BFFC02B010BD0000A0
:105D400038B590F80C3305460C462BB1032B0BD01D
:105D500095F86832DB070CD405F5CA630FCB84E8ED
:105D60000F0095F8600603E01AF082FD0028EFD0DE
:105D700038BD0020FCE7000000F23C4090ED380AFE
:105D80007047000000F23C4090ED390A7047000077
:105D900010B490F80C230C462AB1032A0AD0002034
:105DA0005DF8044B704700F5B56007C884E807004C
:105DB0000120F5E75DF8044B1AF018BD90F8840354
:105DC000431E58425841704738B590F80C330D4681
:105DD0008BB900F23C4001F0A3FC044610B900244A
:105DE000204638BD01F0F0FBD5ED007A27EE800AA1
:105DF00085ED000AF4E7D0EDE07AC1ED007A90F885
:105E00007C43002CEBD090EDDE7ADFED086AB4EE37
:105E1000E67AF1EE10FAF7EE006AB8BFB0EE667AF5
:105E200067EE877AC1ED007ADAE700BF0000003440
:105E300090F80C33032B01D11AF058BC00207047A6
:105E400090F80C23032A01D11AF0D6BD00F23C4091
:105E500002F0CAB830B590F80C3385B004460D4650
:105E60008BB1032B18D004F5257018F0CDFC284613
:105E700001A98DED010ACDED020A8DED031A18F08E
:105E800055FA012006E000F23C4001F0F3FB002847
:105E9000E9D1002005B030BD90F86032002BF8D079
:105EA0001AF084FDDFE700007FB590F80C2332B1D3
:105EB000032A4FF0000309D0039304930CE000F28F
:105EC0003C4007B05DF804EB01F0B0BC03A90393BC
:105ED000049305931AF000FC9DED030ADDED040A1E
:105EE00007B05DF804FB000007B590F80C3333B140
:105EF00000F57F7003B05DF804EB18F0AFBB00F263
:105F00003C4001F093FC68468DED000ACDED010A9E
:105F100018F0A4FB03B05DF804FB000090F80C033C
:105F2000003818BF0120704708B590F80C23032AE9
:105F300005D0BDE8084000F23C4001F05FBC1AF01B
:105F4000CBFB012008BD000010B590F80C230C46D7
:105F50001AB1032A07D0002010BDBDE8104000F29E
:105F60003C4001F0EFBB1AF0CDFB012084ED000AAC
:105F7000F2E7000090F80C33032B01D11AF0D6BCE5
:105F80000020704730B590F80C3385B005460C46BC
:105F900023B1032B09D0002005B030BD00F23C40F6
:105FA00005B0BDE8304002F0D1BA002302A9029347
:105FB00003931AF079FB0028EDD001A928461AF0C6
:105FC0007FFB0028E7D0029B2360039B6360019B5B
:105FD000A360E1E790F80C231AB1032A05D0002052
:105FE000704700F23C4002F0E5BA1AF05DBB0000D9
:105FF00090F80C231AB1032A05D00020704700F254
:106000003C4002F0C9BA1AF05BBB000090F9323292
:106010003BB990F8683213F0010F14BF0320002041
:106020007047032070470000F7B50446FFF7EEFF06
:106030000546002862D0032839D194F860326BB34A
:1060400094F86832D8072BD501A920461AF0DEFE55
:10605000BDF80430002B18BF002594F8146206F038
:10606000FD06012E4AD10023032D019307D101A97A
:1060700020461AF0D7FE20461AF0D6FC064604F257
:106080003C4002F015FB08B994F809039DF8043070
:10609000D90703D55A0701D59F0632D400252DE034
:1060A00020461AF071FA002808BF0025D5E7002520
:1060B000D3E713F0020F2EE094F9443223B99DF890
:1060C0000430DB092FD0E9E7002EF8D00EF0C0F93C
:1060D000FFF798FB022807D99DF805309806DDD513
:1060E0009DF80430D906D9D5FB6A93F89C30002B73
:1060F000E5D118E0DA0601D41B0718D5284603B00D
:10610000F0BD0028FAD094F80923B4F96436002AC7
:10611000CFD013F0010FF1D1154B1F68FB6A93F834
:106120009C30002BC8D19DF804309C07E2D405F0C8
:106130002BFC05F027FB0028B0D10EF089F9FFF702
:1061400061FB0228AAD90EF083F990F8F432B0224C
:1061500002FB030090ED3B7AF0EE007AB4EEE77AB2
:10616000F1EE10FA9AD59DF80530DB09C6D195E716
:10617000F86000202DE9F04790F8603292B00446B4
:10618000002B00F0948020461AF08CFF2046FFF789
:106190004BFF03287BD104F5487800274146204671
:1061A0000097019702971AF0D7FB694620461AF02C
:1061B000C9FB009BC4F80432019BC4F80832029B5F
:1061C000C4F80C32204601F0AFF9204601F094F9F2
:1061D00015F0F4FC054620461AF058FA0028A8BF2E
:1061E000C6B203AA4FF0FF312046BCBF95F8EB942E
:1061F00095F8EC640397A8BFB146049705971AF089
:106200008FFA03A818F000FB4FF00C0A0AFB0950A4
:1062100084EDD10AC4EDD20A84EDD31A04F551718C
:1062200000F55C7018F000FB04F557770AFB065583
:1062300084EDC50AC4EDC60A84EDC71A3A464FF08C
:10624000FF31204605F500751AF07EFA95E8070043
:1062500006AE86E807003946304618F04BFB04F5D9
:106260002B72414609A816F071FC314609A816F0B8
:10627000EFFB09A9204684EDD40AC4EDD50A84EDCC
:10628000D61A1AF0CFFD09A92046FFF72DFD94F884
:106290006636002B3AD109A804F036FB09A920463E
:1062A0001AF0F2FA90B3012384F866362EE0D0F8A3
:1062B00064321BB959F064FAC4F86402154B1B68C8
:1062C000D86A03685B68984788B159F059FAD4F8DE
:1062D0006432C01AB4F86232984204D920461AF0E7
:1062E00063FC84F8600294F860327BB14BE759F0AC
:1062F00047FAD4F86432C01A41F287339842E4D89E
:1063000037F072FC37F056FC0028DED112B0BDE841
:10631000F08700BFF860002090F80C3323B1032B06
:106320004FF0000007D0704790F93222032A04D1C1
:106330000A70012070470870FBE71846704700009C
:1063400073B50D460DF107010446FFF7E5FF06465C
:1063500028B19DF807302BB1032B09D00026304619
:1063600002B070BD04F5CA630FCB85E80F00F6E7F5
:10637000294620461AF07CFA94F86062EFE70000A4
:106380007FB50E460DF103010446FFF7C5FF054634
:1063900018B90025284604B070BD9DF8033083B1BC
:1063A000032B16D004F5257018F02EFA01A93046FB
:1063B0008DED010ACDED020A8DED031A17F0B6FF3F
:1063C000E8E7314604F23C4001F054F90028E9D1F5
:1063D000DFE794F86032002BDBD0314620461AF01C
:1063E000E5FADFE737B50D460DF107010446FFF783
:1063F00093FF28B19DF8073023B1032B0FD0002065
:1064000003B030BD04F5BE631B682B6004F2F45387
:1064100004F5BF641B686B602368AB60F0E720463F
:1064200029461AF08FFA94F86002E9E710B504469D
:10643000FFF7ECFD18B1032807D0002010BD04F2CF
:106440003C40BDE8104001F03FB994F86032002BA9
:10645000F3D020461AF098F80028EED094F81432C1
:1064600003F0FD03012BE9D194F80C03C31E58423D
:106470005841E3E710B50446FFF7C8FD80B1032893
:1064800010D194F8600250B159F07AF9D4F864321E
:10649000C01A44F62063984294BF0020012010BD2A
:1064A0000120FCE70020FAE708B50246FFF7AEFD41
:1064B000032804D110461AF0B5FC012008BD0020C5
:1064C000FCE7000030B585B004460191FFF722F8E3
:1064D0000199054610B9002005B030BD0191FEF7C5
:1064E000E9FF01990028F6D02846FEF7E7FF0028CB
:1064F000F1D0B4F864365907EED494F80933002B80
:10650000EAD00B4A1268D26A92F89C506DB103A986
:106510002046FFF7C9FF30B19DF80E309A07DBD552
:10652000C3F38000D8E72846D6E71846D4E700BF73
:10653000F860002010B50446FFF768FD032804D179
:106540002046BDE810401AF069B9002010BD0000D7
:106550002DE9F04190F80C338CB00027032B064650
:106560000C46154600970197029719D11AF08EF83C
:106570006A4680464FF0FF3130461AF0E5F8B8F130
:10658000FF3FA760676027600DD115F017FB2B4612
:1065900090F8EC14224614F041FA0CB0BDE8F081FA
:1065A0004FF0FF38EBE715F009FB2B4622465FFA68
:1065B00088F114F033FA95ED000A684618F060F996
:1065C00003A920468DED051A8DED030ACDED040AD1
:1065D00018F090F906F52B7206F5487103A816F02D
:1065E000B5FA214603A816F033FA84ED021A84EDB9
:1065F000000AC4ED010A95ED007ADFED037AA7EEFB
:10660000271A84ED021AC8E70AE81C411FB5DFED1E
:106610000B7A20EE270A0C461946094BCDE90042B9
:10662000BDEEC00A18688DED020A064B9DF81820D1
:10663000C06A12F0FDF904B010BD00BFE02E654243
:10664000F86000206CFE09082DE9F0472DED028B63
:1066500092B0002504460F464FF07E5A00F548716F
:1066600006A89046CDF818A009950895079517F04B
:10667000A7FA05F089F905F085F881462046FFF76D
:10668000C5FC032803D094F80C33032B4FD19FEDA6
:10669000558ADFED558A00262379F2B2934247D915
:1066A0000AAA71B22046CDF828A00D950C950B953D
:1066B0001AF05CF90AA906A817F0AAFEB4EEC80AF7
:1066C000F1EE10FA0DDD494ACDF800803B4648490D
:1066D0002046FFF79BFF002012B0BDEC028BBDE807
:1066E000F0870AA906A803950495059517F07AFE88
:1066F00003A90EA88DED0E0ACDED0F0A8DED101A2F
:10670000CDED111A17F0E2FBB9F1000F0DD09DEDA0
:10671000050AB0EEC00AB4EEE80AF1EE10FA04DDA4
:10672000344ACDF800803B46D1E70136B4E7002378
:1067300094F8686216F0010001D0012BCCD104F26C
:10674000FC510AA8CDF828A00D950C950B9517F0D3
:1067500037FA0AA906A817F05BFEDFED227AB4EE3D
:10676000E70AF1EE10FA05DD204ACDF800803B463D
:106770002149ADE72046FFF749FC03282DD12046EB
:106780001AF046F994F86832DB0728D438BB0AA916
:1067900006A803950495059517F024FE03A90EA8F5
:1067A0008DED0E0ACDED0F0A8DED101ACDED111AFB
:1067B00017F08CFBB9F1000F11D09DED050ADFED4C
:1067C0000A7AB0EEC00AB4EEE70AF1EE10FA06DD7E
:1067D000084ACDF800803B46CAE70020D2E70120F6
:1067E0007AE700BFC2B8323EC2B8B23E98FE09088E
:1067F000A3FE0908A7B50908A8FE09082DE9F74373
:106800001446054688460193FFF710FE019A074695
:1068100038B92448244B00682146C06A12F008F9B0
:10682000019A019221462846FFF70EFF064630B333
:106830002846FFF7EBFB95F80C33019A83420DD005
:1068400005F0A2F804F09EFF019A38B1174B1548E5
:1068500000682146C06A12F0EBF810E02846FFF706
:10686000D5FB18B103280FD0114BF0E71346414672
:10687000224605F23C4000F03BFF00B107B900267C
:10688000304603B0BDE8F08395F86092B9F1000F8F
:1068900001D1084BDBE7134641462246284619F052
:1068A00083FEEAE7F8600020ACFE0908B8FE09089C
:1068B000E8FE0908D7FE090890F80C33032B01D134
:1068C0001AF0C6BA0020704737B5054600F50671C4
:1068D00040F6033201A811F0CDFE2846FFF796FBE3
:1068E000044640B103280AD0002401A811F0E4FEB8
:1068F000204603B030BD284619F054FFF5E728467E
:1069000019F050FF0446F0E708B50246FFF77EFB9A
:1069100010B1032806D008BDBDE8084002F23C4093
:1069200000F09CBEBDE8084010461AF087BA00008F
:106930000B4610B411462BB1032B09D000205DF893
:10694000044B70475DF8044B00F23C4000F09CBEE5
:106950005DF8044B19F098BF13B50446FFF756FBDA
:106960000A46014620460192FFF7E2FF70B9084B44
:10697000019A1B68DB6A93F89C0038B194F80C13F9
:10698000204602B0BDE81040FFF7D2BF02B010BDF4
:10699000F860002037B504460D4640F2B25200F5CB
:1069A000067101A811F066FE2946204619F08AFFFB
:1069B00094F80C33032B054610D148B104F58361DC
:1069C0002046FFF7C9FF84F82804204600F0DCFDCC
:1069D00001A811F071FE284603B030BD0025F7E78D
:1069E00070B590F87C32DB0786B004460D460CD4B7
:1069F00003F018F8437C242202FB0300D0ED0B7A4D
:106A0000F1EE677AC5ED007A3BE002A803F07CFF67
:106A100001A92046FFF7ECFAE8B90DF019FD94F949
:106A20004432022B0646E3D1FEF7ECFE0228DFD902
:106A300096F8F4029FED147AB02303FB0066D4F8B5
:106A40007032D6F8E0209B1A07EE903AF8EEE77A1B
:106A500067EE877AD6E702A92046FFF77DFF002878
:106A6000DBD0D4F87022039BDFED076A9DED017A3D
:106A70009B1A07EE903AF8EEE77AA7EEE67A85EDF4
:106A8000007A06B070BD00BF0AD7233CF0B50C46B3
:106A900087B000F50671064640F6863201A811F06F
:106AA000E9FDA36853B9E36843B9636833B90027C4
:106AB00001A811F001FE384607B0F0BD204603F0F2
:106AC000F9FF0028F3D094E80F0002AD85E80F002D
:106AD0000021284603F0B0FF07460028E7D096F8CB
:106AE0007C32DB0704D437F07FF8192136F0B8FF89
:106AF00095E80F0006F51B7C8CE80F0096F87C32B9
:106B000043F0010386F87C32304600F03DFD40F052
:106B1000ABFA462141F0C6F840F0A6FA452141F013
:106B2000C1F8054BA2681B68DB6A1A61E2685A610A
:106B300062689A61BCE700BFF860002038B5144B6A
:106B40001B68DD6A2B6804465B6828469847F0B1ED
:106B50002B690BB96A69D2B1C4F874326B69C4F895
:106B60007832A969002204F51B7003F0D3FE94F873
:106B70007C3223F0030343F0030384F87C3240F0BB
:106B800073FABDE83840034A062139F029BC38BD04
:106B9000F8600020FCFE090813B504460193FFF7D6
:106BA00035FA0328019B05D1204602B0BDE810400C
:106BB00019F006BF002002B010BD000010B588B06B
:106BC00004460593FFF722FA0328059B4FF00000C7
:106BD0000AD10690079006A802900B9801900A9897
:106BE0000090204619F0FAFE08B010BD38B50446F2
:106BF000FEF790FC0546D0B194F80C33032B03D07C
:106C000095F84E41204638BD204619F0FBFDFF287F
:106C10000446F5D001462846FEF750FC0028EFD088
:106C200021462846FEF746FC0028E9D0EAE704465C
:106C3000E8E7000008B590F80C33032B05D014F0FA
:106C4000BDFF90F9EB04C0B208BD19F01FFD431C55
:106C5000F9D1F4E708B590F80C3383B1032B03D1D5
:106C6000BDE8084019F00ABD35F002FB40F6ED42E0
:106C70004FF4801135F0B4FA4FF0FF3008BD1846DC
:106C8000FCE7000090F80C33032B01D11AF056BB3F
:106C90007047000090F80C33032B01D119F0D2BBE0
:106CA0007047000019F058BC10B504461CF0D4FB26
:106CB0002046FEF737FC2046BDE81040FEF738BD01
:106CC00090F80C330BB1032B01D11AF0B3BB0020A9
:106CD0007047000030B500F5757304460D460FCBC4
:106CE00085E80F0094F8E40330BD00007FB5054649
:106CF00068460E4603F008FE95F87C32DB0703D4A5
:106D00000024204604B070BD69462846FFF7E2FF24
:106D100004460028F4D0694605F51B7003F0DAFF3D
:106D200086ED000AC6ED010AEBE70000D0F88033DB
:106D30000B6090F87C037047D0F888330B6090F8B4
:106D40008503704710B500F5637203460C4607CA09
:106D500084E8070093F8980310BD000030B500F5F3
:106D6000677304460D460FCB85E80F0094F8AC031B
:106D700030BD000030B500F5836304460D460FCBEF
:106D800085E80F0094F8280430BD000010B500F22B
:106D90002C4203460C4607CA84E8070093F83804DF
:106DA00010BD00002DE9F0432DED028B8BB00546A0
:106DB0000E461746FFF71AFF014680462846FFF7A2
:106DC00081FB0446002848D0FEF7A4FB4146FEF7AD
:106DD00077FB86ED000A95F93032002B3ADD0DF095
:106DE00037FBFEF70FFD012834D90DF031FB90F889
:106DF000F432D5EDDE7ADFED5D8A96ED000AB02241
:106E000002FB030095F93032D0ED3B0A07EE103A51
:106E1000F4EEE87AB8EEC77AF1EE10FAB7EE008A2F
:106E2000B8BFF0EE487A37EE201A20EE270A70EE4F
:106E3000C70A40F2B63015F0DFFBD5EDDE7AF4EE8E
:106E4000E87AF1EE10FAB8BFF0EE487A80EE277AD1
:106E500086ED007A01233B7003E095F8083333B9DF
:106E6000387020460BB0BDEC028BBDE8F08395F87E
:106E70000C334FF00009CDF80490CDF80890CDF810
:106E80000C9043B1032B10D0CDF81090CDF8149096
:106E9000CDF818907CB902233B703246414605F28A
:106EA0003C4001F0C9FB0446DBE701A9284619F084
:106EB0009DFC0446E8E795F80C33002BEBD004A9C1
:106EC0002846FFF763FF04460028E4D001A904A880
:106ED00017F0C0FC07A8CDED080A8DED091A8DED5D
:106EE000070A18F0CBF804A8B0EE408A18F0C6F8EC
:106EF00095F93032002B30DD07EE903AF8EEE77A64
:106F00004FF47F7070EE670A37EE801AF5EEC00A14
:106F1000F1EE10FA48BFDFED160AF4EE410AF1EE89
:106F200010FAB0EE480AC8BFB0EE601A15F064FB64
:106F3000B0EE408AD5EDDE7A9FED0C7AF4EEC77A9A
:106F4000F1EE10FAB7EE007AB8BFF0EE477A88EEAD
:106F5000277A032386ED007A7DE7B5EEC08AF1EE4D
:106F600010FA48BF9FED028AE4E700BF000000343A
:106F70000000000010B50446FFF75CFE84F80D0326
:106F80002046FFF757FE84F80E032046FFF752FE17
:106F900084F80F032046FFF75DFE04F55A7184F86C
:106FA00010032046FEF7F4FE84F8740300F00CFB97
:106FB00004F5617284EDDE0A04F560712046FFF786
:106FC000F1FE04F5627184F87C032046FEF7FCFEB6
:106FD00004F5637184F885032046FEF729FF04F564
:106FE000677184F898032046FEF734FF04F56C714E
:106FF00084F8AC032046FFF7F5F904F5707184F8C6
:10700000BC032046FFF7BCF904F5757184F8D00382
:107010002046FEF795FE04F57A7184F8E4032046D5
:10702000FFF78EF984F8F8032046FEF73DFF04F5DC
:10703000806384EDFF0A2046C3ED000AFEF754FF8B
:1070400004F2044383ED000A04F2144204F5816162
:107050002046FFF77DFA04F583612046FFF77CFCAC
:1070600004F22C4184F828042046FEF75DFF84F8E2
:10707000380410BD37B50D46044600F041F91DB97E
:1070800014F09CFD13F09EFB4FF4BE7204F50671E4
:1070900001A811F0EFFA94F869322BB92046FFF7F6
:1070A0004DFD012384F86932224B1D68A86A0368EC
:1070B0009B6998472046FEF787FD2046FEF700FEB5
:1070C000204600F093FA2046FFF754F8286B30B1C1
:1070D0000368D4EDD20ADB6894EDD10A9847D4F85E
:1070E000100208B159F0BAFA204600F07DF82046A7
:1070F000FEF79AFF94F8903284F80C0383420ED086
:1071000084F8900298B10C4D0C4B032808BF1D4623
:107110003FF0AAFF0A4A2B46062139F061F92046C2
:10712000FFF728FF01A811F0C7FA03B030BD054DE5
:10713000EEE700BFF860002033CE0908A3FE09087F
:1071400014FF0908A8FE0908D0EDDE7A9FED057A44
:10715000F4EEC77AF1EE10FAB7EE000AA8BFB0EE6F
:10716000670A704700000034014B1868704700BF81
:10717000206100204FF0FF30704700000120704771
:1071800070470000002070470020704770470000E3
:1071900070470000002070470020704700207047B3
:1071A0000020704700207047002070470020704783
:1071B000012070470368D3F89430184700207047C7
:1071C0000020704700207047002070470020704763
:1071D0000020704700207047002070470020704753
:1071E00000207047704700007047000008B514F099
:1071F000E5FC90F8EC0408BD08B514F0DFFC90F84D
:10720000EB0408BD30B52DED028B9FED1A1ADFEDB2
:107210001A0A91ED000A87B005462D200C468DED27
:10722000011ACDED000A15F0E7F99DED011ADDED2B
:10723000000AF0EE408A2E2094ED010A15F0DCF9E8
:107240009DED011ADDED000AB0EE408A2F2094ED8D
:10725000020A15F0D1F903A905F52570CDED038AD1
:107260008DED048A8DED050A33F072F907B0BDEC9F
:10727000028B30BDC2B8323EC2B832BE70B52DED01
:10728000048B00F5257403460E4694E8070084B08D
:10729000D3EDA57A9FED181A93EDA69A01AD85E876
:1072A000070030EE270AF0EE608A3A20DFED130A7D
:1072B00015F0A2F93B20B0EE408A9FED0F1ADFEDEA
:1072C0000F0A38EE890A15F097F98DED018A8DEDD8
:1072D000020A95E8070084E8070046B1002120462D
:1072E00004B0BDEC048BBDE8704031F0CDBB04B000
:1072F000BDEC048B70BD00BFC2B8323EC2B832BE16
:1073000010B5044658F03CFAD4F8F4321BB1C21A56
:10731000B2F57A7F12D30A4A1268D26A92F89C2098
:1073200002B15BB9C4F8F40294F8314214F046FC9F
:1073300080F8E24404F028FB80F8254010BD00BF2F
:10734000F86000202DE9F0432DED028B91ED007ADD
:10735000D1ED037A87B08DED047AB0EEC77AB5EE41
:10736000C07AF1EE10FADDE91087DDF84C90CDED32
:10737000057A0C4615461E4606DCF0EEE77AF5EE79
:10738000C07AF1EE10FA02DD04A817F0E5F96B20DF
:10739000B7EE001AFFEE000A9DED050A15F02CF974
:1073A0006C2089ED000AB7EE001AFFEE000A9DED91
:1073B000040A15F021F904A888ED000A17F028F94D
:1073C000B7EE008A002852D00023C9F8003088EDBB
:1073D000008AD4ED067A67EEA77AF4EEC87AF1EE69
:1073E00010FA4ADB0023336085ED008ADFED3F0AA7
:1073F00096ED000A7C20B7EE001A15F0FDF886ED38
:10740000000A95ED000A7D20B7EE001AFFEE000A93
:1074100015F0F2F885ED000AD4ED067A129BDFED47
:10742000346AF1EE677AC3ED007A96ED007AF0EEF9
:10743000C77AF4EEE67AF1EE10FA2BD503AB02AA86
:1074400001A9204615F030FD9DED018AB0EE480AF5
:107450007DF00AFA85ED000AB0EE480A7DF05AFB8D
:1074600087ED000A07B0BDEC028BBDE8F08304A8ED
:1074700017F0BAF80028A7D1ABE738EE670A15F085
:1074800017F886ED000A94ED087AC7EE007AC5ED8C
:10749000007AABE794ED076AC6EE077AC7ED007A8B
:1074A00096ED007AB0EEC77AB4EEE67AF1EE10FA15
:1074B000C4D495ED007ADFED0F6AB0EEC76AB4EE82
:1074C000666AF1EE10FAB9DCB4EE477AF1EE10FA22
:1074D000B4D6B0EEE77AB4EE667AF1EE10FAADDC2F
:1074E000F4EE677AF1EE10FABCD7A7E700000000CF
:1074F00000000034FFFF7F7F1FB500F51773039373
:1075000000F51673029300F51573019300F51473DB
:10751000009300F5127200F5137300F54871FFF740
:1075200011FF05B05DF804FB9FED156A90ED817ABF
:10753000DFED146AD0ED837A27EE067A67EE867A5D
:1075400027EE267A67EEA67ABDEEC77AFDEEE77AD9
:1075500080ED7E7A90ED827A27EE067A17EE903AE9
:1075600027EE267A002BB8BF03F50C43BDEEC77A91
:10757000B8BFA03380ED7F7AC0F80032704700BFFB
:10758000E02E65420000C8421FB50E4B1B68044642
:10759000B3B1684603F0B8F969462046FFF7EAFB45
:1075A00020B16A4600212046FEF79AF894F87C3212
:1075B000DB0705D504F51B7201212046FEF790F884
:1075C00004B010BDCC63002008B502F02BFABDE872
:1075D000084001F0C3BD000010B580F8F812044661
:1075E00058F0CEF8C4F8FC0210BD000010B590F8B9
:1075F000F832044653B158F0C3F8D4F8FC32C01A3C
:10760000B0F57A7F84BF002384F8F83294F8003311
:1076100053B158F0B5F8D4F80433C01AB0F57A7FF6
:1076200084BF002384F8003310BD000000F5B6705D
:107630000B4607C883E80700012070470023C0F805
:107640009C30C0F89830C0F89430C0F8A830C0F82A
:10765000A430C0F8A030C0F8AC30704770470000CC
:10766000024B0B604FF07C531360704700004842A0
:107670007047000008B50B4600F12801184616F0C7
:107680009FFA012008BD000010B500F5C0700C463F
:107690000FC884E80F00204603F026F930B1FFF749
:1076A00063FD00F51B700FC884E80F00204603F04F
:1076B0001BF980F00100C0B210BD000010B50446F7
:1076C00003F0F2FB204610BD10B5D0F87831044627
:1076D0005BB158F055F8D4F87831C01A41F28833CC
:1076E000984294BF0020012010BD0120FCE700005B
:1076F00013B5009303680192D3F890309847DDE901
:107700000021044628B90448044B0068C06A11F0FF
:107710008FF9204602B010BDF8600020ACFE0908C9
:1077200013B504460191FDF7F5FE2368019A1B6D20
:10773000014608B190F84E11204602B0BDE8104055
:107740001847000030B585B00023019302930393DE
:1077500003680D46DB6D01A99847044620B1039BE1
:107760002B60204605B030BD02F05CF9417C01F091
:1077700031FE04460028F4D002F054F901F090FDE7
:10778000B1EE400A85ED000AEBE7000090ED007ACB
:10779000DFED0F7AB0EEC77AB4EEE77AF1EE10FAC9
:1077A00014D590ED017AB0EEC77AB4EEE77AF1EE37
:1077B00010FA0BD590ED027AB0EEC77AB4EEE77A04
:1077C000F1EE10FA4CBF01200020704700207047F6
:1077D0000000003410B5FDF79DFE044658B190F846
:1077E0004E11FDF767FE30B194F84E112046BDE80A
:1077F0001040FDF763BE002010BD000038B50D46F7
:107800000CF026FE0446FDF7FDFF022881BF94F828
:10781000F402B02303FB004000F5827089BF07C863
:10782000002085E80700012038BD00002DE9F04365
:107830002DED028B8FB003680025DB6C039504955A
:1078400005950695029502A904469847064638B163
:10785000FFF7BAFEDDED027A27EE800A8DED020A0F
:107860000CF0F6FDFDF7CEFF0746002E50D0DDED03
:10787000027AD4ED6A6A94ED6B7A23680B9527EE51
:10788000877A67EEA67A8DED097ACDED0A7A0C95A6
:107890000D959B6C0BA9204609AD98470BA928466E
:1078A00016F010FE012F8DED030ACDED040A40F213
:1078B000B3800CF0CDFD90F8F432DFED5B7AB025AB
:1078C00005FB030090ED3C8A28EE278AB0EE480ABB
:1078D0007CF0CAFFF0EE408AB0EE480A7DF01AF95B
:1078E000CDED0B8A8DED0C0A0CF0B2FD90F8F43260
:1078F00005FB030090ED3B0A0BA816F003FE09AD53
:107900008DED050ACDED060A05A896BB03C885E0F6
:107910000128CED89DED020AB5EEC00AF1EE10FAAC
:107920007FDD07AED4F8AC21D4F8A83107923046F9
:10793000089316F011FE23680B950C950D959B6C22
:107940000BA920469847DDED077A9DED0B7A77EE7F
:10795000877A9DED0C7ACDED077ADDED087A77EE2A
:10796000877A09ABCDED087A96E8030083E8030037
:1079700049E0236993ED000AB7EE008A38EE408AA9
:1079800016F0C0FD04F5C8798DED090A4846B0EE41
:10799000480ACDED0A0A16F0B5FD0BA92846CDED33
:1079A0000C0A8DED0B0A16F08DFD04F5D07603AFB1
:1079B000C4ED650A314684ED640A384616F092FD3E
:1079C00004F5CC788DED090A4046B0EE480ACDEDBD
:1079D0000A0A16F097FD0BA928468DED0B0ACDED8E
:1079E0000C0A16F06FFD97E8030084ED660AC4EDFB
:1079F000670A86E803004946404616F063FD8DEDB0
:107A0000090ACDED0A0A9DED090ADDED0A0A0FB05B
:107A1000BDEC028BBDE8F083DDE9030185E80300DE
:107A2000F1E709950A95EEE735FA8E3C10B590F826
:107A30004213044603F0D2FB7C23C0B203FB004494
:107A4000D4F8A00010BD0000044B026F1B68DB6A75
:107A50005A60426F9A60826FDA607047F860002067
:107A6000F0B58FB0044614F0A9F8002302930393F5
:107A7000049390F8EB1401AB02AA054612F070FFD4
:107A800004F19407D8B39DED010AB5EEC00AF1EEFA
:107A900010FA34DD02A816F003FF04F1B00684EDFD
:107AA0002C0AC4ED2D0A84ED2E1A3946304616F004
:107AB00007FF04F17C01304616F0B6FE04F18801A0
:107AC00005A88DED050ACDED060A8DED071A16F015
:107AD000ABFE08A88DED080A9DED010ACDED090A5F
:107AE0008DED0A1A16F0CCFE0BA904F128008DEDDD
:107AF0000B0ACDED0C0A8DED0D1A15F081FA95F8F3
:107B0000EB040C2303FB0050394600F55C7016F0C3
:107B10008BFE84ED2C0AC4ED2D0A84ED2E1A0FB0D5
:107B2000F0BD00002DE9F047824B00251F682DEDC8
:107B3000028BC0F89C50C0F89850C0F89450C0F820
:107B40008450C0F88050C567C0F89050C0F88C5081
:107B5000C0F88850C0F8B850C0F8B450C0F8B05061
:107B60000446F86A03688AB05B680E46984704F1D9
:107B70002809002854D057F003FE42F20F739842B0
:107B80004ED8FB6A9FED6C8A93ED010A84ED1C0AC6
:107B9000D3ED020AC4ED1D0A93ED031A484684EDA5
:107BA0001E1A15F021F93FF05FFAD4ED1E7A67EE48
:107BB000887A054617EE900AF8F79EFCD4ED1D7AF8
:107BC00067EE887ACDE9040117EE900AF8F794FC85
:107BD000D4ED1C7A67EE887ACDE9020117EE900A9F
:107BE000F8F78AFC554ACDE900010621284638F00D
:107BF000F7FB94ED1E8AB0EE480A7CF035FE84ED6A
:107C00006B0AB0EE480A7CF085FF84ED6A0A57F0F3
:107C1000B7FDC4F87C010AB0BDEC028BBDE8F0876B
:107C2000A6B194ED1C0AB4EE400AF1EE10FA0DD69E
:107C3000D4ED1D0AF4EE600AF1EE10FA06D694EDCA
:107C40001E1AB4EE411AF1EE10FA52D713F0B6FF35
:107C500090F8EC344FF00C0A0AFB030303F50073B1
:107C6000074693E8070007AE86E807004FF01508BF
:107C7000B2EE028AF2EE068A304617F0FFF9B4EE51
:107C8000C80AF1EE10FA38D508F1FF3818F0FF08ED
:107C90003CD1304617F0F2F9F1EE047AB4EEE70A7F
:107CA000F1EE10FA43DD9DED090ADDED087A9DED58
:107CB000078A20EE000AA7EEA70A7DF041F9F0EE50
:107CC000400AB0EE480A7CF0F1FFDDED090A84EDD0
:107CD0001D0A9DED080AF1EE600AB1EE400A7CF043
:107CE000E5FF84ED1C0A9FED161AD4ED1D0A94EDF4
:107CF0001C0A484615F078F87BE7304617F0BEF9C5
:107D0000B4EEE80AF1EE10FABEDCC2E7384612F033
:107D100077FC384612F056FD97F8EC340AFB0373F3
:107D200003F5007393E8070086E80700A4E72567DA
:107D30006567D8E7F8600020E02E654234000A0845
:107D4000000000000021FFF7EDBE000037B504463B
:107D500008461546019117F091F9B7EE007AC7EE83
:107D6000007AB4F8DC3001980133A4F8DC3094EDEB
:107D7000367A37EE277A84ED367AB0EE007AF4EE72
:107D8000C77AF1EE10FA06D5B6EE007AF4EEC77AAD
:107D9000F1EE10FA0DDC9FED0E7AF4EEC77AF1EEFB
:107DA00010FA13D59FED0B7AF4EEC77AF1EE10FAC4
:107DB0000CDDB0EE670A16F063FD012085ED000AC8
:107DC000C5ED010A85ED021A03B030BD0020FBE7C6
:107DD00000247449BD37863570B52DED028B00F156
:107DE000280600F134058AB029460446304616F0CC
:107DF000C3FDB6EE008A20EE088A2846B0EE480A97
:107E000016F03EFD07A93046CDED080A8DED091AA2
:107E10008DED070A16F01EFD30468DED010AB0EE1D
:107E2000480ACDED020A8DED031A16F029FD07A9C7
:107E300028468DED070ACDED080A8DED091A16F0DA
:107E400009FD04A901A88DED040ACDED050A8DED0B
:107E5000061A16F0A5FD324601A920468DED070A47
:107E6000CDED080A8DED091AFFF770FF58B957F0EC
:107E700087FC0121C4F878012046FFF753FE0AB0C1
:107E8000BDEC028B70BD2A4604A92046FFF75EFFB9
:107E90000028ECD004F1400207A92046FFF756FF66
:107EA0000028E4D0EBE7000030B52DED028B0D4645
:107EB00083B091F842130446284603F08FF9C1B20B
:107EC0007C2000FB0151903104F1280014F01CFECD
:107ED00068468DED000ACDED010A16F0BFFBDFED1F
:107EE0001C7AB4EEE70AF1EE10FA05D59FED190AF7
:107EF00003B0BDEC028B30BD684616F02DFC684621
:107F000016F086FB0028F1D1284694ED488A03F04C
:107F1000C9FAF0EE400AB0EE480A14F095FA80B9BA
:107F2000284603F0BFFA84ED480AB0EE408A7CF0A0
:107F30009BFC84ED490AB0EE480A7CF0EBFD84ED31
:107F40004A0A04F59271684616F030FBD0E700BF8C
:107F500000000034000000009FED0C7AB4EEC70A68
:107F6000F1EE10FA0BD4DFED0A7AB4EEE70AF1EE87
:107F700010FA07DCC0EE077AB0EE670A7047F7EE3A
:107F8000007AF9E7F2EE047AF6E700BFF3665F3FA6
:107F900058A00B4108B51C3016F060FBF1EE007ADA
:107FA000B4EEE70AF1EE10FA9DBFF1EE027A37EE79
:107FB000C00ADFED047A9FED040A98BF20EE270A7D
:107FC00008BD00BFCDCC4C3ECDCCCC3D08B58369BF
:107FD00093F9000038B10CF03BFAFDF713FC0128CF
:107FE00094BF0020012008BDF8B52DED028B054699
:107FF00003F0CAFC03F0C6FB0446B8B3FFF7B4F8BD
:1080000090F8093393B32846FFF7E0FF064668B3BC
:108010000CF01EFA90F8F432B02707FB030090ED45
:108020003B7AF0EE087AB4EEE77AF1EE10FA1DD45E
:1080300095ED1E8A0CF00CFA90F8F432DFED1E7A02
:1080400007FB030090ED3C0A98EE270A14F080FA33
:10805000DFED1A7AB0EEC00AB4EEE70AF1EE10FADC
:1080600008DC57F08DFB3446C5F86801BDEC028B87
:108070002046F8BD05F5B67017F000F8B0EE408A5E
:108080000CF0E6F990F8F4329FED0D7A07FB03034C
:10809000D3ED3B7A67EE877AB4EEE78AF1EE10FA19
:1080A000DFD557F06DFBD5F86841001BB0F5FA6FCE
:1080B0008CBF00240124D9E7E02E65420000344241
:1080C000CDCC4C3F10B50A4B1B68DB6A93F89C3053
:1080D00004465BB957F054FBD4F87C31C01A44F61F
:1080E0001F6398428CBF0020012010BD0020FCE7D8
:1080F000F8600020F8B52DED068B04460CF0A8F9C9
:10810000054603F041FC064606F078F9002840F0E9
:10811000AB802046FFF768FF002800F0A8803046BB
:10812000FFF784FCD4F8E830984200F01A8130461A
:10813000FFF77CFCD4F8E830DFED8F7AC31A08EE45
:10814000903AF8EE688A304668EEA78AFFF76EFC30
:1081500094F8BC30C4F8E800F3B9304603F024FBCF
:10816000D0B104F1280796F842233946304603F08F
:108170009DF9D4ED1D0AB0EE401A384694ED1C0A64
:1081800014F032FE0023C4F89030C4F88C30C4F8E8
:108190008830012384F8BC3020463146FFF784FE46
:1081A00095F8F40205EB0015B0EE408AD5F8A03042
:1081B000C4F8EC3004F1B000D4ED129A16F05EFF72
:1081C0006368DFED6E7A93ED007AB4EEE77AF1EE54
:1081D00010FA68EE299AB0EE40AA01D5C3ED007AF4
:1081E0002046B0EE4A0AFFF7B7FE636820EE299AF0
:1081F00093ED000A29EE009AFFF7CCFE29EE009AD3
:10820000204684ED249AFFF75DFF38B1D4ED247A3F
:10821000B2EE007A67EE877AC4ED247AF0EE007A47
:10822000F4EEE78AF1EE10FA10D5DFED557AB4EEF0
:10823000E7AAF1EE10FA09D5DFED527A69EEA79AB6
:10824000D4ED2A7AE9EEA87AC4ED2A7A9FED4E0A97
:1082500094ED397ADFED4D7AB0EEC88A28EE008AC7
:10826000A7EE278A84ED398ABDEC068BF8BDFEF7B0
:108270007BFF90F80933002B73D02046FFF7A6FE52
:1082800000286ED095F8F42205EB0213D3F8A01065
:10829000D4F8EC308B4264D0B02606FB025292ED4B
:1082A0003B7AF0EE087AB4EEE77AF1EE10FA58DB9A
:1082B000CB1AC4F8EC1008EE903A95F8F4329FED22
:1082C000341A94ED1E0ADFED337A06FB0353D3ED27
:1082D0003C9A69EE819AF8EE688A39EEC00A68EE37
:1082E000A78A14F075F9B0EE409A7CF013FC94F86C
:1082F000BC30B0EE408AF3B1F3EE047AF4EEE78AD4
:10830000F1EE10FA17DC95F8F40206FB005595ED36
:108310003B7AF2EE027AB4EEE77AF1EE10FAFFF66B
:1083200049AFDFED1D7AB0EEC99AB4EEE79AF1EEEF
:1083300010FAFFF63FAF9FED198AD4ED1D0A94EDB8
:108340001C0AB0EE691A04F1280014F04DFD012357
:1083500084ED248A84ED238A84ED228A84F8BC305B
:1083600028E7BDEC068B04F188009FED0D0ABDE8FF
:10837000F84016F0D9BA00BFBD378635CDCC4C3D9C
:10838000C2B8B23E0AD7233CCDCC4C3ECDCC4C3FFC
:1083900035FA8E3C6F12833A1904863F00000000C4
:1083A000EC51783F30B50C2303FB010101F1C00310
:1083B000144693E807008BB004AD85E8070094E805
:1083C000070083E807002846FFF7E0F907AB58B13C
:1083D00094E8070083E807009DED070ADDED080A31
:1083E0009DED091A0BB030BD95E80700F2E70000DB
:1083F000F0B52DED028BD0F830318B60D0F83431F0
:10840000CB6085B004460D4601F00CFB06460CF02F
:108410001FF8A36993F90030022B07464BD1FDF7F3
:10842000F1F9022847D997F8F432B02202FB03731E
:10843000D3F8E0100022284602F06CFAD4ED500A7E
:1084400094ED4F0A284602F01BFD94F8443163B3C3
:1084500057F096F99FED228A97F8F4128DED018A74
:1084600001AA064638460BF077F8D4F838019FED9C
:108470001D0A361A07EE906AF8EE677A4FF48760A5
:1084800027EE800AB6EE001AF0EE480A14F0B4F8AF
:10849000DDED017A30EE270A04F584708DED010AD6
:1084A00016F030F8284602F0EBFC94F8440105B0D1
:1084B000BDEC028BF0BD707C242303FB006696EDBF
:1084C0000B8AFEF751FED0ED9C7A9FED077AF8EE0D
:1084D000E77AE8EE077AFDEEE77A17EE901AA9E759
:1084E000000000006F12833A0000C842F8B5036F25
:1084F0000B60436F4B60836F8B6000F14C050E4641
:10850000074601F10C040FCD0FC40FCD0FC42B682B
:10851000236007F1B00207CA06F1300383E80700C1
:1085200007F1940207CA06F13C0383E8070007F14C
:108530001C0207CA06F1480383E8070006F1600140
:108540003846FFF755FF86F87000F8BD30B589B0A2
:10855000044668460D4602F0D7F969462046FFF703
:1085600093F818B90024204609B030BD04A802F0E1
:10857000CBF9204604A9FFF73BFF04460028F1D0C1
:1085800004A9684602F0D4FB85ED000AC5ED010A96
:1085900085ED021AE7E700001FB500230C4601A98C
:1085A000019302930393FFF7D1FF08B1039B23606C
:1085B00004B010BD30B585B001AD00230C4629468E
:1085C000019302930393FFF7C1FF034618B195E8A7
:1085D000030084E80300184605B030BDF8B5064630
:1085E0000F461546FCF796FF044690B13946FCF756
:1085F00061FF70B120463946FCF760FF044640B188
:10860000FCF788FF3946FCF75BFF85ED000A204642
:10861000F8BDFEF7A9FD90F8083343B13046FFF7E7
:10862000D5FC044618B1D6F864312B60EFE7D6F8D4
:1086300064312B600024EAE770B52DED048B1646FB
:10864000FFF7CCFF054670B3FEF78EFD90F9304280
:108650004CB30BF0FDFEFDF7D5F8012823D9E4B2A9
:1086600007EE904AB8EE678A0BF0F2FE90F8F4320B
:1086700096ED009AB02202FB0300D0ED3B8AFEF794
:10868000A3FF38EE281A78EEC80A40F2614029EEBE
:10869000000A13F0B1FFB0EE408AFEF795FFC8EE76
:1086A000007AC6ED007ABDEC048B284670BD000050
:1086B00008B503F069F9BDE8084003F063B80000AD
:1086C00010B5044616F088F950B904F10C0016F004
:1086D00083F928B904F11800BDE8104016F07CB900
:1086E000012010BD38B500F1280504462846FFF7E3
:1086F000E7FF28B120460121BDE83840FFF712BA54
:10870000D4ED107AB7EE007AF4EEC77AF1EE10FAF3
:1087100006D5BFEE007AF4EEC77AF1EE10FA12DC5D
:108720002046FFF759FB2846FFF7CAFF0028E1D192
:10873000D4ED107AB2EE047AF0EEE77AF4EEC77A6E
:10874000F1EE10FAD6DC38BD10B5044616F096FCF2
:108750002046BDE8104016F0FBB800002DE9F04FB0
:108760002DED028BA3B000270446B0EE408A0A9795
:108770000B970C97FFF7BEFC13F020FA04F1F00BF7
:1087800005465E464FF0000804F1280A95F8F131DD
:10879000022B5FFA88F1A8BF02238B423AD9284600
:1087A000019111F04BFE019980B310AB13AA28463A
:1087B00013971497159712F031F99DED100AB5EE45
:1087C000C00AF1EE10FA21DD13A816F069F81CA911
:1087D00050468DED1C0ACDED1D0A8DED1E1A14F0CC
:1087E00037F916A88DED160AB0EE480ACDED170A36
:1087F0008DED181A16F044F81CA930468DED1C0AB0
:10880000CDED1D0A8DED1E1A16F05AF808F101087B
:108810000C36BBE795F8EC140C2303FB015101F572
:108820000071504614F014F984ED070A94ED450ADE
:10883000C4ED080A30EE088A84ED091A84ED458AF1
:108840000BF006FE0646FEF78FFC90F80933039303
:108850002046FFF7BBFB80B13046FCF7D3FF022870
:108860000BD996F8F4226169B02303FB026391F9F6
:10887000001093F80201884261DA94ED457ADFED49
:10888000847AB4EEE77AF1EE10FA62D494ED598A64
:10889000FEF7A0FF38B1FCF73DFE90F84E11FCF753
:1088A0000FFEB0EE408A236C626BA16A1E93B0EE9D
:1088B000480A1CA81D921C9115F0E2FF04F5B67140
:1088C0000AA88DED0A0ACDED0B0A8DED0C1A15F0F4
:1088D000F7FF56F055FF0023019084F82C31204615
:1088E000FFF774FB00286BD096F8F422B02101FB4F
:1088F0000262D2F8E430C4F8303196F8F43201FB69
:108900000363D3F8E830C4F8343156F039FF01235B
:10891000C4F83801C4F83C71C4F8407184F844319B
:10892000D4F81831002B5ED1019BC4F818310AAB82
:1089300093E8070004F5847484E8070009E006EB77
:108940000212D2F8A02001920199D4F818218A428B
:1089500004D123B0BDEC028BBDE8F08F03F5827328
:1089600093E8070094F82C310DF1280C8CE80700EF
:108970001BB904F5847383E807000123604684F87B
:108980002C3104F5B67115F065FF1CA904F14C00FB
:108990008DED1C0ACDED1D0A8DED1E1A14F086F822
:1089A000B5EEC00AF1EE10FA8DED1C0AD8BF9FEDAE
:1089B000370ACDED1D0A8DED1E1A84ED590A8EE79A
:1089C00094ED457AD4ED4F7ADDED0A6AE6EE877ACA
:1089D000DDED0B6AC4ED4F7AD4ED507AE7EE267ADE
:1089E000C4ED507A9CE7D4ED457A254B0D97F5EE12
:1089F000C07AF1EE10FA0E970F93AAD9214B9FED92
:108A0000227A1B68DB6A67EE877A93F89C300293C0
:108A1000B7EE007AC7EE278A002B4BD094F82C31A2
:108A200013B9039B002B43D0E36804F5847193EDE5
:108A3000008A0AA815F00EFF28EE888A8DED1C0A20
:108A40001CA8B0EE480ACDED1D0A8DED1E1A15F0DA
:108A500017FF16A90DA88DED160ACDED170A8DED9D
:108A6000181A15F02DFF0DA8FFF76EFE0DA815F0D2
:108A7000CDFFF8B156F084FEC4F8780169E700BF75
:108A8000000080BFF86000200AE81C4100000000E0
:108A9000CDCC4C3ECDCC4C3FCDCC4C3D920A06BF0C
:108AA000920A063FC2B8B23E728A0E3C5B82183907
:108AB000039B02931822002116A87EF0DDFA1822EB
:108AC00000211CA87EF0D8FA1FED108A05F20E5383
:108AD0000DF170084FF000094FF0FF37059395F83E
:108AE000F131022B1A465FFA89F1A8BF02228A42AD
:108AF0007AD98B4204916BD9059B13F80930002B6E
:108B000066D0B0EE680A584615F00EFF029B049935
:108B1000002B64D00C2222AB02FB0933A3F1180214
:108B2000049220465A460693FFF73CFC069B03ED51
:108B3000060A049BC3ED010A83ED021A4046FEF7C4
:108B400025FE002844D14046FFF7FEFD404615F0C3
:108B50005DFF00283CD10C2303FB09F222AB134438
:108B600007920DA9A3F1300240460492069315F036
:108B700017FF069B03ED0C0A049B0DA9C3ED010A28
:108B800083ED021A404615F0F7FE22AB079A03EB7D
:108B9000890303ED1A0A16AB981816F06FFA7A1CBF
:108BA00004D0B4EEC08AF1EE10FA03DD4FFA89F773
:108BB000B0EE408A22AB03EB870353ED1A7AF5EE51
:108BC000407AF1EE10FAF7EE007A48BFB0EE678A0D
:108BD00009F1010908F10C080BF10C0B7FE79BE888
:108BE000070088E80700A9E77B1C3FF443AF84F83F
:108BF0001C712046FFF7F8F960B12046FFF7E6F94F
:108C0000002840F0348122AA0C2303FB0723002212
:108C100043F8282C16AA07EB470895F8EB3402EB2B
:108C2000880895F8F0219A4240F23C812B4493F851
:108C30000C35002B00F0368195F8EC3495F8F121D5
:108C40009A4240F22F812B4493F80E35002B00F00E
:108C500029810C2322AA4146504603FB072713F023
:108C600025FF07ED0C0A47ED0B0A07ED0A1A4046EF
:108C700015F0B2FE002840F02181404615F0C6FEF6
:108C8000002840F01B815FED7E7A94ED387A28EE63
:108C9000278A5FED807AA7EE278A04F1B00084ED81
:108CA000388A16F0EBF9A3685FED857A93ED007AC8
:108CB000B4EEE77AF1EE10FAB0EE408A00F10281EC
:108CC0002046B0EE480AFFF747F9404615F0D8FDB8
:108CD000A3688DED130ACDED140A8DED151A93EDF1
:108CE000000A13A815F0CCFD204684ED1F0AC4ED40
:108CF000200A84ED211AFFF7E5F928B1B2EE000A47
:108D000004F17C0015F010FE039BB3B33046FCF772
:108D100079FD012831D996F8F402B02303FB0066EF
:108D200096ED3B7AF0EE087AB4EEE77AF1EE10FABF
:108D300023D595F8EC040C2303FB005595ED807AC0
:108D4000F1EE0C7AB4EEE77AF1EE10FA15DBD4ED21
:108D50001D7A1FEDAE7AF4EEC77AF1EE10FA0CDD53
:108D60001FEDB17AF4EEC77AF1EE10FA05D5B6EE42
:108D7000000A04F17C0015F0D7FD5FEDB67AB4EE81
:108D8000E78AF1EE10FA22D51FEDB90A404615F038
:108D900077FD10A88DED100A94ED450ACDED110A6E
:108DA0008DED121A15F06CFD13A904F1A0008DEDE4
:108DB000130ACDED140A8DED151A15F081FDD4EDD1
:108DC0002B7A94ED457A77EE877AC4ED2B7A94ED81
:108DD0002B7AF1EE047AB4EEE77AF1EE10FA4FF066
:108DE00000053BDB12F0EAFE5FEDD07A94ED2B1A22
:108DF00094ED280A21EE271A40F2C530F1EE410A1F
:108E00008DED031ACDED020A13F0F6FB9DED031A6A
:108E1000DDED020A84ED280A40F2C63094ED290AFD
:108E200013F0EAFB9DED031ADDED020A84ED290A39
:108E300040F2C73094ED2A0A13F0DEFB04F1A001E2
:108E400084ED2A0A04F1940015F03AFDC4F8A85004
:108E5000C4F8A450C4F8A050C4F8AC5018220021A3
:108E600004F1F0007EF008F9C4F814515CE5E36801
:108E7000F7EE000A93ED000A13F0E6FA00283FF43B
:108E8000C2AE94ED1C0AB0EEC00A7BF043FE0C2388
:108E900022AA03FB072353ED0A7A27EE800A03ED8B
:108EA0000A0AB7E60C2322AA03FB0727002347F888
:108EB000283C47F82C3C47F8303CD8E62046FFF7E2
:108EC00011FCD7E5C3ED007AFAE600BF2DE9F04DBD
:108ED0002DED048B9EB0044612F070FE00F59F63EA
:108EE000D3ED007A90ED7F8AF4EE487AF1EE10FA35
:108EF00048BFB0EE678ADFED5C7AB4EEE78AF1EE48
:108F000010FA0DDD1822002104F1F0007EF0B4F813
:108F10000023C4F814311EB0BDEC048BBDE8F08D05
:108F20002046FEF79DFD2046FEF756FFB0EE480AAC
:108F30002046FFF713FC2046FFF7D4FBFEF714F999
:108F400014AD00F5347204F1280114A813F0FEFDED
:108F50000FCD04F14C060FC60FCD0FC62B68336042
:108F600004F1740204F1780304F1700104F14C007F
:108F700013F09AFF94ED1E8AB0EE480A7BF074FC61
:108F800084ED6B0AB0EE480A7BF0C4FD204684ED08
:108F90006A0AFEF759FDFEF7E7F804F5C071FDF720
:108FA000E9FE56F0EDFBD4F8B031C31A632BB2D909
:108FB000C4F8B00134F018FE9FED2C9A054656F027
:108FC000E7FBD4ED1C7A67EE897A074617EE900A24
:108FD0000E46F7F791FAD4ED1D7A67EE897A82464C
:108FE00017EE900A8B46F7F787FA94ED1E0A20EEEB
:108FF000090A41EC180B13F095FAD4F8740110EE3D
:10900000108AF7F779FACDE91201D4F87001F7F771
:1090100073FACDE91001D4F86C01F7F76DFACDE9D8
:109020000E01D4F8E400F7F767FACDE90C01D4F8A3
:10903000E000F7F761FACDE90A014046F7F75CFA7C
:109040000B4B01930B4B0093CDE908018DED068B83
:10905000CDE904ABCDE90276074B084A084928461A
:1090600034F04EFB57E700BFCDCC4C3EE02E6542BE
:1090700094E0090899000A0860000A086A000A08D2
:10908000A8FE090808B52DED048BB0EE609AF0EE4D
:10909000408A00F011F9B0EE408A89EE280A7BF090
:1090A0006FFEDFED0B7A20EE270A7BF001FEDFED8D
:1090B000097A38EE278ADFED087A28EE278AF7EE5C
:1090C000007A37EEC00A28EE000ABDEC048B08BD1A
:1090D00041D3423E33938843A1D81943FFF7D2BF0F
:1090E00008B52DED048B9FED189AF0EEE07AF4EEC2
:1090F000C97AF1EE10FAF0EE408AB0EE608A1ED422
:1091000000F0DAF8DFED117A9FED117A70EE277A30
:109110009FED100AE8EEC77A9FED0F7A27EE800ADE
:10912000C8EE007A87EE270AB4EEC90AF1EE10FA0B
:1091300005DBBDEC048BBDE808407BF001BFBDEC56
:10914000048BB7EE000A08BD000000343393884357
:10915000F4FDD43B48A18F43CDCC9C3F427CD0ED65
:10916000257A242101FB020292ED0B0AD2ED090AB5
:1091700030EE270AFFF7B4BF38B52DED088BDFEDD1
:1091800021AA9FED21AA9FED21BA0546B0EE409A93
:10919000F0EE609AB0EE408A1524013CA4B25CB3B4
:1091A000F0EE490A2846B0EE480AFFF76BFFF0EEF2
:1091B000490A70EE698A284638EE2A0AFFF762FFEC
:1091C000B0EEE87A70EE697AB4EECA7AF1EE10FA8F
:1091D00077EEE87A10D468EEAA8A40F2631088EE3F
:1091E000A70AB0EE4B1A38EE400AF0EE4A0A13F026
:1091F00003FAB0EE408AD0E7B0EE480ABDEC088B27
:1092000038BD00BFCDCCCC3D0AD7233C00247449E7
:10921000002343608360C360036143618361C36172
:10922000002380F82030704790F82020531CDBB2D8
:10923000062B80F8203000EB820288BF002382EDED
:10924000010A88BF80F82030704700004FF0FF33DC
:1092500010B543610E4BC0F8A8300023044680F8D7
:10926000C830A830FFF7D4FF0A4BC4F8A83004F583
:10927000867055F03BFC084B08491C60204630F0D6
:109280007DFAD4F89030C4F89430204610BD00BF69
:10929000C0020A08D0020A082461002068030A08F4
:1092A00008B5A83035F0E8FCDFED027A20EE270A99
:1092B00008BD00BF00007A4490ED3C0ADFED057A5E
:1092C000B0EEC07AB4EEE77AF1EE10FA48BF90ED56
:1092D0003D0A70470000003473B5D0F8A43004464E
:1092E0000E4663B156F04CFAD4F8A430C01A42F2DC
:1092F0000F73984203D894ED280A02B070BD114B49
:109300001D687DB195F84E112846FCF7D7F848B195
:1093100095F84E1101AA2846FCF7C6F810B19DED4C
:10932000010AEAE7242101FB064494ED0A0ADFED75
:10933000067AB4EEE70AF1EE10FA58BFB0EE670A0B
:10934000DBE700BF1C61002000000C4208B561B1E2
:109350000378022B02D9064856F0E0F95A1C027035
:1093600000EB83004160012008BD0846FCE700BF18
:109370007C010A082DE9F84305460E469146002473
:1093800000F13C082B78A34211DD00234A46314608
:1093900001200EF0E3FF242363430746002158F821
:1093A00003000EF0EBFF874204D00134EAE700200F
:1093B000BDE8F8830120FBE7054B1B682BB1416931
:1093C0004A1C02D0184634F0D9BB0020704700BFB9
:1093D000CC63002002290BD8242303FB010191F860
:1093E000390030B191F83A0018B191F83B0070475C
:1093F000002070472DE9F047044656F0C1F9D4F833
:10940000F86042F21073861B9E4288BFC4F8F800D1
:1094100000274FF0240942F2107A237CFDB2AB42C0
:109420001CD929462046FFF7D5FF70B109FB054836
:1094300098ED0D0AD8ED097AD4ED250A30EE270A09
:109440002046FFF799FE88ED0C0A564504D909FB22
:109450000540303030F06AFB0137DEE7617C2046A2
:10946000FFF73AFF84ED3D0ABDE8F08770B504468A
:1094700086B056F085F9D4F89830C31AB3F57A7FE0
:1094800005464FD3344B94ED257A1B68DFED336AE4
:10949000DB6AD4ED247A93F89C60B0EEC76AB4EE30
:1094A000E66AF1EE10FA32D5B0EEE76AB4EEE66A9B
:1094B000F1EE10FA2BD502A801F026FA96BBFDF7C3
:1094C00053FE02A9FDF756FC60B3DDED037A9FED74
:1094D000247AF8EEE77A67EE877AC4ED257AC4F845
:1094E0009850FDF741FEFDF7EFF92046FFF782FFA8
:1094F0003DF0BAFD0546D4F89400F6F7FDFF194A91
:10950000CDE900010621284636F06AFF0AE037EE71
:10951000676AF7EE005AB0EEC66AB4EEE56AF1EE9D
:1095200010FA01DC06B070BDB0EEE76AB4EEE66A90
:10953000F1EE10FAF6D4002ECFD02046903080ED18
:10954000007A30F0F3FA3DF08FFD074A012106B0B2
:10955000BDE8704036F044BFF860002000000034E1
:109560000AD7233CBD010A0898010A08F0B52DED81
:10957000048B85B004464FF4537200F5867103A83E
:109580000FF078F8D4ED227AD4ED236A9FED796A52
:10959000637C37EEE67A2422B0EEC77AB4EEC67A60
:1095A000F1EE10FAC1BF9FED747A67EE877A9FEDF6
:1095B000737AE6EE877A02FB03430025C4ED237A33
:1095C00093F839602378E9B28B4206D904EB810322
:1095D0000135586858F060FAF4E7DFED698A9FEDCD
:1095E000698A9FED699A0027237CFDB2AB4264D95A
:1095F000242303FB054393F83920002A5BD0D3EDE5
:109600000C7AF4EEE87AF1EE10FA0BDBF4EE677AFE
:10961000F1EE10FA06D6F0EEE77AF4EE487AF1EEC3
:1096200010FA04DD242303FB05435A6A1A6324233A
:1096300003FB0543D3ED090AD3ED0D7A93F83820E7
:1096400070EEA70AA2B993ED0C0A2046FFF746FD7B
:10965000D4ED257A30EE670AB4EE400AF1EE10FA46
:1096600016D7242303FB0545002385F83A3022E072
:10967000012A09BFD3ED0C7A93ED0B0A77EEE00ACD
:10968000D4ED3B7A04BF80EE897A87EE270AE3E7C0
:10969000F0EEC07AF4EE487A2423F1EE10FA03FBE0
:1096A0000545E1DC012385F83A30D4ED237A37EE25
:1096B000800A85ED0B0A013796E7627C2046114649
:1096C000FFF788FE48B1242101FB024292ED0B0A0C
:1096D000D16904F1A80035F0AFFA94F99C10277C09
:1096E000002907DBB94205DACAB211462046FFF766
:1096F00071FE68B900226274D5B2AF4209D9294619
:109700002046FFF767FE01320028F5D0657400E0BF
:1097100062742046FFF7AAFE2046FFF74DFE10B107
:10972000204659F0C1F9637C242505FB034393F8D7
:109730003930B34216D034F057FA4FF6FF7134F097
:109740001DFA78B1607C05FB004494F83930002B99
:1097500014BF00220422019234F046FA019A122129
:1097600034F09EF903A80EF0A7FF05B0BDEC048B02
:10977000F0BD00BF0AD7233C0AD7A33C48E17A3F9B
:1097800000000034FFFF7F7F002019462DE9F04FD5
:109790000446007C0F4687B004F13A030022012101
:1097A000D5B2A84203F1240305D903F8231C03F81A
:1097B000241C0132F4E7744B1E68F06A03685B688E
:1097C000984740B13DF050FC704A062107B0BDE813
:1097D000F04F36F005BE23781BB1237C0BB16368D4
:1097E0001BB93DF041FC6A4AEFE73DF03DFC694A98
:1097F000062136F0F5FD002303A904F18800039348
:1098000030F058FD0A2555F0BBFF80462046FFF793
:10981000ADFE55F0B5FFA0EB0800B0F5FA7F02D918
:109820005D4801F055F8B06A03680A215B68984703
:10983000617C2046FFF7CEFD0028E7D0B06A0368C0
:1098400064215B68013D984715F0FF05DBD1534B60
:1098500005951B888DF80650CDE90355ADF8043009
:10986000052555F08DFF80462046FFF77FFE55F019
:1098700087FFA0EB0800B0F5FA7FD1D8617C2046C5
:10988000FFF7A8FD0028EFD094F810B00DF10C08F8
:10989000A14601AA4FF0000A5FFA8AF18B4516D95A
:1098A0002046FFF797FD50B1D8ED007A99ED097A7F
:1098B000137877EE877A0133C8ED007A13700AF1D6
:1098C000010A08F1040809F124090132E4E7B06A49
:1098D000036864215B68013D984715F0FF05C0D11E
:1098E000A9464FF02408237C5FFA89F6B34226D9B3
:1098F00006AB334413F8143C33B908FB064686F82C
:109900003B3009F10109EEE7002FFAD007EE903A5B
:1099100006AA02EB8602F8EEE77A12ED030AD4ED0E
:10992000250A204680EE270AFFF726FC08FB0640A2
:1099300002A930308DED020A30F0BCFCE1E7617C19
:10994000DFF860902046FFF7C7FC002684ED3D0A53
:109950004FF02408237CF7B2BB420FD908FB074322
:1099600093F83B3043B13DF07FFB7B1C4A46062118
:1099700036F036FD0135EDB20136EBE70DB908489A
:109980004FE707B0BDE8F08FF8600020D8010A0863
:1099900003020A0830020A0846020A088CB20908C3
:1099A00082020A0860020A0808B5037C022B02D969
:1099B000034855F0B3FE5A1C0274184608BD00BF98
:1099C000A4020A0838B5057C02460024E1B28D42A3
:1099D00006D91046FFF7FEFC01340028F6D138BD49
:1099E000281E18BF0120FAE770B50D46097807292F
:1099F000044606D8027E437E22B901228A401343E0
:109A0000437670BD002BFCD000262278F3B29A4238
:109A1000F7D904EB8303294658680368DB68984745
:109A20000136F2E7014B1868704700BF246100203F
:109A300010B50446006810B103685B68984720467B
:109A400010BD000013B500220B680A6001A9019344
:109A500058F072FB044601A8FFF7EAFF204602B067
:109A600010BD000013B500220B680A60022201A994
:109A7000019359F04DFD044601A8FFF7D9FF204698
:109A800002B010BD13B500220B680A60012201A9C3
:109A9000019359F03DFD044601A8FFF7C9FF204698
:109AA00002B010BD13B500220B680A6001A9019332
:109AB00059F02EFD044601A8FFF7BAFF204602B078
:109AC00010BD000010B50446006810B103685B6863
:109AD0009847204610BD00002DE9F04F8FB0D0F818
:109AE00000310893344B354D1B6805930446586884
:109AF00003689B68984794F99D300690002BA2BF9D
:109B0000012606FA03F3069305F1D80A2B68089A92
:109B10001A420BD000274FF0010BB946069A0BFAF8
:109B200007F3134206D10137202FF7D10C355545E5
:109B3000ECD12DE0F9B26B682A7A0991204607939F
:109B4000FFF718FC0999804628B3CDE90A990B9BC9
:109B50000D930DA9079BCDE90B9920469847014627
:109B60002046FFF7F3FB0DA8FFF762FF0CA8FFF7F5
:109B70005FFF0BA8FFF7A6FFB8F1000F02D00AA8FD
:109B8000FFF7A0FF2378032B02D0237C032BCAD13D
:109B90000FB0BDE8F08F059B586804220368CDE93B
:109BA0000182074A00921B680A461E4601462B7A2C
:109BB0000BA8B047CBE700BFF860002058040A08A4
:109BC000801A060070B5D0ED247A9FED607AF0EE31
:109BD000E77AF4EEC77A0123F1EE10FA8AB0044670
:109BE000037609D49030002309A90590099330F039
:109BF00061FB05982FF09AFF0026E6632666C4F8FD
:109C00008460762231462046FFF7B4FB05460028E3
:109C100036D0CDE90666079A0992002309A92046A5
:109C2000CDE9073357F0CAFA01462046FFF78EFB0D
:109C300009A8FFF7FDFE08A8FFF7FAFE07A8FFF73F
:109C400041FF15B106A8FFF73DFF2378032B50D045
:109C5000237C032B4DD094F99D1000291FDA204658
:109C6000FFF73AFFD4F80031DA0454D40025637EBC
:109C7000EB40DB07EAB254D40135082DF7D138E0C8
:109C8000334B1B68596804220B68CDE90102314A45
:109C900000921E680246762307A8B047BBE77722EA
:109CA000C9B22046FFF766FB054620B30023CDE985
:109CB0000633079B0993002209A92046CDE9072214
:109CC00059F026FC01462046FFF740FB09A8FFF7A4
:109CD000AFFE08A8FFF7ACFE07A8FFF7F3FE15B12B
:109CE00006A8FFF7EFFE2378032B02D0237C032B7B
:109CF000B5D10AB070BD164B1B68596804220B68B9
:109D0000CDE90102134A00921E6894F89D20772342
:109D100007A8B047CDE7637E002BA7D10123637668
:109D2000A4E73820059201F0B7F8064618B1059A65
:109D3000214659F08BFC31462046FFF707FB23787C
:109D4000032BD6D0237C032B96D1D2E7000000341E
:109D5000F8600020801A060090F86035934207D919
:109D600002F5A77250F8220010B103689B6A1847E9
:109D7000002070472DE9F34105466E4686E80C0049
:109D8000134B45F8043B04460F4600F5C8782846B7
:109D90002C3500F0C5FCA845F9D196E8030004F283
:109DA0006453C4F85C7583E80300089BC4F86C3501
:109DB000084920462FF0E2FC074B1A6812B1074809
:109DC00055F0ACFC20461C6002B0BDE8F08100BF3D
:109DD00060070A0828060A08286100206C050A089E
:109DE0002DE9F041A2B00C4607A92EF031FE002863
:109DF00055D000210D220CA80591ADF818100B913B
:109E00007DF03AF92B4B611C1F68C9B20BAD0129DB
:109E1000F86A0A9546D1284B062205A90EF008FEDD
:109E2000264B019305AB0093002411222946244BB5
:109E3000F86A8DF819400EF0FBFD04AA0DF10F0130
:109E400028468DF83C40049430F00CF938B31D4995
:109E5000DFF86C80482210A87DF0C4F8062610AC0C
:109E60002268531E049AC2F3513202EB8312237903
:109E70008DF82430A368019305AB00930892434604
:109E800011222946F86A0EF0D3FD0021B7EE000A30
:109E900007A82EF0A9FF013E04F10C04E0D122B086
:109EA000BDE8F0810091084B062205A90EF0C0FD27
:109EB000B6E700BFF8600020A1F209089D050A0876
:109EC00097050A0890B2090890050A082DE9F74F8E
:109ED00090F860650446002E51D17F2380F87035DC
:109EE00000F5C87500F5A768071D5FFA86FA182205
:109EF000FF2128467DF0C0F885F85FA097F92690ED
:109F0000B9F10A0F5CD03DDCB9F1040F0FDCB9F1F7
:109F1000020F0FDD442000F0BFFF834620B13B4617
:109F20002A46214659F0F8FEC8F800B002E0B9F11F
:109F3000090F39D0D8F8000050B1696EC5F86090AB
:109F400031B12C4B43F826102FF026FE2FF01CFECB
:109F500058F8040B0AF101095FFA89F940B1036866
:109F60009B68984784F8609551462046FFF738FF74
:109F70000136092E05F1680507F12C07B5D103B0AC
:109F8000BDE8F08FB9F1150F28D0B9F1190FD1D173
:109F9000482000F081FF83460028C5D03B462A4672
:109FA00021465BF08DF8BFE7382000F075FF83464F
:109FB0000028B9D03B462A4621465AF013FBB3E7A6
:109FC000302000F069FF83460028ADD0CDF800A016
:109FD0003B462A4621465AF0F5FFA5E7782000F0D7
:109FE0005BFF834600289FD03B462A4621465AF015
:109FF00061FB99E72C61002090F860358B4283BFAC
:10A00000682303FB010090F8DD0100207047000089
:10A0100090F860358B4283BF682303FB010090ED0D
:10A020006A0A9FED010A70470000000090F8603551
:10A030008B4206D901F5A77150F8210008B15AF0FA
:10A040000BB89FED010A70470000000010B490F8B3
:10A0500060458C420A4614D901F5A77450F8244093
:10A060007CB1E468246A640603D55DF8044BFFF70D
:10A07000DDBF682101FB020393ED6A0A5DF8044B22
:10A0800070479FED010AF9E70000000090F8603585
:10A090008B420BD901F5A77150F8210038B1C36884
:10A0A0001B6A1A4214BF012000207047002070472D
:10A0B00070B590F86035934204460E46154601D8B7
:10A0C000002070BD02F5A77350F823000028F7D0D8
:10A0D00003689B6998470028F2D0682202FB054478
:10A0E000D4F8AC313360ECE770B590F8603593424A
:10A0F00004460E46154601D8002070BD02F5A77330
:10A1000050F823000028F7D003689B69984700287F
:10A11000F2D0682202FB0544D4ED6C7AF4EE677A43
:10A12000F1EE10FAE8D6C6ED007AE6E770B590F8E1
:10A130006035934204460E46154601D8002070BD96
:10A1400002F5A77350F823000028F7D003685B6975
:10A1500098470028F2D0682202FB0544D4F8B431B5
:10A160003360ECE790F8603593420ED902F5A7739F
:10A1700050F823305BB1682303FB020292F8EC0134
:10A1800030B1D2F8E8310B607047002070471846B4
:10A190007047000008299DBF2C2303FB0100406885
:10A1A000002070472DE9F04F4B4B2DED028B1B68C3
:10A1B000DB6A93F89C3089B00446002B00F086805F
:10A1C000DFF82CB19FED458A4FF0000994F8603517
:10A1D0005FFA89F5AB4279D905F5A77354F82300E6
:10A1E00000285DD003685B6B9847682303FB054339
:10A1F000074693F8DC31834252D2032861D8DFE866
:10A2000000F04F025259364E4FF000083CF02CFF40
:10A2100094F86025AA4284BF682202FB05424FF0F1
:10A22000680105F1010301FB05458CBFD2F8A821A7
:10A2300018EE102A8246D5F8B001CDE90632F6F7BD
:10A240005BF9079ACDE904011046F6F755F9069B2C
:10A250000096CDE902015A460421504636F0C0F876
:10A260000123204A84F8713585F8DC71D372D4F863
:10A270006C354BB3002255B25957481C03D04145A9
:10A2800002F10102F7D194F97035AB4208DBD4F842
:10A290006835D4F8640542463146984784F87055CD
:10A2A00009F1010992E72C2303FB05430E4E93F9B4
:10A2B0002D80ABE72C2303FB05430C4E93F92E8036
:10A2C000A4E70026B046A1E71D46DCE709B0BDECD7
:10A2D000028BBDE8F08F00BFF86000200000000096
:10A2E000B1050A0885610020D24E0B08A8050A08AE
:10A2F000C0050A0890F860358B4207D901F5A771AF
:10A3000050F8210010B10368DB691847002070473E
:10A3100008299CBF682303FB010000F5C870704743
:10A3200090F86035934207D902F5A77250F82200E1
:10A3300010B103685B6A18470020704790F86035D9
:10A340008B420DD901F5A77350F8233043B1682330
:10A3500003FB0101012081ED730A81F8C8017047F8
:10A3600000207047F8B5002402460E4625462C27EB
:10A3700092F86035E1B28B4210D901F5A77352F81B
:10A3800023304BB107FB01239B689E4204D110464A
:10A39000FFF7D4FF2843C5B20134E9E72846F8BDEA
:10A3A0002DE9F04F002493B005460E46174621468E
:10A3B0002F2206A8059405F5A7697CF05DFE05F13E
:10A3C0002A0A4FF02C0B05F5F8730BFB04F259F831
:10A3D000040B1AF90210E5B230B951B90134092C55
:10A3E000F3D14FF0010813E0682262439A5891427A
:10A3F00012D01548154B006801930135EDB2009558
:10A40000134BC06A324639460EF012FB4FF000087B
:10A41000404613B0BDE8F08F05A93322039359F0ED
:10A42000FDFE039B804605A90028D7D1064801916F
:10A430000135EDB200680095054BC06A32463946D9
:10A440000EF0F6FAE4E700BFF8600020F6050A080F
:10A45000E8050A082DE9F04FDFF88090DFF880A0CA
:10A46000DFF880B08DB00646002796F86035FCB264
:10A47000A3422ED9682505FB046595F8E43133B372
:10A4800095F8E51119BB4FF001082022444404A8B7
:10A4900089F819807CF0F0FD07EE904A4AF21043EB
:10A4A000F8EEE77A03AA4C21ADF828305046242371
:10A4B000CDED037A37F0AAFE3CF0D6FD9BF80030D4
:10A4C000054A0094042135F08BFF85F8E5810137BA
:10A4D000CBE70DB0BDE8F08F00060A0885610020CB
:10A4E00059640020CD2200202DE9F04F2F4B1E682B
:10A4F00085B0044646B1D0F85C15304633F03EFBDB
:10A5000010B1304632F03CFA55F03AF94FF00008FD
:10A5100001904FF02C0A4FF0680B94F860355FFA09
:10A5200088F5AB4239D904EB8507D7F8380588B3ED
:10A530000AFB05430BFB054993F92A20D9F8F011D2
:10A540008A4227D132B30268D2689047D7F83805DB
:10A550000268126B904799F8DD2112B1019BC9F88E
:10A56000E031BEB1D4F85C15304633F007FB88B15A
:10A5700055F00EF9CDE9021002460B46D7F8380522
:10A5800029465AF091FBDDE90232D7F83805294611
:10A590005AF008FC08F10108BFE72046FFF702FE69
:10A5A000204605B0BDE8F04FFFF754BFCC63002054
:10A5B0002DE9F0474FF000082DED028B0446894647
:10A5C000B0EE408A474601264FF0680A94F860359D
:10A5D0005FFA88F5AB421AD929FA05F3DB070AD5E9
:10A5E00005F5A77354F8230078B10368B0EE480A64
:10A5F0009B6B984706400AFB054508F1010895F852
:10A60000DC319F4238BF1F46E0E70646F3E727B933
:10A610007F23A4F87035034BDF72BDEC028B30460C
:10A62000BDE8F0878561002090F860358B4207D93E
:10A6300001F5A77150F8210010B10368DB6B1847D2
:10A64000002070470B46114690F860259A4207D9C2
:10A6500003F5A77350F8230010B103681B6C18476B
:10A660007047000070B504460E46002594F860352A
:10A67000E9B28B4205D932462046FFF7E3FF0135A8
:10A68000F4E770BD2DE9F84390F8605502460024C8
:10A6900000F12A062C2700F5F8784FF06809E1B29E
:10A6A0008D420FD907FB04F309FB04F0F35658F869
:10A6B0000000834209D11BB11046FFF79DFC10B189
:10A6C0000134ECE70120BDE8F8830020FBE700003F
:10A6D00010B590F860258A42044617D9682202FB1B
:10A6E000010393F8DC31022B03D004D9032B18BFEC
:10A6F0000023184610BDFFF797FF48B92046FFF723
:10A70000C1FF00280CBF06230123F2E70023F0E776
:10A710000623EEE7014B1868704700BF2861002050
:10A7200010B5034904462FF029F8204610BD00BF9C
:10A73000E0070A0810B50446203046F009FF044B34
:10A7400004491C6020462FF019F8204610BD00BFB8
:10A750005061002064090A08F7B5B7EE000A00222C
:10A76000022104462EF074FC20465AF011FD46F0FA
:10A7700069FF144B1D680646E86A03685B6A9847E0
:10A780000B46022102460091304646F0F7FEB4F92E
:10A790004A60002E14DDEF6A3B6838465B68B4B24D
:10A7A000984728B197F84D3013B1C92EA8BFC824D7
:10A7B000A86A03685B68214603B0BDE8F04018470B
:10A7C00003B0F0BDF860002010B504465AF096FCC6
:10A7D0002046BDE810405AF0C1BC00002DE9804879
:10A7E000284BDFF8A490DFF8A4A0DFF8A4B014464B
:10A7F000012293B005460E461A704FF0000854F03F
:10A80000BFFFD9F800300393A0EB080241F2873371
:10A810009A4207461FD9CDE9005603985346342281
:10A8200005A9C06A0EF004F9214605A8049454F065
:10A83000DBF9CDE9005603985B46342205A9C06ACE
:10A840000EF0F6F804943CF00FFC049B05AA0221DC
:10A8500035F0ACFDB8463CF007FC3BF0A1FE3CF007
:10A8600003FC3DF065FD0A2105A80DF0E9FE039B00
:10A87000986A036805215B68984705A80DF0ECFE0F
:10A88000BDE700BF54610020F8600020E0080A081E
:10A89000356A0B080FB400B595B016AA002152F81E
:10A8A000043B039205A83C22019304917CF0E4FB55
:10A8B000054A019B402104A854F03EF9039A03483D
:10A8C00004A9FFF78BFF00BFE8080A08FE080A0882
:10A8D0000FB407B504AA034852F8041B0192FFF70E
:10A8E0007DFF00BF10090A0808B5044910227CF05A
:10A8F00069FBB0FA80F0400908BD00BF5861002034
:10A90000102200217CF0B8BB10B50446FFF7F8FF19
:10A91000204610BD0378416023F00D03022A037026
:10A9200008D0032A0AD0012A03D1DBB243F0010385
:10A9300003707047037843F00803F9E7037823F0C6
:10A94000050343F00503F3E773B504460E461546C9
:10A950000193FFF7D5FF2046C4E90265069A0199E5
:10A96000FFF7D8FF02B070BD0078420704D4030798
:10A9700004D400F0010070470320704702207047A4
:10A98000F0B585B005461646FFF7EEFF88420F4644
:10A9900005D16B6833600124204605B0F0BD032863
:10A9A00001D10024F8E70329FBD001280BD00228AD
:10A9B00016D018BB6D68012F22D0022F2ED0002F89
:10A9C000EFD13560E7E7FCF7CFFB90F87C32DB078F
:10A9D000E7D56D68FCF7C8FBD0F870321D44EAE794
:10A9E0006846FFF78DFFFCF7BFFB6946FCF7C2F92D
:10A9F00004460028D0D06D68019BEFE70025DAE718
:10AA0000FCF7B2FB90F87C4214F00104C9D0FCF7CB
:10AA1000ABFBD0F87032ED1A3560BDE76846FFF742
:10AA20006FFFFCF7A1FB6946FCF7A4F90446002878
:10AA3000B2D0019BEFE7000073B501AA05460E46B0
:10AA4000FFF79EFF044620B1019932462846FFF7E2
:10AA500061FF204602B070BD13B5144601AAFFF78E
:10AA60008FFF48B1DDED017A9FED047AF8EEE77AC9
:10AA700067EE877AC4ED007A02B010BD0AD7233C96
:10AA800007EE900A9FED090AF8EEE77A08B527EE7F
:10AA9000800A79F0E9FEDFED067AB4EEE70AF1EE1E
:10AAA00010FAD8BFB0EE670A08BD00BF50E0EF3023
:10AAB0000AD7233C10B50446806811F05FFF20B12F
:10AAC000E068BDE8104011F06DBF10BD73B585683A
:10AAD00004460E461DBBC36823B98B688360CB68F0
:10AAE000C3600125636873B92378DB070BD5204663
:10AAF000FFF73AFF01AA01463046FFF741FF10B1C8
:10AB0000019B636005462046FFF7D4FF20B9B36878
:10AB1000A360F368E3600125284602B070BD0025FC
:10AB2000E0E700000D4B83424FF000038B4106DA53
:10AB300000F1255000F5311000F5E0507047084B4A
:10AB400098424FF0FF3371EB0303BEBF00F1564054
:10AB500000F5130000F52440704700BF00D2496B98
:10AB6000002EB69490EA010F01D4401A7047C31723
:10AB7000401A63EBE1710D4B83424FF000038B41B0
:10AB800006DA00F1255000F5311000F5E05070476D
:10AB9000074B98424FF0FF3371EB0303BEBF00F148
:10ABA000564000F5130000F52440704700D2496B71
:10ABB000002EB69470B52DED028B84B00446684625
:10ABC0000D46FFF79DFEFCF7CFFA6946FCF7D2F879
:10ABD000064608B3A368029ADFED128A03999B1A0E
:10ABE00007EE903AF8EEE77A67EEA87AC5ED007ABC
:10ABF000E068FFF7B7FF08EE100AA068024402EB16
:10AC0000D272B8EEC88A5010FFF73AFF28EE288AB1
:10AC100028EE000A85ED010A304604B0BDEC028B37
:10AC200070BD00BFF67C8E3F37B500230C4601AAED
:10AC3000022105460193FFF7A3FE10B9002003B0DF
:10AC400030BD21462846FFF7B5FF0028F6D0DDEDE0
:10AC5000017AF8EEE77AC4ED027AF0E738B52DED27
:10AC6000028B0C460246C168E068FFF77BFF9568DF
:10AC7000A46808EE100A601900EBD0704010641B45
:10AC8000FFF7FEFE07EE904AF8EEE77AF8EEC80A04
:10AC900087EE807ABDEEC70A10EE103A5B4200EEF6
:10ACA000103AB8EEC00A7AF001F8DFED087A30EE1B
:10ACB000270ABDEC028BB5EEC00AF1EE10FA44BFD4
:10ACC000DFED037A30EE270A38BD00BFDB0FC93F46
:10ACD000DB0FC94030B52DED028B0B4685B08C687B
:10ACE000D0E90251D868FFF73DFF08EE100A60195D
:10ACF00000EBD0704010FFF7C3FE641B07EE904AD4
:10AD0000F0EE400AB8EEC88A9FED060AF8EEE77A40
:10AD100028EE008A27EE800A68EE200A05B0BDEC16
:10AD2000028B30BD8262363C82B002B0FFF7D2BFE8
:10AD3000F0B52DED028B0D4689B08C680646D0E942
:10AD40000271E868FFF70EFF08EE100AE01900EB49
:10AD5000D0704010FFF794FE73686A689FED0E1A7A
:10AD60009B1A07EE903AE41BB8EEE77AF0EE400A41
:10AD700007EE904A9FED090AB8EEC88AF8EEE77A26
:10AD800028EE008A27EE011A27EE800A68EE200AD4
:10AD900009B0BDEC028BF0BD0AD7233C8262363C81
:10ADA00010B52DED028B84688A680B46111B08EEE6
:10ADB000901AC168D868FFF7D5FE224402EBD27220
:10ADC00008EE100A5010FFF75BFEB8EEC88AF8EEE6
:10ADD000E88A28EE000A20EE000AA8EEA80A7AF017
:10ADE000AFF8BDEC028BDFED027A20EE270A10BD32
:10ADF0008262363C094B984206DDC0F1D64000F530
:10AE0000930000F5A4407047054B9842BEBFC0F1C7
:10AE1000144000F5360000F53850704700E9A435BD
:10AE200000175BCAF8B52DED028BDFED148A0768B9
:10AE300020EE280A0646FDEEC07A0D4617EE904A2F
:10AE400004EBD47007EB6000B0EE608AFFF718FEE9
:10AE500028EE288A3819C8EE007AFFF7CBFF306059
:10AE600017EE900AF6F772F82B68C01841EBE37101
:10AE7000FFF758FEBDEC028B2860F8BD02AAB34272
:10AE800000F10C010830FFF7CDBF00000148FFF7CB
:10AE900037BD00BF586100200121884238BF0846F5
:10AEA00077F006BEFFF7F8BF08B177F005BE704730
:10AEB000FFF7FABF00214FF0FF3310B50022036304
:10AEC000044601600171C0F80510417280F8251038
:10AED00000F13C0300F50B70D9709A60DA601A61DA
:10AEE0005A619A61DA611A625A629A62DA631A6482
:10AEF0005A649A64DA641A655A659A65DA65DA669C
:10AF00001A675A677C339842E6D1214604F51670D9
:10AF100007F016FC044B1A6822B904491C6020464D
:10AF20002EF02CFC204610BD68610020B80B0A08EA
:10AF300073B5D0F83C3201919942044613D0D0F851
:10AF40004032994218D0D0F844328B4216D10220B8
:10AF50000AE0D4F8343253B3D4F838324BB34FF05C
:10AF6000030002B070BD002094F822308342F8D86C
:10AF7000431C84F82230F4E70120F5E7D0F8306272
:10AF8000002EE6D194F841233546B6009AB1A319B4
:10AF9000C3F83012A319019AC3F83C2294F8223066
:10AFA000AB429CBF6B1C84F822302846D9E70126AF
:10AFB000E8E70226E6E704F50C7001A930442FF01B
:10AFC00087FAE7E738B504460D462FF0F7F9291D53
:10AFD000201D2FF0F3F905F1080104F108002FF00E
:10AFE000C7FA05F1140104F114002FF0C1FA05F1BC
:10AFF000200104F120002FF0BBFA05F12C0104F12F
:10B000002C002FF06FF905F1300104F130002FF022
:10B0100077FA05F13C0104F13C002FF0A9FAAB6B83
:10B02000A3636B6B636338BD2DE9F043A1B00023CC
:10B03000002500F13C0706468DF807500393049362
:10B04000059306930793089309930A930B93109320
:10B0500011931293139314931593169317931893B4
:10B060001C931D931E9300F50F78B94658F8043BC6
:10B07000F3B1F26E934223D0D6F8E820934221D068
:10B08000D6F86421934213D10221EBB299420FD03A
:10B09000C1EB411109EB8104214601A8FFF792FFA2
:10B0A00039462046FFF78EFF01A93846FFF78AFF91
:10B0B0000135032D07F17C07D8D121B0BDE8F0831D
:10B0C0000021E2E70121E0E72DE9F04706460F46BF
:10B0D0001546804604464FF0000A39463046FFF7D1
:10B0E00027FF626FBA425FFA8AF90ED1C3B2022B10
:10B0F0000BD87C2202FB0A66012086F83E0086F807
:10B100003F3085F80090BDE8F0870AF1010ABAF1F6
:10B11000030F04F17C04E0D1002439463046FFF7E8
:10B1200007FFD8F86C205FFA84F912B9C3B2022B7A
:10B1300022D90134032C08F17C08EED100244FF011
:10B140007C0906F13E0A39463046FFF7F1FE034618
:10B1500009FB04F05FFA84F81AF8002012B9DBB298
:10B16000022B12D90134032CEDD196F823000428C8
:10B1700014D9194854F0D2FA7C2000FB0464012051
:10B1800084F83E0084F83F30BBE70644012086F88F
:10B190003E0086F83F3085F80080B4E706F543713D
:10B1A000002251F8043BBB42D4B208D1A04202D8DD
:10B1B000631C86F8233003342C700020A3E73BB9CE
:10B1C000421C06EB800086F82320C0F80C73F2E7DF
:10B1D0000132052AE5D1F0E7F4090A08C9B200EB0B
:10B1E0008101D1F83C3253B1026F93420AD0D0F8BA
:10B1F000EC20934208D0D0F86821934206D04FF05B
:10B2000003007047002070470120704702207047FC
:10B2100059B190F82030032B07D05A1C80F8202019
:10B2200000EB83004161012070470020704700005F
:10B230002DE9F8430F469146044600F5BA7894F894
:10B240003E5035B97C344445F9D100252846BDE847
:10B25000F88300234A46394601200DF07FF800218B
:10B260000646E06E0DF08AF88642EBD1EEE700006C
:10B270002DE9F043DFF87C8085B0044600F50F76B9
:10B2800000257C27B14656F80C3CD9F800209342A3
:10B29000E9B206F1040619D1C3B12046FFF79EFFBB
:10B2A000C0B207FB004090F83E307BB903A9A9F17A
:10B2B0000C0003932FF00CF93BF0D6FE56F8043C3B
:10B2C000009342462B46012135F08AF80135032DC3
:10B2D000D8D104F16C0504F5F074296821B9AB6884
:10B2E00013B128462DF0D0FB7C35A542F5D105B031
:10B2F000BDE8F083100A0A0838B504461546FFF782
:10B300006DFFC0B2022808D87C2303FB0040294609
:10B310005030BDE838402FF01BB938BD38B5044671
:10B320001546FFF75BFFC0B2022808D87C2303FB59
:10B33000004029465C30BDE838402FF009B938BDDF
:10B3400037B50D4604468DED010AFFF747FF022D84
:10B3500007D8C0B27C2303FB004001A968302EF05F
:10B36000A9FF03B030BD000038B50546FFF736FF32
:10B37000C4B2022C13D8C4EB4414A4003C3504F12D
:10B380000800284400212DF07FFB04F1340104F172
:10B39000300029442844BDE838402FF099B838BD22
:10B3A00070B505460E461446FFF718FFC3B2022BD0
:10B3B0000DD87C2000FB035394E80700443383E856
:10B3C000070031462846BDE87040FFF7CDBF70BD8D
:10B3D00037B504461546FFF701FFC0B2022809D869
:10B3E0007C2303FB00400DF1070140308DF807502E
:10B3F0002EF0E4FF03B030BD1FB590F92C300446A9
:10B4000023B390F921300BB36846FFF77DFAFBF7C1
:10B41000ABFE6946FBF75EFCC0B1DDED037A9FED44
:10B420000C0AF8EEE70ADDED027AF8EEE77A01237E
:10B43000C0EE800A84F83D3387EE800A07F0C2FB35
:10B44000DFED047A20EE270A84ED0A0A04B010BD6D
:10B450008096184B35FA8E3C024690F9210058B17F
:10B4600092F8400340B1114491F92C0220B192F9B5
:10B470002400033818BF01207047000038B590F849
:10B48000223005465BB100242346E1B22846FFF78F
:10B49000E3FF08B10133DBB20134032CF5D11846C8
:10B4A00038BD000090ED0A0A7047000038B50C4620
:10B4B000D1ED066A11460546FFF790FEC3B27C2027
:10B4C00000FB0353D4ED087AD3ED260A94ED076A06
:10B4D000D3ED255A93ED245A26EE600A67EEA00AB2
:10B4E000A5EEA70AF0EE607AE5EE867AB7EE007A6E
:10B4F000A6EEE67A67EEE60AB1EE400AE5EE070A46
:10B5000079F0D4FB9FED071ADFED070A40F61C0027
:10B5100011F072F8D5ED0A7ABDE8384030EE270A0E
:10B5200011F056B8DB0F4940DB0F49C02DE9F0415F
:10B5300090F822308B4204460D4602D20020BDE82E
:10B54000F081FFF74BFEC0B204F13C06C0EB4010A7
:10B5500006EB8000083013F091FDDFED157AB0EEB8
:10B56000C00AB4EEE70AF1EE10FAE7D42946204605
:10B57000FFF734FEC5B27C2000FB05473B6F002B74
:10B58000DCD0032DDAD000FB05603030D7F86C80BA
:10B590002EF0CAF9D7E91B32934201D1984505D064
:10B5A0007C2000FB0544C4F86C80C7E70120C6E797
:10B5B000000000342DE9F74F04460E46174600F50B
:10B5C0000F7A4FF0000B5AF8049B5FFA8BF8B9F131
:10B5D000000F26D041462046FFF73EFF08B3414604
:10B5E0002046FFF7FBFD7C23C0B203FB004090F830
:10B5F0003E505DB908F101031B4ADBB239463046C3
:10B6000053F09AFA284603B0BDE8F08F5AF8102C90
:10B61000914506D0154A3946304653F08DFA00253B
:10B62000F0E70BF1010BBBF1030FCCD14FF0000899
:10B6300094F822305FFA88F18B420DD920460191AF
:10B64000FFF774FF054620B901992046FFF704FF74
:10B6500020B908F10108EBE70125D3E7044A394690
:10B66000304653F069FACDE7380A0A084D0A0A084D
:10B67000720A0A082DE9F0412DED048B90F842136F
:10B680009FED348ADFED348A9FED349A82B006460E
:10B69000FFF7A4FD06F13C07C5B27C2000FB057551
:10B6A00054354FF0000896F822205FFA88F39A424A
:10B6B0004ED919463046FFF7CFFE10B908F1010800
:10B6C000F1E719463046FFF789FDC4B27C2000FB44
:10B6D0000474D4ED157AF0EEE77AF4EEC87AF1EE60
:10B6E00010FA04F154040ED5D4ED017AF0EEE77AA5
:10B6F000F4EEC87AF1EE10FA05D5002002B0BDECE8
:10B70000048BBDE8F0812946204613F0CFFCB4EE4F
:10B71000E80AF1EE10FAF0DC2946204612F0B2FFFA
:10B72000B4EEC90AF1EE10FAE7DC2146284612F021
:10B73000D9FE68468DED000ACDED010A12F08EFFAC
:10B74000DFED077AB4EEE70AF1EE10FAB6DDD4E7E2
:10B750000120D3E700000034DB0FC93F920A863F87
:10B7600000004843022910B5044608D8FFF736FD0B
:10B770007C23C0B203FB004494F83D0010BD0020C0
:10B78000FCE7000013B590F8421301910446FFF75F
:10B79000E9FF30B10199204602B0BDE81040FFF743
:10B7A0005BBE02B010BD0000F7B590F92150044611
:10B7B000002D73D090F84053002D6FD090F84213B5
:10B7C000FFF7D0FF94F83D33064613B92046FFF744
:10B7D00013FE002594F82020EBB29A4207D904EB1F
:10B7E00083030135586903689B689847F2E753F073
:10B7F000C7FF0027224604F5BA7140F2F315D2F8CC
:10B800009C30C31AAB428CBF0023012382F83D3029
:10B810007C32914247EA0307F1D194F92430032B9B
:10B8200007D194F83C33002B3BD0D4F838030028E0
:10B8300049D167B1236B013309D032F0D5F9216BBF
:10B8400032F09CF918B132F0CFF931F0ADF994F93A
:10B850002C32002B3AD194F92D32CBBB94F92E32F5
:10B8600013B1022384F8423394F842132046FFF7C1
:10B8700079FF8642054611D032F0B6F94FF6FF71D6
:10B8800032F07CF950B1002D14BF00220422019245
:10B8900032F0AAF9019A032132F002F9284603B0E6
:10B8A000F0BD012384F83C330420FFF7F5FA054688
:10B8B00010B1214606F0DAFF94F92430C4F8385369
:10B8C000032BB2D0B5E706F0DFFFB2E70023C9E7EC
:10B8D0000123C7E738B590F921300446D3B190F879
:10B8E0004053BDB1FFF77AFCC0B2022812D87C23C6
:10B8F00003FB0044D4ED1A7A9FED087AF4EEC77A80
:10B90000F1EE10FA06D4B7EE087AF4EEC77AF1EE4B
:10B9100010FA00DD0025284638BD00BFABAA2A3F3B
:10B9200070B5D0F8085315F4003504460E460DD115
:10B9300090F840335BB90A78072A07D8012303FA45
:10B9400002F290F83F33134380F83F3370BD94F810
:10B950002020EBB29A42F9D904EB830331465869AF
:10B960000368DB6898470135F1E7000038B5054604
:10B970006C242B591BB1002128192DF085F87C343B
:10B98000B4F5F07FF5D138BD014B1868704700BFA2
:10B99000686100202DE9F04FB24BD3F800800446D7
:10B9A000D8F8040003688DB09B68984700250746C7
:10B9B0004FF0010909FA05F33B4240F0928201354C
:10B9C000202DF7D1D8F804000368DB6898470025DC
:10B9D00007464FF0010909FA05F33B4240F0C382E4
:10B9E0000135202DF7D1D8F8040003689B689847EB
:10B9F000002507464FF0010909FA05F33B4240F0E4
:10BA0000F1820135202DF7D1D8F8040003689B6836
:10BA10009847002507464FF0010909FA05F33B4214
:10BA200040F01C830135202DF7D1D8F80400DFF851
:10BA300040B203689B68984700250490049A01234C
:10BA4000AB40134240F046830135202DF6D1D8F8A3
:10BA50000400DFF81CB20368DB68984700250490F7
:10BA6000049A0123AB40134240F005840135202D98
:10BA7000F6D1D8F804000368DB689847002507462C
:10BA80004FF0010909FA05F33B4240F0BF8401354C
:10BA9000202DF7D1D8F804000368DB68984700250B
:10BAA00007464FF0010909FA05F33B4240F0ED84E7
:10BAB0000135202DF7D1D8F8040003689B6898471A
:10BAC000002507464FF0010909FA05F33B4240F013
:10BAD0001B850135202DF7D1D8F8040003689B6839
:10BAE0009847002507464FF0010909FA05F33B4244
:10BAF00040F04A850135202DF7D1D8F804000368BD
:10BB00009B689847002507464FF0010909FA05F39D
:10BB10003B4240F079850135202DF7D1D8F804005B
:10BB20000368DB689847002507464FF0010909FACA
:10BB300005F33B4240F0A4850135202DF7D14A4B57
:10BB4000089308AF0425D8F8040003689B68984759
:10BB5000002683460123B34013EA0B0F40F0CB8548
:10BB60000136202EF6D1D8F804000368DB68984728
:10BB7000002683460123B34013EA0B0F40F00186F1
:10BB80000136202EF6D1013D15F0FF0507F1010722
:10BB9000D9D1D8F8040003689B6898474FF0010991
:10BBA000074609FA05F33B4240F02F860135202D68
:10BBB000F7D1D8F804000368DB68984700250746EA
:10BBC0004FF0010909FA05F33B4240F05A8601356E
:10BBD000202DF7D1D8F8040003689B68984700250A
:10BBE00007464FF0010909FA05F33B4240F085860C
:10BBF0000135202DF7D1D8F804000368DB68984799
:10BC0000002507464FF0010909FA05F33B4240F0D1
:10BC1000B0860135202DF7D1144B0793D8F80400D6
:10BC200003689B689847002583460123AB4013EACD
:10BC30000B0F41D000275FFA85F9D4F8083313F4CD
:10BC4000803A31D107AB4946DB5D04931A46204662
:10BC5000FFF7EEFA049B0646002800F0C686CDE901
:10BC600008AA07E0F86000200C0D0E0F2021222307
:10BC7000801A0600099B0B93002201210BA8CDE935
:10BC8000092204F06FFF01462046FFF7C1FA0BA816
:10BC9000FDF7CEFE0AA8FDF7CBFE09A8FDF712FFBF
:10BCA00016B108A8FDF70EFF94F82330052B00F01D
:10BCB00048810137042FC0D10135202DB5D1D8F8E6
:10BCC00004000368DB689847002583460123AB40E6
:10BCD00013EA0B0F38D000275FFA85F9D4F8083340
:10BCE00013F4803A28D107AB4946DB5D04931A462A
:10BCF0002046FFF79DFA049B0646002800F0848644
:10BD0000CDE908AA0022099B0B9311460BA8CDE9A7
:10BD1000092204F027FF01462046FFF779FA0BA815
:10BD2000FDF786FE0AA8FDF783FE09A8FDF7CAFE07
:10BD300016B108A8FDF7C6FE94F82330052B00F0D5
:10BD400000810137042FC9D10135202DBED1D8F88B
:10BD5000040003689B689847002682460123B3408D
:10BD600013EA0A0F31D010255FFA86F9D4F80833A8
:10BD700013F0080B20D12A4649462046FFF758FA0F
:10BD80000746002800F04F86CDE909BB0A9B002238
:10BD900001210BA8CDE90A2301F048FC0146204609
:10BDA000FFF736FA0BA8FDF78DFE0AA8FDF78AFE0D
:10BDB00017B109A8FDF786FE94F82330052B00F093
:10BDC000C0800135EDB2142DD0D10136202EC5D161
:10BDD000D8F8040003689B68984700268246012330
:10BDE000B34013EA0A0F34D014255FFA86F9D4F869
:10BDF000083313F4001B24D12A4649462046FFF796
:10BE000017FA0746002800F02186CDE908BB099BF8
:10BE10000B93002201210BA8CDE9092202F018F8AA
:10BE200001462046FFF7F4F90BA8FDF701FE0AA82A
:10BE3000FDF7FEFD09A8FDF745FE17B108A8FDF7BF
:10BE400041FE94F82330052B7BD00135EDB2182D3F
:10BE5000CDD10136202EC2D1D8F804000368DB68AA
:10BE60009847002682460123B34013EA0A0F34D0D4
:10BE700014255FFA86F9D4F8083313F4001B24D193
:10BE80002A4649462046FFF7D3F90746002800F026
:10BE9000ED85CDE908BB0022099B0B9311460BA849
:10BEA000CDE9092201F0D4FF01462046FFF7B0F9A1
:10BEB0000BA8FDF7BDFD0AA8FDF7BAFD09A8FDF71F
:10BEC00001FE17B108A8FDF7FDFD94F82330052BFE
:10BED00037D00135EDB2182DCDD10136202EC2D18B
:10BEE0002FE0D4F8083313F0010A25D15FFA85FB5F
:10BEF0001E2259462046FFF79BF9064620B3CDE99E
:10BF000008AA099A0B920023082201210BA8CDE967
:10BF1000093303F0C7FA01462046FFF779F90BA869
:10BF2000FDF786FD0AA8FDF783FD09A8FDF7CAFD08
:10BF300016B108A8FDF7C6FD94F82330052B7FF451
:10BF40003EAD0DB0BDE8F08FD8F8041004220B68A8
:10BF5000CDE90102B84A0092D3F800A05A461E2348
:10BF600009A8D047CDE7D4F8083313F0010A24D14B
:10BF70005FFA85FB1E2259462046FFF759F906460F
:10BF800008B3CDE908AA099B0B93062200210BA850
:10BF9000CDE9091103F086FA01462046FFF738F98A
:10BFA0000BA8FDF745FD0AA8FDF742FD09A8FDF71E
:10BFB00089FD16B108A8FDF785FD94F82330052BFF
:10BFC0007FF40EADBDE7D8F8041004220B68CDE96C
:10BFD0000102994A0092D3F800A05A461E2309A8EC
:10BFE000D047D0E7D4F8083313F4805A21D15FFA50
:10BFF00085FB0D2259462046FFF71AF90646F0B197
:10C00000CDE909AA0A9B0022CDE90A2301210822D1
:10C010000BA804F0B5FA01462046FFF7F9F80BA883
:10C02000FDF750FD0AA8FDF74DFD16B109A8FDF773
:10C0300049FD94F82330052B7FF4E3AC81E7D8F871
:10C04000041004220B68CDE901027B4A0092D3F868
:10C0500000A05A460D230AA8D047D3E7D4F80833E6
:10C0600013F4801A21D15FFA85FB2C225946204611
:10C07000FFF7DEF80646F0B1CDE909AA0A9B0022D7
:10C08000CDE90A23012108220BA804F0A7FB0146F1
:10C090002046FFF7BDF80BA8FDF714FD0AA8FDF731
:10C0A00011FD16B109A8FDF70DFD94F82330052BFD
:10C0B0007FF4B8AC45E7D8F8041004220B68CDE94A
:10C0C00001025D4A0092D3F800A05A462C230AA828
:10C0D000D047D3E7D4F8083313F480773FD15FFA21
:10C0E00085F90C2249462046FFF7A2F806460028AB
:10C0F00000F08480CDE90677079B0A934FF0000A91
:10C10000692249462046CDF81CA0FFF791F8074662
:10C11000002800F08180CDE908AA099B0B9300223A
:10C120001A2309920BA901220AA801F007F8014677
:10C130002046FFF76DF80BA8FDF7C4FC09A8FDF732
:10C14000C1FC17B108A8FDF7BDFC0AA8FDF7BAFCB1
:10C1500007A8FDF7B7FC16B106A8FDF7B3FC94F8E5
:10C160002330052B3FF4EDAED4F8083313F4807779
:10C170007FF46AAC5FFA85F90C2249462046FFF746
:10C1800057F80646002859D0CDE90677079B0A9351
:10C190004FF0000A682249462046CDF81CA0FFF760
:10C1A00047F80746002857D0CDE908AA099B0B930A
:10C1B00000221A2309920BA901220AA800F0BEFF4F
:10C1C00001462046FFF724F80BA8FDF77BFC09A8E1
:10C1D000FDF778FC17B108A8FDF774FC0AA8FDF775
:10C1E00071FC07A8FDF76EFC16B106A8FDF76AFC06
:10C1F00094F82330052B7FF427ACA2E6D8F804107E
:10C2000004220B68CDF800B0CDE901024A461F6850
:10C2100007A80C23B8476FE7D8F8041004220B686E
:10C22000CDF800B0CDE901024A46D3F800A009A834
:10C230006923D04771E700BF801A0600D8F80410C0
:10C2400004220B68CDF800B0CDE901024A461F6810
:10C2500007A80C23B84799E7D8F8041004220B6804
:10C26000CDF800B0CDE901024A46D3F800A009A8F4
:10C270006823D0479AE7D4F8083313F480773DD188
:10C280005FFA85F90C2249462046FEF7D1FF0646A3
:10C29000002800F08180CDE90677079B0A934FF0D4
:10C2A000000A692249462046CDF81CA0FEF7C0FFCF
:10C2B000074600287ED0CDE908AA099B0B930022EF
:10C2C0001A230BA90AA8099200F038FF014620465C
:10C2D000FEF79EFF0BA8FDF7F5FB09A8FDF7F2FBA3
:10C2E00017B108A8FDF7EEFB0AA8FDF7EBFB07A8BE
:10C2F000FDF7E8FB16B106A8FDF7E4FB94F8233040
:10C30000052B3FF41EAED4F8083313F480777FF486
:10C31000ADAB5FFA85F90C2249462046FEF788FF4F
:10C320000646002855D0CDE90677079B0A934FF0C3
:10C33000000A682249462046CDF81CA0FEF778FF87
:10C340000746002853D0CDE908AA099B0B93002289
:10C350001A230BA90AA8099200F0F0FE0146204614
:10C36000FEF756FF0BA8FDF7ADFB09A8FDF7AAFBEA
:10C3700017B108A8FDF7A6FB0AA8FDF7A3FB07A8BD
:10C38000FDF7A0FB16B106A8FDF79CFB94F823303F
:10C39000052B7FF46BABD4E5D8F8041004220B68AE
:10C3A000CDF800B0CDE901024A461F6807A80C236A
:10C3B000B84772E7D8F8041004220B68CDF800B033
:10C3C000CDE901024A46D3F800A009A86923D04765
:10C3D00073E7D8F8041004220B68CDF800B0CDE95B
:10C3E00001024A461F6807A80C23B8479DE7D8F802
:10C3F000041004220B68CDF800B0CDE901024A46D2
:10C40000D3F800A009A86823D0479EE7D4F80833E2
:10C4100013F0200A24D15FFA85FB1C2259462046DE
:10C42000FEF706FF064608B3CDE908AA0022099BDD
:10C430000B9311460BA8CDE9092203F031FC01460C
:10C440002046FEF7E5FE0BA8FDF7F2FA0AA8FDF775
:10C45000EFFA09A8FDF736FB16B108A8FDF732FB85
:10C4600094F82330052B7FF412AB6AE5D8F804105A
:10C4700004220B68CDE90102B84A0092D3F800A06B
:10C480005A461C2309A8D047D0E7D4F8083313F044
:10C49000200A24D15FFA85FB1E2259462046FEF76A
:10C4A000C7FE064608B3CDE908AA0022099B0B93F4
:10C4B00011460BA8CDE9092203F0F2FB0146204604
:10C4C000FEF7A6FE0BA8FDF7B3FA0AA8FDF7B0FA2F
:10C4D00009A8FDF7F7FA16B108A8FDF7F3FA94F8E2
:10C4E0002330052B7FF4E4AA2BE5D8F804100422AE
:10C4F0000B68CDE90102994A0092D3F800A05A4690
:10C500001E2309A8D047D0E7D4F8083313F0200A37
:10C5100025D15FFA85FB1C2259462046FEF788FE8E
:10C52000064610B3CDE908AA099A0B92002302220D
:10C5300001210BA8CDE9093303F0B2FB01462046E7
:10C54000FEF766FE0BA8FDF773FA0AA8FDF770FA6E
:10C5500009A8FDF7B7FA16B108A8FDF7B3FA94F8E1
:10C560002330052B7FF4B5AAEBE4D8F8041004229D
:10C570000B68CDE90102794A0092D3F800A05A462F
:10C580001C2309A8D047CFE7D4F8083313F0200ABA
:10C5900025D15FFA85FB1E2259462046FEF748FE4C
:10C5A000064610B3CDE908AA099A0B92002302228D
:10C5B00001210BA8CDE9093303F072FB01462046A7
:10C5C000FEF726FE0BA8FDF733FA0AA8FDF730FAAE
:10C5D00009A8FDF777FA16B108A8FDF773FA94F8E1
:10C5E0002330052B7FF486AAABE4D8F8041004228C
:10C5F0000B68CDE90102594A0092D3F800A05A46CF
:10C600001E2309A8D047CFE7D4F8083313F0400A17
:10C6100021D15FFA85FB0C2259462046FEF708FE21
:10C620000646F0B1CDE909AA0A9B0022CDE90A230A
:10C63000012106220BA800F047FD01462046FEF727
:10C64000E7FD0BA8FDF73EFA0AA8FDF73BFA16B185
:10C6500009A8FDF737FA94F82330052B7FF45BAA7D
:10C660006FE4D8F8041004220B68CDE901023B4ABC
:10C670000092D3F800A05A460C230AA8D047D3E76B
:10C68000D4F8083313F0400A20D15FFA85FB0C225E
:10C6900059462046FEF7CCFD0646E8B1CDE909AA89
:10C6A00000220A9B11460BA8CDE90A2300F00CFDDD
:10C6B00001462046FEF7ACFD0BA8FDF703FA0AA8D9
:10C6C000FDF700FA16B109A8FDF7FCF994F823303C
:10C6D000052B7FF431AA34E4D8F8041004220B6847
:10C6E000CDE901021D4A0092D3F800A05A460C235E
:10C6F0000AA8D047D4E7D4F8083313F0800A26D12B
:10C700003B78F1B21A462046CDE90413FEF790FDBE
:10C71000DDE90413814618B3CDE909AA0A9B00227A
:10C72000CDE90A2301210C220BA803F087F9014669
:10C730002046FEF76DFD0BA8FDF7C4F90AA8FDF72A
:10C74000C1F9B9F1000F02D009A8FDF7BBF994F8BF
:10C750002330052B7FF404AAFFF7F3BB801A0600F1
:10C76000D8F80400B84AD0F800E000924FF0040C6A
:10C77000CDE9019C0A46DEF800A001460AA8D04790
:10C78000CCE7D4F8083313F0800A26D13B78F1B215
:10C790001A462046CDE90413FEF74AFDDDE90413ED
:10C7A000814608B3CDE909AA0A9B0022CDE90A23F4
:10C7B00000210C220BA803F041F901462046FEF7A8
:10C7C00027FD0BA8FDF77EF90AA8FDF77BF9B9F163
:10C7D000000F02D009A8FDF775F994F82330052B56
:10C7E0007FF4CEA9FFF7ADBBD8F80400964AD0F885
:10C7F00000E000924FF0040CCDE9019C0A46DEF8FF
:10C8000000A001460AA8D047CEE7D4F8083313F4B5
:10C81000004A20D15FFA85FB0C2259462046FEF7DC
:10C8200007FD0646F0B1CDE909AA0A9B00220121C5
:10C830000BA8CDE90A2302F077FF01462046FEF758
:10C84000E7FC0BA8FDF73EF90AA8FDF73BF916B186
:10C8500009A8FDF737F994F82330052B7FF4A6A932
:10C86000FFF76FBBD8F8041004220B68CDE9010272
:10C87000754A0092D3F800A05A460C230AA8D04764
:10C88000D3E7D4F8083313F4004A20D15FFA85FBCC
:10C890000C2259462046FEF7CBFC0646F0B1CDE906
:10C8A00009AA00220A9B11460BA8CDE90A2302F02F
:10C8B0003BFF01462046FEF7ABFC0BA8FDF702F953
:10C8C0000AA8FDF7FFF816B109A8FDF7FBF894F8E0
:10C8D0002330052B7FF47BA9FFF733BBD8F8041076
:10C8E00004220B68CDE90102574A0092D3F800A058
:10C8F0005A460C230AA8D047D3E7D4F8083313F4D8
:10C90000007A20D15FFA85FB302259462046FEF797
:10C910008FFC0646F0B1CDE909AA0A9B002201214D
:10C920000BA8CDE90A2303F087FC01462046FEF759
:10C930006FFC0BA8FDF7C6F80AA8FDF7C3F816B1FF
:10C9400009A8FDF7BFF894F82330052B7FF450A910
:10C95000FFF7F7BAD8F8041004220B68CDE90102FA
:10C96000394A0092D3F800A05A4630230AA8D0478B
:10C97000D3E7D4F8083313F4007A20D15FFA85FBAB
:10C98000302259462046FEF753FC0646F0B1CDE969
:10C9900009AA00220A9B11460BA8CDE90A2303F03D
:10C9A0004BFC01462046FEF733FC0BA8FDF78AF846
:10C9B0000AA8FDF787F816B109A8FDF783F894F8DF
:10C9C0002330052B7FF425A9FFF7BBBAD8F8041054
:10C9D00004220B68CDE901021B4A0092D3F800A0A3
:10C9E0005A4630230AA8D047D3E7D8F804100420C9
:10C9F0000A68CDE9016014480090D2F800A009A8A7
:10CA00004A46D047FFF736B9D8F8041004200A6820
:10CA1000CDE901600C480090D2F800A009A84A4670
:10CA2000D047FFF76FB9D8F8041004220B68CDE99E
:10CA30000102054A0092D3F800B04A462B460AA8E4
:10CA4000D847FFF7A3B900BF801A0600D8F8041032
:10CA500004220B68CDE901020C4A0092D3F800B021
:10CA60004A462B4609A8D847FFF7D1B9D8F8041091
:10CA700004220B68CDE90102044A0092D3F800B009
:10CA80004A462B4609A8D847FFF705BA801A060080
:10CA900073B50446FEF77EFF94F82330052B32D0A1
:10CAA000002594F83F33EB40DA07E9B216D401359C
:10CAB000082DF6D194F82330052B24D094F820309B
:10CAC00013B194F82230F3B9104B11491B689869DF
:10CAD00003681B6802B0BDE870401847D4F80833FB
:10CAE0009B030CD42C200191FEF7D6F9064610B119
:10CAF000019903F019FC31462046FEF789FB94F8B2
:10CB00002330052BD3D102B070BD00BFF8600020E8
:10CB10008C0A0A082DE9F04F90F9213089B00446BB
:10CB2000002B00F00481012300F50C7580F84133DF
:10CB3000024600F50F712B462E46D06E002859D0C4
:10CB4000002384F8413394F94030642B5BD094F98E
:10CB5000BC30642B00F08D8094F93831642B00F0E8
:10CB60008A80D4F830722FBB01A920462BF070FFC9
:10CB700000B30C230593012306978DF81830714BF1
:10CB800007936946BDF80430049704A8ADF8103047
:10CB90008DF800702CF0DCF89DF9001051B10229DD
:10CBA00008DC38B1C9B27C2303FB01416C31284653
:10CBB0002DF0A6FC94F841B3BBF1000F5DD0E36EFD
:10CBC0006367D4F8E830C4F8F030D4F86431C4F8BE
:10CBD0006C3194F8233003F1C30204EB820200218C
:10CBE000042B7CD852F8040B1061013342F8041C6A
:10CBF000DBB2F5E753F8040B0028A1D18B4202F118
:10CC00007C029AD19FE7002066238DF810307C23A8
:10CC100003FB004004A940302DF0B6FB04A92046D8
:10CC20002BF016FF00289CD004238DF81830002329
:10CC3000CDE90133039331230593694604A82CF011
:10CC400087F8059B28B108AA02EB8302009942F8F5
:10CC5000E01C0133332B0593EFD950F03DF99DEDE6
:10CC6000031ADDED020A9DED010A662150F0F2F88B
:10CC700077E70120C8E70220C6E70127A94655F853
:10CC8000043B23B1AB600137042FF7D197E7AA46E5
:10CC9000B8465FFA88F3022BF5D8DAF8002055F889
:10CCA000043C9A4205D104A95046CDF810B02DF0AD
:10CCB00027FC5AF8043B08F101020BB99046E8E75B
:10CCC00004A906EB88000193CDF810B02DF018FCF4
:10CCD000019BAB6001A948462DF012FCD3E794F804
:10CCE000413313B92046FEF79FF994F822300BB375
:10CCF000154B1B68986A036864215B689847204657
:10CD0000FEF752FD94F83E3003B9E36694F8BA306A
:10CD10000BB9C4F8E83094F836310BB9C4F8643173
:10CD2000FAF722FAFAF7ECFA0123A4F8403309B033
:10CD3000BDE8F08F2046FFF7ABFE94F82230002BC1
:10CD4000E0D0D5E7B0A40A08F860002070470000E2
:10CD500001207047012070474368986870470000C1
:10CD600010B5054B03600446806A10B103685B6828
:10CD70009847204610BD00BF4C0F0A084068036862
:10CD80005B6A184733B46C46406884E80C0003685B
:10CD90009D6A94E80C00AC4602B030BC60470000CD
:10CDA00010B50446FFF7DCFF2046FEF77DF820466D
:10CDB00010BD000040680BF003BA0000406801237A
:10CDC0000BF0FEB940680BF0D7B9000040680A22AA
:10CDD0000BF07CB940680BF091B9000040680BF093
:10CDE00013BA000090F82E2022B190F82D100022E6
:10CDF00001F06EB97047000073B5044605250026A2
:10CE0000A06A8DF8076003680DF10702DB68012155
:10CE1000984778B19DF807300C2B09D0102B05D01E
:10CE2000092B07D184F8303002B070BD1523F9E723
:10CE30001423F7E7013DE3D12846F5E710B4806AF3
:10CE400003681C690822A44601235DF8044B3121C4
:10CE50006047000010B4806A03681C690122A44680
:10CE600000235DF8044B322160470000F0B5044612
:10CE7000806A036885B05B6998470546002800F022
:10CE80008480A06A03685B69984703689B68984739
:10CE9000A06A03689B69984760B93D4B3D491B6890
:10CEA000986903681B6898472B682846DB68984791
:10CEB000002667E02046FFF7CDFF0028F4D020468B
:10CEC000FFF79AFF0028EFD0A06A03680121DB6A10
:10CED00098472046FFF7B2FF30B92D4B2E491B680B
:10CEE000986903681B68DEE7A06A0368DB699847F6
:10CEF00030B9274B29491B68986903681B68D2E73A
:10CF0000A06A94F83010012784F82E7003685B6AD9
:10CF10009847A06A03689B6A984704F12D0201466E
:10CF2000204601F023F906460028BDD0A06A94F8F7
:10CF30002D10036801919B6A98470199024620468B
:10CF400001F018F994F82C302BB194F82D103A46D2
:10CF5000204601F023F994F82F2094F82D10204654
:10CF600001F03EF92B682846DB689847A06A0294D6
:10CF700003681D6A0A4B039304AB13E90C0042F2E9
:10CF80001071A847304605B0F0BD0646FAE700BF6D
:10CF9000F8600020B80E0A08DE0E0A08FD0E0A0826
:10CFA00099D0010870B5002586B0CDE90055002361
:10CFB0000446806A8DF80850059303930493036830
:10CFC0006A469E6810210923B047A0B19DF8003041
:10CFD00013F0010615D194F831300133DBB2052B83
:10CFE00084F8313007D12046FFF734FF2046FFF7A1
:10CFF00025FF84F83160A06A03681B6B984706B070
:10D0000070BD9DF8083084F831501B07F3D4BDF98A
:10D0100001309FED1F6A06EE903ABDF9033007EE2E
:10D02000103ABDF90530F8EEE66A07EE903ACDED1C
:10D03000036AF0EEE66AB8EEC77AF8EEE77AF4EE45
:10D04000C66AF1EE10FA8DED047ACDED057A0DD5B4
:10D05000B0EEC77AB4EEC67AF1EE10FA06D5F0EE6D
:10D06000E77AF4EEC67AF1EE10FAC4D49FED090A1D
:10D0700003A811F059FCB2EE040A03A811F054FC05
:10D0800094F82D200A2303A9204601F00FF9B2E7F6
:10D09000000000349A99193EFFF784BF10B5044B85
:10D0A000044640F8043BFCF70DFD204610BD00BFD0
:10D0B000640F0A0810B50446FFF7F0FF2046FDF79D
:10D0C000F3FE204610BD0000F7B503680F46164674
:10D0D0001BB90024204603B0F0BD002404600820E2
:10D0E0000193FDF7D9FE054620B1124B0360019B69
:10D0F0004360019401A8FCF7E5FC002DE9D0342041
:10D10000FDF7CAFE04460028E3D000F0E1FE0A4B1A
:10D11000A562236084F82C7084F82F602046FFF706
:10D12000A5FE05460028D5D1236820465B689847B0
:10D130002C46CFE7640F0A084C0F0A082DE9F74F79
:10D14000046806460D4690469946002C6CD00B6844
:10D15000002B49D0236820465B6A984703689B6888
:10D160009847012328680DEB030200210BF028F8F3
:10D1700098B39DF80130EA2B2FD1DFF8F0B04FF0D3
:10D18000060A28680023802206210AF0F5FF20B352
:10D19000DBF80070B86A03680A215B6898470023CF
:10D1A00028681A4606210AF0E7FFB0B1B86A03689A
:10D1B0000A215B689847012328680DEB03020621CA
:10D1C0000AF0FEFF48B19DF8014014F040042FD052
:10D1D0000AF1FF3A1AF0FF0AD3D1306803685B6A9C
:10D1E00098470368DB68984700241DE00222234625
:10D1F0000F2128680AF0C0FFB86A036801215B6844
:10D200009847306803685B6A98470368DB6898470B
:10D21000336834604A46414601A80193FFF754FF42
:10D22000044601A8FCF74EFC204603B0BDE8F08F91
:10D23000224623460F2128680AF09EFFB86A036839
:10D2400001215B6898470223214630680DEB0302F9
:10D250000AF0B6FF04460028C8D0B869024903683E
:10D260001B689847B9E700BF240F0A08F860002040
:10D2700090F82C10002200F02BBF000070B504467F
:10D280008CB00426013E76B2731C4AD0A06A1523E6
:10D290006A465D210AF094FF0028F3D0A06A1523A6
:10D2A00006AA5D210AF08CFF05460028EAD0152267
:10D2B00006A9684679F086FE0028E3D19DF8003083
:10D2C00084F82E309DF8073084F830309DF8143003
:10D2D00084F83A309DF813309DF8102084F83B30E4
:10D2E0009DF80F3043EA0223A3879DF8013084F8AC
:10D2F0002F309DF8083084F83130039B9DF80C20C6
:10D30000C3F30F2363869DF80B3043EA0223A38601
:10D31000049BC3F30F23E386019BC3F30F232387EF
:10D3200007E0054B05491B68986903681B68984727
:10D33000002528460CB070BDF8600020980F0A0840
:10D340002DE9FF4104460023806A8DF80730036809
:10D35000DFF868815B6A984703689B689847A06A12
:10D3600003680A219B6C9847A06A0A2204210AF0EC
:10D37000ADFE0425013D6DB26B1C32D000234B2164
:10D38000A06A82220AF0F8FED8F800600746B06A68
:10D39000036802215B689847002FEBD001231A46EF
:10D3A0004B21A06A0AF0E8FE0746B06A0368022132
:10D3B0005B689847002FDDD0A06A01230DF10702BA
:10D3C00040210AF0FDFE0028D4D09DF80720322A23
:10D3D00010D0002DCED1B069364903681D683223C4
:10D3E000A847A06A03685B6A98470368DB689847A8
:10D3F00000255BE02046FFF741FF0028F1D0A06A3E
:10D400000123172251210AF0B7FE0028E9D0522249
:10D41000A06A012311460AF0AFFE0028E1D0A06AFD
:10D42000012338224C210AF0A7FE0028D9D0A06A97
:10D4300003685B6A98470368DB689847A06A052120
:10D440000AF05CFEA36A04F12C029968204600F001
:10D450008DFE054650B3A36A94F82C109A682046B6
:10D4600000F088FE94F8442094F82C10204600F038
:10D47000B7FE94F845302BB194F82C1001222046C9
:10D4800000F08CFEA06A036802219B6C9847A06A9A
:10D49000029403689E6A084B039304AB13E90C00E3
:10D4A00044F21B11B04752F06BF92064284604B0D7
:10D4B000BDE8F081C00F0A0829D60108F8600020F5
:10D4C00070B5858F90F93B60AD03B5FBF2F2A2F524
:10D4D000804404FB04F2D51190F83A200498D2015C
:10D4E000624306FB05225212A03002F5801242432D
:10D4F00012134A43DB0003EB623000B270BD000040
:10D5000010B5448E53005C43B0F93830C91A838F8C
:10D51000D31AB0F93620B0F93400534304F500446F
:10D520009B10C3EBC13300EB2440044993FBF0F0A4
:10D530004FF400420FF08EF800B210BD0080FFFFE4
:10D5400010B52DED028B8AB004460823806A05AA27
:10D5500042210AF035FE18B1BDF81A20D30719D4BC
:10D56000A06A0AF051FE52F00BF9236CC31AFA2B91
:10D570000CD92064002382224B21A06A0AF0FCFD12
:10D580000123A06A1A464B210AF0F6FD0AB0BDEC51
:10D59000028B10BDBDF9141094F93030009392083D
:10D5A00094F92E300392C9102046FFF789FFBDF988
:10D5B000161094F93130039A009308EE900A94F90A
:10D5C0002F30C9102046FFF77BFFBDF91810039AD2
:10D5D000491008EE100A2046FFF792FF07EE900A66
:10D5E000F8EEE88AF8EEE77AB8EEC88AB3EE000AF9
:10D5F00007A8CDED097ACDED078A8DED088A11F0E7
:10D60000A7F9B2EE040A07A811F08EF952F0B8F8A3
:10D6100094F82C2020640A23204607A900F046FE37
:10D62000A06A0AF0F1FDB1E7FFF78ABFF7B503681A
:10D630000D4616461BB90024204603B0F0BD002756
:10D6400007604820CDE90073FDF726FC044650B181
:10D6500000F03EFC0E4B2360019BA362019784F80F
:10D66000446084F8455001A8FCF7E2F96846FCF7ED
:10D67000DFF9002CDFD02046FFF762FE05460028C8
:10D68000DAD1236820465B6898472C46D4E700BF70
:10D69000F80F0A0810B5044B044640F8283BFCF785
:10D6A000C7F9204610BD00BFF80F0A0810B50446A0
:10D6B000FFF7F0FF2046FDF7F7FB204610BD000006
:10D6C00090F82C10002200F003BD0000F8B50446CD
:10D6D0000D4617461E4600F0FBFB094B23602B68E6
:10D6E000A362002200232A6084F82D7084F82E6043
:10D6F00023656365A365E365236663662046F8BD1D
:10D7000010100A08F8B51C4609331646DB086A46AD
:10D71000A2EBC30300AF9D46806AA31C6A460AF0D1
:10D720004FFD054628B122460DF10201304679F041
:10D7300059FC2846BD46F8BD2DE9F34106460F4683
:10D74000144652F01DF8114BD3F800800546D8F866
:10D750002800036801215B68984701230DF1070247
:10D7600007213046FFF7CEFF60B19DF80730DA079A
:10D7700002D4B7EB531F05D052F002F8431BA3426B
:10D78000E5D3002002B0BDE8F08100BFF8600020C2
:10D790002DE9F041DFF8608292B0044602AF002626
:10D7A00046F02002A06A0023D2B250210AF0E4FC25
:10D7B000002800F00C810325013D6DB26A1C00F0C9
:10D7C0000681D8F80030986A03684FF496719B6818
:10D7D000984701230DF1060255212046FFF792FFDD
:10D7E000002800F0F4809DF8063013F0E00F40F0C0
:10D7F000EE80DB07E0D502230DF106025221204620
:10D80000FFF780FF002800F0E280BDF80630013607
:10D810005BBA202E27F8023BC2D1BDF824309DF818
:10D8200026109FED6D7ADFED6D6A9FED6D6A43F313
:10D830000B0207EE902A1B0903F47063BDF8262043
:10D84000F8EEE77A0B4343F30B03C4ED0C7A07EED3
:10D85000903A02F470639DF82820F8EEE77A1343BB
:10D8600043F30B03C4ED0D7A07EE903A9DF9223095
:10D87000F8EEE77AC4ED0E7A07EE903A9DF929307A
:10D88000F8EEE77A67EE877A07EE103AB8EEC77AD5
:10D890009DF92A30C4ED0F7A27EE267ADFED517A12
:10D8A00084ED107A07EE103AB8EEC77A9DF92B3066
:10D8B000E7EE267AC4ED117A07EE903AF8EEE77AB1
:10D8C0009DF9233067EEA67ADFED476AC4ED127A40
:10D8D00007EE903A9DF92C3007EE103AB8EEC77A71
:10D8E0009DF92E3027EE267AF8EEE77A84ED147A49
:10D8F00067EE867A07EE103A9DF93030C4ED137A60
:10D9000007EE903AF8EEE77A9DF92D3067EEA67AA9
:10D91000B8EEC77AC4ED167A27EE267A07EE903A6B
:10D9200084ED157AF8EEE77A9FED307A9DF92F3085
:10D9300067EE877AC4ED177A07EE903A9DF9313099
:10D94000F8EEE77A06EE903A67EE877AF8EEE66A46
:10D95000C4ED187ADFED267ABDF93830E6EE877A25
:10D9600007EE103A9DF93230C4ED197AB8EEC77A55
:10D97000F3EE077AE7EE067A07EE103ADFED1D6A5E
:10D98000C4ED1A7AB8EEC77A27EE267A84ED1B7AB0
:10D990009DF9333007EE103AB8EEC77A9DF934306E
:10D9A00027EE267A84ED1C7A07EE103A9DF9353081
:10D9B00007EE903AB8EEC77AF8EEE77A27EE267AC5
:10D9C00067EEA67A84ED1D7AC4ED1E7A00E0002091
:10D9D00012B0BDE8F08100BFCDCC4C3E0000803BD2
:10D9E0000000003B0AD7233C0000003D00008038C7
:10D9F00017B7D1B80AD7A33AF860002073B501234E
:10DA00000E460DF1070206210446FFF77BFE18B90A
:10DA10000025284602B070BD9DF80730013B012B60
:10DA20000CD80023A06A1A4606210AF0A5FB00289C
:10DA3000EED0062200212046FFF77EFEA06A0023DA
:10DA4000324606210AF098FB05460028E0D026223F
:10DA500031462046FFF770FEDBE7000013B50123D7
:10DA60000DF1070207210446FFF74CFE10B9002014
:10DA700002B010BD9DF807301B070CD50023A06A2B
:10DA80001A4606210AF078FB0028F0D00622002171
:10DA90002046FFF751FEA06A0023072206210AF064
:10DAA0006BFB0028E3D0132207212046FFF744FE3A
:10DAB0000028DCD0A06A0023052206210AF05CFBC6
:10DAC0000028D4D0172205212046FFF735FE002874
:10DAD000CDD001212046FFF791FFC9E7F7B50446F5
:10DAE000806A5B4F03685B6A984703689B68984746
:10DAF000A06A03680A219B6C9847A06A0A22042145
:10DB00000AF0E4FA0525013D6DB26B1C00F0968029
:10DB1000A06A0023B6227E210AF02EFB0028F2D054
:10DB20003B68986A036818215B686E469847012332
:10DB3000324600212046FFF7E5FD0028E3D09DF89E
:10DB40000030332BDFD12046FFF722FE002875D0AE
:10DB5000A06A0023802250210AF00EFB00286DD01D
:10DB60002046FFF77BFF002868D0A06A00238622AA
:10DB70002E210AF001FB002860D0A06A0023242295
:10DB800004210AF0F9FA002858D0A06A00230222E2
:10DB900006210AF0F1FA002850D014220221204672
:10DBA000FFF7CAFDA06A0023072205210AF0E4FA64
:10DBB000002843D001212046FFF720FF00283DD058
:10DBC000A06A036803219B6C9847A06A03685B6A9C
:10DBD00098470368DB689847A06A17210AF08EFA15
:10DBE000A36A04F12C029968204600F0BFFA0546AA
:10DBF00008B3A36A94F82C109A68204600F0BAFA89
:10DC000094F82E2094F82C10204600F0E9FA94F8AD
:10DC10002D302BB194F82C100122204600F0BEFAD2
:10DC2000A06A03689F6A0B4B0094019396E80C006E
:10DC300042F21071B847284603B0F0BDA06A0368ED
:10DC40005B6A98470368DB6898470025F3E700BFE5
:10DC5000F86000204DDE010810B586B00C236A463E
:10DC600031210446FFF74EFD002800F0DF809DF8CB
:10DC700001309DF80020DFED717ADFED715A1B0451
:10DC800003EB02239DF8022003EB02631B1206EE56
:10DC9000903A9DF804309DF803201B0403EB022307
:10DCA0009DF8052003EB02631B1207EE103A9DF866
:10DCB00007309DF806201B0403EB02239DF8082083
:10DCC00003EB02631B1206EE103A9DF80A309DF832
:10DCD00009201B0403EB0223F8EEE66AB8EEC77ACC
:10DCE0009DF80B2066EEA76A27EE277AB8EEC66A83
:10DCF000DFED547A03EB02631B1226EE276A07EE70
:10DD0000903AF8EEE77A67EEA57AF5EEC07AF1EE92
:10DD100010FA40F38D80DFED4C5A77EEE57AD4EDC2
:10DD2000134A94ED0F5A94ED1C4AD4ED1D3A94F821
:10DD30002C20F7EE005A74EEA54AF0EE632AA4EE0A
:10DD4000A75A0A2303A9D4ED107AD4ED0C4A77EE32
:10DD5000A57A2046E7EEA64AD4ED1A7A75EE677AE0
:10DD600094ED145AF0EE646AD4ED174AE5EE276A92
:10DD7000B0EE655AA7EEA45AC6EE854A94ED115A44
:10DD8000D4ED0D6A35EE255AE5EE076A94ED157A65
:10DD9000E7EE876A94ED187AB0EE655AA7EE875AD7
:10DDA00086EE857A94ED125AD4ED0E6A35EE255A38
:10DDB000E5EE066A94ED166A94ED195AE7EE866A66
:10DDC000B0EE656AA7EE856AF0EE657A86EE863A71
:10DDD00094ED1B6AF0EE646AE6EE447AE6EE476A7A
:10DDE00086EEA75AF0EE476AE4EE646AC6EEA75ADA
:10DDF000D4ED1E6AD4EE262AE6EE636AB2EE046A19
:10DE000027EE667A65EE066AA2EEA47ACDED036A85
:10DE100065EE866ACDED046AC7EE276A76EE837AF0
:10DE200067EE867ACDED057A00F040FA06B010BDB7
:10DE300044BFDFED055A77EEA57A70E747ABE73BC5
:10DE40005B9E803AF61BEB3B85EBCB41FFF704BFB3
:10DE500030B51346026885B00D461AB90024204635
:10DE600005B030BD002101607C2001930392FDF7D5
:10DE700013F8044620B1019B2A4603A9FFF726FCAC
:10DE800003A8FBF7D5FD002CE8D02046FFF726FEBF
:10DE900005460028E3D1236820465B6898472C4656
:10DEA000DDE7000010B5044B044640F8283BFBF7C3
:10DEB000BFFD204610BD00BF10100A0810B5044673
:10DEC000FFF7F0FF2046FCF7EFFF204610BD0000F3
:10DED000064B10B503600446FDF756FD606004F183
:10DEE000080050F003FE204610BD00BF28100A08AD
:10DEF00073B50646144675687C2303FB0253C4EBD6
:10DF0000441405EB8404084693F8A410019010F023
:10DF1000A1FD94F93C3001983BB9736893F8251042
:10DF200002B0BDE8704010F095BD94F84010F7E7DE
:10DF300037B5446801917C2505FB024595F83F30D3
:10DF400004EB8304D4F84C325BB151F019FCC5F8F2
:10DF50009C000199D4F84C0203B0BDE8304003F0B6
:10DF6000A7BF03B030BD00002DE9F04FC2EB421453
:10DF700047684FEA840881460E4607F13C0B08F1DA
:10DF800008018BB015465944304610F099FCD9F879
:10DF9000040029460BEB8404FDF79CFC38B17C237C
:10DFA00003FB057393ED1A0A304610F0BDFC7C2389
:10DFB00003FB057393ED146ADFED3A7AD3ED156A2E
:10DFC000B0EEC67AB4EEE77AF1EE10FA0FD5B0EE05
:10DFD000E67AB4EEE77AF1EE10FA08D594ED077A16
:10DFE000B0EEC77AB4EEE77AF1EE10FA1BD47C23D8
:10DFF00003FB0573D86D196E5A6E9B6D02900391E9
:10E000000490079101A831468DED016ACDED056AB6
:10E010000692089209930EF01BFD86ED000AC6EDEC
:10E02000010A86ED021A7C2303FB05770023C7F85B
:10E030008C30C7F88830C7F88430D9F8040090F9DC
:10E040005C3208F13C0A08F14808DA44D84463B16C
:10E050005DB9414600F5167004F0E2FB41463046DA
:10E060000BB0BDE8F04F10F02BBC90F93430012B11
:10E070000BD190ED0E0A504610F002FC84ED120A0E
:10E08000C4ED130A84ED141AE8E7022BE6D1FCF77D
:10E0900041FB002201A9FCF70BF80028DED09DED22
:10E0A000010AE8E70000003410B543687C2404FB53
:10E0B000023407C904F1900383E8070051F060FBC4
:10E0C000C4F89C0051F050FBC4F8A00010BD000043
:10E0D000F0B5074685B00D46164600F10801A922A5
:10E0E00003A80AF0C7FA7C687C2303FB0543D3F836
:10E0F000B42022B903A80AF0DFFA05B0F0BDBEB122
:10E1000096ED007AD3ED2A7A67EE877AC3ED2A7A04
:10E1100096ED017AD3ED2B7A67EE877AC3ED2B7AF1
:10E1200096ED027AD3ED2C7A67EE877AC3ED2C7ADE
:10E130007C2607EE902A06FB0541A831B8EE670A57
:10E140000846019110F004FC01992A463846FFF771
:10E15000ABFF06FB05410023C1F8B030C1F8AC307D
:10E16000C1F8A8300023C1F8B430C3E74068FCF719
:10E17000ABBF0000F7B50646406801927C2707FB5D
:10E1800001000D466C3001A914462CF099F9716814
:10E1900007FB05152C6703B0F0BD000007B540680C
:10E1A0007C2303FB010393F93C30022B0BD000F1DD
:10E1B0003C03C1EB411003EB80000DF107018DF82A
:10E1C00007202CF0D7F803B05DF804FB43687C22ED
:10E1D00002FB013191F93C00003818BF0120704763
:10E1E00043687C2000FB013181F8A42070470000C7
:10E1F000F8B5054608460F4610F008FC10B100249B
:10E200002046F8BD384610F0E7FB04460028F6D15A
:10E210006B6893F934637EB1384610F02FFF95EDAB
:10E22000087ADFED1F7AF0EEC76AF4EEE76AF1EEE6
:10E2300010FA03D585ED080A0124E1E777EE407A6C
:10E2400030EE076AF0EEE77AC7EE866AF6B207EEBE
:10E25000906A9FED146AF8EE677A26EE866AF4EE0D
:10E26000C67AF1EE10FA48BFB2EE046ADFED0E7A1C
:10E2700045BF6B6A66EE866AB0EE676A87EEA66A8D
:10E2800046BF01336B620124F7EE007A77EEC67A5F
:10E2900020EE060AA7EE270A85ED080AB0E700BFC0
:10E2A0000000003400004843CDCCCC3D2DE9F743BD
:10E2B00004460E4615461F46FFF71AFE2A4631460B
:10E2C0002046FFF735FE314620462A46FFF74CFE32
:10E2D00031462046FFF78CFF28B39B2204F108014A
:10E2E00001A80AF0C7F964684FF07C0909FB0548EA
:10E2F00008F1A8083146404610F0E2FA09FB054251
:10E30000D2F8B4100131C2F8B4104FB1B94207D3FA
:10E310004908C2F8B410B0EE000A404610F018FBED
:10E3200001A80AF0C9F903B0BDE8F08310B50446AE
:10E33000FCF754FFC0B23C34C0EB401004EB80004B
:10E3400010BD0000F8B50A4E044600F5167704F536
:10E35000137555F8040B08B104F0DEF8BD42F8D18E
:10E360003368986A036801215B689847EFE700BF4C
:10E37000F860002008B5FFF7E5FF0000F0B5144E87
:10E3800000EB810773780446D7F84C026FF3410322
:10E3900087B00D467370C8B102F0ACFC68B17378F9
:10E3A00043F0100373702C440023A372D7F84C027F
:10E3B00007B0BDE8F04002F021BCD7F84C12684627
:10E3C00002F0C8FC009B012BEDD1E8E707B0F0BDDF
:10E3D000A461002070B506460D46002445FA04F3FA
:10E3E000DB07E1B202D53046FFF7C8FF0134032C4A
:10E3F000F4D170BDFF21FFF7EDBF000030B500F58F
:10E40000137587B000F5167455F8041B21B9A542A1
:10E41000FAD1002007B030BD684602F09BFC009B9B
